 gor4

 Timestamp is 5c7621b4 (Wed Feb 27 12:35:48 2019)

 Preferred load address is 10000000

 Start         Length     Name                   Class
 0001:00000000 00001524H .text$di                CODE
 0001:00001530 00005bd8H .text$mn                CODE
 0001:00007110 00000a64H .text$x                 CODE
 0001:00007b80 0000051aH .text$yd                CODE
 0002:00000000 00000258H .idata$5                DATA
 0002:00000258 00000004H .CRT$XCA                DATA
 0002:0000025c 00000118H .CRT$XCU                DATA
 0002:00000374 00000004H .CRT$XCZ                DATA
 0002:00000378 00000004H .CRT$XIA                DATA
 0002:0000037c 00000004H .CRT$XIAA               DATA
 0002:00000380 00000004H .CRT$XIC                DATA
 0002:00000384 00000004H .CRT$XIZ                DATA
 0002:00000390 0001a850H .rdata                  DATA
 0002:0001abe0 0000006cH .rdata$debug            DATA
 0002:0001ac4c 00000464H .rdata$r                DATA
 0002:0001b0b0 000000ccH .rdata$sxdata           DATA
 0002:0001b17c 00000004H .rtc$IAA                DATA
 0002:0001b180 00000004H .rtc$IZZ                DATA
 0002:0001b184 00000004H .rtc$TAA                DATA
 0002:0001b188 00000004H .rtc$TZZ                DATA
 0002:0001b190 00000ce4H .xdata$x                DATA
 0002:0001be80 0000004dH .edata                  DATA
 0002:0001bed0 000000a0H .idata$2                DATA
 0002:0001bf70 00000014H .idata$3                DATA
 0002:0001bf84 00000258H .idata$4                DATA
 0002:0001c1dc 00001410H .idata$6                DATA
 0003:00000000 00000124H .data                   DATA
 0003:00000124 00000234H .data$r                 DATA
 0003:00000358 002c817cH .bss                    DATA
 0004:00000000 00000058H .rsrc$01                DATA
 0004:00000060 00000180H .rsrc$02                DATA

  Address         Publics by Value              Rva+Base       Lib:Object

 0000:00000000       __except_list              00000000     <absolute>
 0000:00000000       ___guard_fids_count        00000000     <absolute>
 0000:00000000       ___guard_flags             00000000     <absolute>
 0000:00000000       ___guard_fids_table        00000000     <absolute>
 0000:00000033       ___safe_se_handler_count   00000033     <absolute>
 0000:00009876       __fltused                  00009876     <absolute>
 0000:00009876       __ldused                   00009876     <absolute>
 0000:00000000       ___ImageBase               10000000     <linker-defined>
 0001:00001530       ??$_Allocate@D@std@@YAPADIPAD@Z 10002530 f i GorIVAlgTask.obj
 0001:00001560       ??$_Move@AAPAUData@QListData@@@std@@YA$$QAPAUData@QListData@@AAPAU12@@Z 10002560 f i GorIVAlgTask.obj
 0001:00001570       ??$addressof@D@std@@YAPADAAD@Z 10002570 f i GorIVAlgTask.obj
 0001:00001580       ??$atomic@H@?$QAtomicOpsBySize@$03@@CAPAJPAH@Z 10002580 f i GorIVAlgTask.obj
 0001:00001590       ??$construct@PADAAPAD@?$_Wrap_alloc@V?$allocator@D@std@@@std@@QAEXPAPADAAPAD@Z 10002590 f i GorIVAlgTask.obj
 0001:000015b0       ??$construct@PADAAPAD@?$allocator@D@std@@QAEXPAPADAAPAD@Z 100025b0 f i GorIVAlgTask.obj
 0001:000015d0       ??$construct@PADAAPAD@?$allocator_traits@V?$allocator@D@std@@@std@@SAXAAV?$allocator@D@1@PAPADAAPAD@Z 100025d0 f i GorIVAlgTask.obj
 0001:000015f0       ??$deref@H@?$QAtomicOpsBySize@$03@@SA_NAAH@Z 100025f0 f i GorIVAlgTask.obj
 0001:00001610       ??$destroy@PAD@?$_Wrap_alloc@V?$allocator@D@std@@@std@@QAEXPAPAD@Z 10002610 f i GorIVAlgTask.obj
 0001:00001620       ??$destroy@PAD@?$allocator@D@std@@QAEXPAPAD@Z 10002620 f i GorIVAlgTask.obj
 0001:00001630       ??$destroy@PAD@?$allocator_traits@V?$allocator@D@std@@@std@@SAXAAV?$allocator@D@1@PAPAD@Z 10002630 f i GorIVAlgTask.obj
 0001:00001640       ??$forward@AAPAD@std@@YAAAPADAAPAD@Z 10002640 f i GorIVAlgTask.obj
 0001:00001650       ??$load@H@?$QGenericAtomicOps@U?$QAtomicOpsBySize@$03@@@@SAHABH@Z 10002650 f i GorIVAlgTask.obj
 0001:00001660       ??$qSwap@PAUData@QListData@@@@YAXAAPAUData@QListData@@0@Z 10002660 f i GorIVAlgTask.obj
 0001:00001680       ??$swap@PAUData@QListData@@@std@@YAXAAPAUData@QListData@@0@Z 10002680 f i GorIVAlgTask.obj
 0001:000016a0       ??0?$AbstractId@H@U2@@IAE@ABH@Z 100026a0 f i GorIVAlgTask.obj
 0001:000016c0       ??0?$QFlags@W4OpenModeFlag@QIODevice@@@@QAE@W4OpenModeFlag@QIODevice@@@Z 100026c0 f i GorIVAlgTask.obj
 0001:000016d0       ??0?$_String_alloc@$0A@U?$_String_base_types@DV?$allocator@D@std@@@std@@@std@@QAE@ABV?$allocator@D@1@@Z 100026d0 f i GorIVAlgTask.obj
 0001:000016f0       ??0?$_String_val@U?$_Simple_types@D@std@@@std@@QAE@XZ 100026f0 f i GorIVAlgTask.obj
 0001:00001710       ??0?$_Wrap_alloc@V?$allocator@D@std@@@std@@QAE@XZ 10002710 f i GorIVAlgTask.obj
 0001:00001720       ??0?$allocator@D@std@@QAE@XZ 10002720 f i GorIVAlgTask.obj
 0001:00001730       ??0?$basic_string@DU?$char_traits@D@std@@V?$allocator@D@2@@std@@QAE@PBD@Z 10002730 f i GorIVAlgTask.obj
 0001:00001790       ??0AbstractInt32Id@U2@@IAE@H@Z 10002790 f i GorIVAlgTask.obj
 0001:000017b0       ??0GorIVAlgTask@U2@@QAE@ABVQByteArray@@@Z 100027b0 f   GorIVAlgTask.obj
 0001:000018a0       ??0ServiceType@U2@@QAE@H@Z 100028a0 f i GorIVAlgTask.obj
 0001:000018c0       ??0_Generic_error_category@std@@QAE@XZ 100028c0 f i GorIVAlgTask.obj
 0001:000018d0       ??0_Ignore@std@@QAE@XZ     100028d0 f i GorIVAlgTask.obj
 0001:000018e0       ??0_Iostream_error_category@std@@QAE@XZ 100028e0 f i GorIVAlgTask.obj
 0001:000018f0       ??0_System_error_category@std@@QAE@XZ 100028f0 f i GorIVAlgTask.obj
 0001:00001900       ??0error_category@std@@QAE@XZ 10002900 f i GorIVAlgTask.obj
 0001:00001910       ??0error_condition@std@@QAE@HABVerror_category@1@@Z 10002910 f i GorIVAlgTask.obj
 0001:00001930       ??1?$AbstractId@H@U2@@MAE@XZ 10002930 f i GorIVAlgTask.obj
 0001:00001940       ??1?$QList@V?$QSharedDataPointer@VAnnotationData@U2@@@@@@QAE@XZ 10002940 f i GorIVAlgTask.obj
 0001:00001990       ??1?$QSharedDataPointer@VAnnotationData@U2@@@@QAE@XZ 10002990 f i GorIVAlgTask.obj
 0001:000019c0       ??1?$basic_string@DU?$char_traits@D@std@@V?$allocator@D@2@@std@@QAE@XZ 100029c0 f i GorIVAlgTask.obj
 0001:000019f0       ??1AbstractInt32Id@U2@@UAE@XZ 100029f0 f i GorIVAlgTask.obj
 0001:00001a00       ??1GorIVAlgTask@U2@@UAE@XZ 10002a00 f i GorIVAlgTask.obj
 0001:00001a10       ??1ServiceType@U2@@UAE@XZ  10002a10 f i GorIVAlgTask.obj
 0001:00001a20       ??1_Generic_error_category@std@@UAE@XZ 10002a20 f i GorIVAlgTask.obj
 0001:00001a30       ??1_Iostream_error_category@std@@UAE@XZ 10002a30 f i GorIVAlgTask.obj
 0001:00001a40       ??1_System_error_category@std@@UAE@XZ 10002a40 f i GorIVAlgTask.obj
 0001:00001a50       ??1error_category@std@@UAE@XZ 10002a50 f i GorIVAlgTask.obj
 0001:00001a60       ??2@YAPAXIPAX@Z            10002a60 f i GorIVAlgTask.obj
 0001:00001a70       ??3@YAXPAX0@Z              10002a70 f i GorIVAlgTask.obj
 0001:00001a80       ??4?$QList@V?$QSharedDataPointer@VAnnotationData@U2@@@@@@QAEAAV0@$$QAV0@@Z 10002a80 f i GorIVAlgTask.obj
 0001:00001aa0       ??8error_category@std@@QBE_NABV01@@Z 10002aa0 f i GorIVAlgTask.obj
 0001:00001ab0       ??8error_condition@std@@QBE_NABV01@@Z 10002ab0 f i GorIVAlgTask.obj
 0001:00001ad0       ??_G?$AbstractId@H@U2@@MAEPAXI@Z 10002ad0 f i GorIVAlgTask.obj
 0001:00001ad0       ??_E?$AbstractId@H@U2@@MAEPAXI@Z 10002ad0 f i GorIVAlgTask.obj
 0001:00001b00       ??_G?$QSharedDataPointer@VAnnotationData@U2@@@@QAEPAXI@Z 10002b00 f i GorIVAlgTask.obj
 0001:00001b50       ??_EAbstractInt32Id@U2@@UAEPAXI@Z 10002b50 f i GorIVAlgTask.obj
 0001:00001b50       ??_GAbstractInt32Id@U2@@UAEPAXI@Z 10002b50 f i GorIVAlgTask.obj
 0001:00001b80       ??_GAnnotationData@U2@@QAEPAXI@Z 10002b80 f i GorIVAlgTask.obj
 0001:00001bb0       ??_EGorIVAlgTask@U2@@UAEPAXI@Z 10002bb0 f i GorIVAlgTask.obj
 0001:00001bb0       ??_GGorIVAlgTask@U2@@UAEPAXI@Z 10002bb0 f i GorIVAlgTask.obj
 0001:00001be0       ??_EServiceType@U2@@UAEPAXI@Z 10002be0 f i GorIVAlgTask.obj
 0001:00001be0       ??_GServiceType@U2@@UAEPAXI@Z 10002be0 f i GorIVAlgTask.obj
 0001:00001c10       ??_G_Generic_error_category@std@@UAEPAXI@Z 10002c10 f i GorIVAlgTask.obj
 0001:00001c10       ??_E_Generic_error_category@std@@UAEPAXI@Z 10002c10 f i GorIVAlgTask.obj
 0001:00001c40       ??_G_Iostream_error_category@std@@UAEPAXI@Z 10002c40 f i GorIVAlgTask.obj
 0001:00001c40       ??_E_Iostream_error_category@std@@UAEPAXI@Z 10002c40 f i GorIVAlgTask.obj
 0001:00001c70       ??_E_System_error_category@std@@UAEPAXI@Z 10002c70 f i GorIVAlgTask.obj
 0001:00001c70       ??_G_System_error_category@std@@UAEPAXI@Z 10002c70 f i GorIVAlgTask.obj
 0001:00001ca0       ??_Eerror_category@std@@UAEPAXI@Z 10002ca0 f i GorIVAlgTask.obj
 0001:00001ca0       ??_Gerror_category@std@@UAEPAXI@Z 10002ca0 f i GorIVAlgTask.obj
 0001:00001cd0       ?_Copy@?$basic_string@DU?$char_traits@D@std@@V?$allocator@D@2@@std@@QAEXII@Z 10002cd0 f i GorIVAlgTask.obj
 0001:00001e20       ?_Eos@?$basic_string@DU?$char_traits@D@std@@V?$allocator@D@2@@std@@QAEXI@Z 10002e20 f i GorIVAlgTask.obj
 0001:00001e50       ?_Getal@?$_String_alloc@$0A@U?$_String_base_types@DV?$allocator@D@std@@@std@@@std@@QBE?AU?$_Wrap_alloc@V?$allocator@D@std@@@2@XZ 10002e50 f i GorIVAlgTask.obj
 0001:00001e60       ?_Grow@?$basic_string@DU?$char_traits@D@std@@V?$allocator@D@2@@std@@QAE_NI_N@Z 10002e60 f i GorIVAlgTask.obj
 0001:00001f10       ?_Inside@?$basic_string@DU?$char_traits@D@std@@V?$allocator@D@2@@std@@QAE_NPBD@Z 10002f10 f i GorIVAlgTask.obj
 0001:00001f50       ?_Myptr@?$_String_val@U?$_Simple_types@D@std@@@std@@QAEPADXZ 10002f50 f i GorIVAlgTask.obj
 0001:00001f60       ?_Myptr@?$_String_val@U?$_Simple_types@D@std@@@std@@QBEPBDXZ 10002f60 f i GorIVAlgTask.obj
 0001:00001f70       ?_Tidy@?$basic_string@DU?$char_traits@D@std@@V?$allocator@D@2@@std@@QAEX_NI@Z 10002f70 f i GorIVAlgTask.obj
 0001:00001fc0       ?_Xlen@?$basic_string@DU?$char_traits@D@std@@V?$allocator@D@2@@std@@QBEXXZ 10002fc0 f i GorIVAlgTask.obj
 0001:00001fd0       ?_Xran@?$basic_string@DU?$char_traits@D@std@@V?$allocator@D@2@@std@@QBEXXZ 10002fd0 f i GorIVAlgTask.obj
 0001:00001fe0       ?allocate@?$_Wrap_alloc@V?$allocator@D@std@@@std@@QAEPADI@Z 10002fe0 f i GorIVAlgTask.obj
 0001:00002010       ?allocate@?$allocator@D@std@@QAEPADI@Z 10003010 f i GorIVAlgTask.obj
 0001:00002040       ?assign@?$basic_string@DU?$char_traits@D@std@@V?$allocator@D@2@@std@@QAEAAV12@ABV12@II@Z 10003040 f i GorIVAlgTask.obj
 0001:00002160       ?assign@?$basic_string@DU?$char_traits@D@std@@V?$allocator@D@2@@std@@QAEAAV12@PBD@Z 10003160 f i GorIVAlgTask.obj
 0001:000021a0       ?assign@?$basic_string@DU?$char_traits@D@std@@V?$allocator@D@2@@std@@QAEAAV12@PBDI@Z 100031a0 f i GorIVAlgTask.obj
 0001:000022a0       ?assign@?$char_traits@D@std@@SAXAADABD@Z 100032a0 f i GorIVAlgTask.obj
 0001:000022b0       ?category@error_code@std@@QBEABVerror_category@2@XZ 100032b0 f i GorIVAlgTask.obj
 0001:000022c0       ?category@error_condition@std@@QBEABVerror_category@2@XZ 100032c0 f i GorIVAlgTask.obj
 0001:000022d0       ?copy@?$char_traits@D@std@@SAPADPADPBDI@Z 100032d0 f i GorIVAlgTask.obj
 0001:000022f0       ?dealloc@?$QList@V?$QSharedDataPointer@VAnnotationData@U2@@@@@@AAEXPAUData@QListData@@@Z 100032f0 f i GorIVAlgTask.obj
 0001:00002320       ?deallocate@?$_Wrap_alloc@V?$allocator@D@std@@@std@@QAEXPADI@Z 10003320 f i GorIVAlgTask.obj
 0001:00002340       ?deallocate@?$allocator@D@std@@QAEXPADI@Z 10003340 f i GorIVAlgTask.obj
 0001:00002360       ?default_error_condition@_System_error_category@std@@UBE?AVerror_condition@2@H@Z 10003360 f i GorIVAlgTask.obj
 0001:000023a0       ?default_error_condition@error_category@std@@UBE?AVerror_condition@2@H@Z 100033a0 f i GorIVAlgTask.obj
 0001:000023c0       ?deref@?$QBasicAtomicInteger@H@@QAE_NXZ 100033c0 f i GorIVAlgTask.obj
 0001:000023d0       ?deref@RefCount@QtPrivate@@QAE_NXZ 100033d0 f i GorIVAlgTask.obj
 0001:000023f0       ?equivalent@error_category@std@@UBE_NABVerror_code@2@H@Z 100033f0 f i GorIVAlgTask.obj
 0001:00002410       ?equivalent@error_category@std@@UBE_NHABVerror_condition@2@@Z 10003410 f i GorIVAlgTask.obj
 0001:00002450       ?erase@?$basic_string@DU?$char_traits@D@std@@V?$allocator@D@2@@std@@QAEAAV12@I@Z 10003450 f i GorIVAlgTask.obj
 0001:00002490       ?erase@?$basic_string@DU?$char_traits@D@std@@V?$allocator@D@2@@std@@QAEAAV12@II@Z 10003490 f i GorIVAlgTask.obj
 0001:00002530       ?generic_category@std@@YAABVerror_category@1@XZ 10003530 f i GorIVAlgTask.obj
 0001:00002540       ?isValid@AbstractInt32Id@U2@@UBE_NXZ 10003540 f i GorIVAlgTask.obj
 0001:00002550       ?length@?$char_traits@D@std@@SAIPBD@Z 10003550 f i GorIVAlgTask.obj
 0001:00002570       ?load@?$QBasicAtomicInteger@H@@QBEHXZ 10003570 f i GorIVAlgTask.obj
 0001:00002580       ?max_size@?$_Wrap_alloc@V?$allocator@D@std@@@std@@QBEIXZ 10003580 f i GorIVAlgTask.obj
 0001:00002590       ?max_size@?$allocator@D@std@@QBEIXZ 10003590 f i GorIVAlgTask.obj
 0001:000025a0       ?max_size@?$allocator_traits@V?$allocator@D@std@@@std@@SAIABV?$allocator@D@2@@Z 100035a0 f i GorIVAlgTask.obj
 0001:000025b0       ?max_size@?$basic_string@DU?$char_traits@D@std@@V?$allocator@D@2@@std@@QBEIXZ 100035b0 f i GorIVAlgTask.obj
 0001:000025c0       ?message@_Generic_error_category@std@@UBE?AV?$basic_string@DU?$char_traits@D@std@@V?$allocator@D@2@@2@H@Z 100035c0 f i GorIVAlgTask.obj
 0001:00002640       ?message@_Iostream_error_category@std@@UBE?AV?$basic_string@DU?$char_traits@D@std@@V?$allocator@D@2@@2@H@Z 10003640 f i GorIVAlgTask.obj
 0001:00002690       ?message@_System_error_category@std@@UBE?AV?$basic_string@DU?$char_traits@D@std@@V?$allocator@D@2@@2@H@Z 10003690 f i GorIVAlgTask.obj
 0001:00002710       ?move@?$char_traits@D@std@@SAPADPADPBDI@Z 10003710 f i GorIVAlgTask.obj
 0001:00002730       ?name@_Generic_error_category@std@@UBEPBDXZ 10003730 f i GorIVAlgTask.obj
 0001:00002740       ?name@_Iostream_error_category@std@@UBEPBDXZ 10003740 f i GorIVAlgTask.obj
 0001:00002750       ?name@_System_error_category@std@@UBEPBDXZ 10003750 f i GorIVAlgTask.obj
 0001:00002760       ?node_destruct@?$QList@V?$QSharedDataPointer@VAnnotationData@U2@@@@@@AAEXPAUNode@1@0@Z 10003760 f i GorIVAlgTask.obj
 0001:000027b0       ?run@GorIVAlgTask@U2@@UAEXXZ 100037b0 f   GorIVAlgTask.obj
 0001:00002a10       ?size@?$basic_string@DU?$char_traits@D@std@@V?$allocator@D@2@@std@@QBEIXZ 10003a10 f i GorIVAlgTask.obj
 0001:00002a20       ?system_category@std@@YAABVerror_category@1@XZ 10003a20 f i GorIVAlgTask.obj
 0001:00002a30       ?value@error_code@std@@QBEHXZ 10003a30 f i GorIVAlgTask.obj
 0001:00002a40       ?value@error_condition@std@@QBEHXZ 10003a40 f i GorIVAlgTask.obj
 0001:00002a50       _hypot                     10003a50 f i GorIVAlgTask.obj
 0001:00002a80       ??0?$QList@PAVAnnotationSettings@U2@@@@QAE@XZ 10003a80 f i GorIVPlugin.obj
 0001:00002a90       ??0Factory@GorIVAlgTask@U2@@QAE@XZ 10003a90 f i GorIVPlugin.obj
 0001:00002aa0       ??0SecStructPredictPlugin@U2@@QAE@XZ 10003aa0 f   GorIVPlugin.obj
 0001:00002c70       ??1?$QList@PAVAnnotationSettings@U2@@@@QAE@XZ 10003c70 f i GorIVPlugin.obj
 0001:00002ca0       ??1Factory@GorIVAlgTask@U2@@UAE@XZ 10003ca0 f i GorIVPlugin.obj
 0001:00002cb0       ??1SecStructPredictPlugin@U2@@UAE@XZ 10003cb0 f   GorIVPlugin.obj
 0001:00002cc0       ??6?$QList@PAVAnnotationSettings@U2@@@@QAEAAV0@ABQAVAnnotationSettings@U2@@@Z 10003cc0 f i GorIVPlugin.obj
 0001:00002ce0       ??_GFactory@GorIVAlgTask@U2@@UAEPAXI@Z 10003ce0 f i GorIVPlugin.obj
 0001:00002ce0       ??_EFactory@GorIVAlgTask@U2@@UAEPAXI@Z 10003ce0 f i GorIVPlugin.obj
 0001:00002d10       ??_GQString@@QAEPAXI@Z     10003d10 f i GorIVPlugin.obj
 0001:00002d40       ??_GSecStructPredictPlugin@U2@@UAEPAXI@Z 10003d40 f i GorIVPlugin.obj
 0001:00002d40       ??_ESecStructPredictPlugin@U2@@UAEPAXI@Z 10003d40 f i GorIVPlugin.obj
 0001:00002d70       ?append@?$QList@PAVAnnotationSettings@U2@@@@QAEXABQAVAnnotationSettings@U2@@@Z 10003d70 f i GorIVPlugin.obj
 0001:00002e00       ?append@?$QList@VQString@@@@QAEXABVQString@@@Z 10003e00 f i GorIVPlugin.obj
 0001:00002ef0       ?createTaskInstance@Factory@GorIVAlgTask@U2@@UAEPAVSecStructPredictTask@3@ABVQByteArray@@@Z 10003ef0 f i GorIVPlugin.obj
 0001:00002f60       ?dealloc@?$QList@PAVAnnotationSettings@U2@@@@AAEXPAUData@QListData@@@Z 10003f60 f i GorIVPlugin.obj
 0001:00002f80       ?dealloc@?$QList@VQString@@@@AAEXPAUData@QListData@@@Z 10003f80 f i GorIVPlugin.obj
 0001:00002fc0       ?detach_helper_grow@?$QList@PAVAnnotationSettings@U2@@@@AAEPAUNode@1@HH@Z 10003fc0 f i GorIVPlugin.obj
 0001:000030d0       ?detach_helper_grow@?$QList@VQString@@@@AAEPAUNode@1@HH@Z 100040d0 f i GorIVPlugin.obj
 0001:00003250       ?isShared@RefCount@QtPrivate@@QBE_NXZ 10004250 f i GorIVPlugin.obj
 0001:00003270       ?node_construct@?$QList@PAVAnnotationSettings@U2@@@@AAEXPAUNode@1@ABQAVAnnotationSettings@U2@@@Z 10004270 f i GorIVPlugin.obj
 0001:00003290       ?node_construct@?$QList@VQString@@@@AAEXPAUNode@1@ABVQString@@@Z 10004290 f i GorIVPlugin.obj
 0001:000032e0       ?node_copy@?$QList@PAVAnnotationSettings@U2@@@@AAEXPAUNode@1@00@Z 100042e0 f i GorIVPlugin.obj
 0001:00003310       ?node_copy@?$QList@VQString@@@@AAEXPAUNode@1@00@Z 10004310 f i GorIVPlugin.obj
 0001:000033b0       ?node_destruct@?$QList@PAVAnnotationSettings@U2@@@@AAEXPAUNode@1@0@Z 100043b0 f i GorIVPlugin.obj
 0001:000033c0       ?node_destruct@?$QList@PAVAnnotationSettings@U2@@@@AAEXPAUNode@1@@Z 100043c0 f i GorIVPlugin.obj
 0001:000033d0       ?node_destruct@?$QList@VQString@@@@AAEXPAUNode@1@0@Z 100043d0 f i GorIVPlugin.obj
 0001:00003400       ?node_destruct@?$QList@VQString@@@@AAEXPAUNode@1@@Z 10004400 f i GorIVPlugin.obj
 0001:00003410       ?tr@SecStructPredictPlugin@U2@@SA?AVQString@@PBD0H@Z 10004410 f i GorIVPlugin.obj
 0001:00003440       _ugene_plugin_init         10004440 f   GorIVPlugin.obj
 0001:00003460       ??0QLatin1Char@@QAE@D@Z    10004460 f i gor.obj
 0001:00003470       ?First_Pass@@YAXHPAPAMPAD@Z 10004470 f   gor.obj
 0001:00003720       ?Indices@@YAXHPAH0AAVU2OpStatus@U2@@@Z 10004720 f   gor.obj
 0001:00003840       ?Normalize@@YAXQAMQAN@Z    10004840 f   gor.obj
 0001:000038d0       ?Parameters@@YAXHPAHPAPAD1AAVU2OpStatus@U2@@@Z 100048d0 f   gor.obj
 0001:00003f60       ?Second_Pass@@YAXHPAPAMPAD@Z 10004f60 f   gor.obj
 0001:000044e0       ?log@@YAMM@Z               100054e0 f i gor.obj
 0001:00004500       ?obs_indx@@YAHH@Z          10005500 f   gor.obj
 0001:00004570       ?predic@@YAXHPAD0PAPAM@Z   10005570 f   gor.obj
 0001:00004810       ?printout@@YAXHPAD00PAPAMPAU_iobuf@@@Z 10005810 f   gor.obj
 0001:00004ab0       ?qt_noop@@YAXXZ            10005ab0 f i gor.obj
 0001:00004ac0       ?readFile@@YAXAAVQFile@@HPAPAD1PAHAAVU2OpStatus@U2@@@Z 10005ac0 f   gor.obj
 0001:00004ea0       ?runGORIV@@YAHAAVQFile@@0PADH1AAVU2OpStatus@U2@@@Z 10005ea0 f   gor.obj
 0001:000052d0       ?seq_indx@@YAHH@Z          100062d0 f   gor.obj
 0001:00005430       ?tr@GorIVAlgTask@U2@@SA?AVQString@@PBD0H@Z 10006430 f i gor.obj
 0001:00005460       _logf                      10006460 f i gor.obj
 0001:00005480       ?INDMAXVAL@@YAHQAMHH@Z     10006480 f   nrutil.obj
 0001:00005580       ?INDMINVAL@@YAHQAMHH@Z     10006580 f   nrutil.obj
 0001:000056a0       ?check_boundaries@@YAHHHQADH@Z 100066a0 f   nrutil.obj
 0001:000056f0       ?cmatrix@@YAPAPADJJJJ@Z    100066f0 f   nrutil.obj
 0001:00005790       ?convert_matrix@@YAPAPAMPAMJJJJ@Z 10006790 f   nrutil.obj
 0001:00005810       ?cvector@@YAPADJJ@Z        10006810 f   nrutil.obj
 0001:00005840       ?dmatrix@@YAPAPANJJJJ@Z    10006840 f   nrutil.obj
 0001:000058f0       ?dvector@@YAPANJJ@Z        100068f0 f   nrutil.obj
 0001:00005930       ?f3tensor@@YAPAPAPAMJJJJJJ@Z 10006930 f   nrutil.obj
 0001:00005ad0       ?free_cmatrix@@YAXPAPADJJJJ@Z 10006ad0 f   nrutil.obj
 0001:00005b00       ?free_convert_matrix@@YAXPAPAMJJJJ@Z 10006b00 f   nrutil.obj
 0001:00005b20       ?free_cvector@@YAXPADJJ@Z  10006b20 f   nrutil.obj
 0001:00005b40       ?free_dmatrix@@YAXPAPANJJJJ@Z 10006b40 f   nrutil.obj
 0001:00005b70       ?free_dvector@@YAXPANJJ@Z  10006b70 f   nrutil.obj
 0001:00005b90       ?free_f3tensor@@YAXPAPAPAMJJJJJJ@Z 10006b90 f   nrutil.obj
 0001:00005be0       ?free_imatrix@@YAXPAPAHJJJJ@Z 10006be0 f   nrutil.obj
 0001:00005c10       ?free_ivector@@YAXPAHJJ@Z  10006c10 f   nrutil.obj
 0001:00005c30       ?free_lvector@@YAXPAJJJ@Z  10006c30 f   nrutil.obj
 0001:00005c50       ?free_matrix@@YAXPAPAMJJJJ@Z 10006c50 f   nrutil.obj
 0001:00005c80       ?free_submatrix@@YAXPAPAMJJJJ@Z 10006c80 f   nrutil.obj
 0001:00005ca0       ?free_svector@@YAXPAGJJ@Z  10006ca0 f   nrutil.obj
 0001:00005cc0       ?free_vector@@YAXPAMJJ@Z   10006cc0 f   nrutil.obj
 0001:00005ce0       ?imatrix@@YAPAPAHJJJJ@Z    10006ce0 f   nrutil.obj
 0001:00005d90       ?ivector@@YAPAHJJ@Z        10006d90 f   nrutil.obj
 0001:00005dd0       ?lvector@@YAPAJJJ@Z        10006dd0 f   nrutil.obj
 0001:00005e10       ?matrix@@YAPAPAMJJJJ@Z     10006e10 f   nrutil.obj
 0001:00005ec0       ?nerror@@YAXPBD@Z          10006ec0 f   nrutil.obj
 0001:00005f10       ?submatrix@@YAPAPAMPAPAMJJJJJJ@Z 10006f10 f   nrutil.obj
 0001:00005f90       ?svector@@YAPAGJJ@Z        10006f90 f   nrutil.obj
 0001:00005fd0       ?vector@@YAPAMJJ@Z         10006fd0 f   nrutil.obj
 0001:00006010       ??C?$QScopedPointer@VQObjectData@@U?$QScopedPointerDeleter@VQObjectData@@@@@@QBEPAVQObjectData@@XZ 10007010 f i moc_GorIVAlgTask.obj
 0001:00006020       ?metaObject@GorIVAlgTask@U2@@UBEPBUQMetaObject@@XZ 10007020 f   moc_GorIVAlgTask.obj
 0001:00006040       ?qt_metacall@GorIVAlgTask@U2@@UAEHW4Call@QMetaObject@@HPAPAX@Z 10007040 f   moc_GorIVAlgTask.obj
 0001:00006050       ?qt_metacast@GorIVAlgTask@U2@@UAEPAXPBD@Z 10007050 f   moc_GorIVAlgTask.obj
 0001:000060b0       ?qt_static_metacall@GorIVAlgTask@U2@@CAXPAVQObject@@W4Call@QMetaObject@@HPAPAX@Z 100070b0 f   moc_GorIVAlgTask.obj
 0001:000060c0       ?metaObject@SecStructPredictPlugin@U2@@UBEPBUQMetaObject@@XZ 100070c0 f   moc_GorIVPlugin.obj
 0001:000060e0       ?qt_metacall@SecStructPredictPlugin@U2@@UAEHW4Call@QMetaObject@@HPAPAX@Z 100070e0 f   moc_GorIVPlugin.obj
 0001:000060f0       ?qt_metacast@SecStructPredictPlugin@U2@@UAEPAXPBD@Z 100070f0 f   moc_GorIVPlugin.obj
 0001:00006150       ?qt_static_metacall@SecStructPredictPlugin@U2@@CAXPAVQObject@@W4Call@QMetaObject@@HPAPAX@Z 10007150 f   moc_GorIVPlugin.obj
 0001:00006160       ??0initializer@?A0xa2c253da@@QAE@XZ 10007160 f i qrc_gor4.obj
 0001:00006180       ??1initializer@?A0xa2c253da@@QAE@XZ 10007180 f i qrc_gor4.obj
 0001:000061a0       ?qCleanupResources_gor4@@YAHXZ 100071a0 f   qrc_gor4.obj
 0001:000061c0       ?qInitResources_gor4@@YAHXZ 100071c0 f   qrc_gor4.obj
 0001:000061e0       ??1GCounter@U2@@UAE@XZ     100071e0 f   U2Core:U2Core.dll
 0001:000061e6       ??0GReportableCounter@U2@@QAE@ABVQString@@0N@Z 100071e6 f   U2Core:U2Core.dll
 0001:000061ec       ??0Logger@U2@@QAE@ABVQString@@@Z 100071ec f   U2Core:U2Core.dll
 0001:000061f2       ??1Logger@U2@@UAE@XZ       100071f2 f   U2Core:U2Core.dll
 0001:000061f8       ??1AnnotationData@U2@@QAE@XZ 100071f8 f   U2Core:U2Core.dll
 0001:000061fe       ?cleanup@Task@U2@@UAEXXZ   100071fe f   U2Core:U2Core.dll
 0001:00006204       ?generateReport@Task@U2@@UBE?AVQString@@XZ 10007204 f   U2Core:U2Core.dll
 0001:0000620a       ?getNumParallelSubtasks@Task@U2@@UBEHXZ 1000720a f   U2Core:U2Core.dll
 0001:00006210       ?getParentTask@Task@U2@@UBEPAV12@XZ 10007210 f   U2Core:U2Core.dll
 0001:00006216       ?getSubtaskWithErrors@Task@U2@@UBEPAV12@XZ 10007216 f   U2Core:U2Core.dll
 0001:0000621c       ?getTaskId@Task@U2@@UBE_JXZ 1000721c f   U2Core:U2Core.dll
 0001:00006222       ?getTopLevelParentTask@Task@U2@@UAEPAV12@XZ 10007222 f   U2Core:U2Core.dll
 0001:00006228       ?getWarnings@Task@U2@@UBE?AVQStringList@@XZ 10007228 f   U2Core:U2Core.dll
 0001:0000622e       ?hasSubtasksWithErrors@Task@U2@@UBE_NXZ 1000722e f   U2Core:U2Core.dll
 0001:00006234       ?hasWarning@Task@U2@@UBE_NXZ 10007234 f   U2Core:U2Core.dll
 0001:0000623a       ?isNotificationReport@Task@U2@@UBE_NXZ 1000723a f   U2Core:U2Core.dll
 0001:00006240       ?isReportingEnabled@Task@U2@@UBE_NXZ 10007240 f   U2Core:U2Core.dll
 0001:00006246       ?isReportingSupported@Task@U2@@UBE_NXZ 10007246 f   U2Core:U2Core.dll
 0001:0000624c       ?isTopLevelTask@Task@U2@@UBE_NXZ 1000724c f   U2Core:U2Core.dll
 0001:00006252       ?onSubTaskFinished@Task@U2@@MAE?AV?$QList@PAVTask@U2@@@@PAV12@@Z 10007252 f   U2Core:U2Core.dll
 0001:00006258       ?propagateSubtaskError@Task@U2@@UAE_NXZ 10007258 f   U2Core:U2Core.dll
 0001:0000625e       ?report@Task@U2@@UAE?AW4ReportResult@12@XZ 1000725e f   U2Core:U2Core.dll
 0001:00006264       ?setCollectChildrensWarningsFlag@Task@U2@@UAEX_N@Z 10007264 f   U2Core:U2Core.dll
 0001:0000626a       ?setNoAutoDelete@Task@U2@@UAEX_N@Z 1000726a f   U2Core:U2Core.dll
 0001:00006270       ?setNotificationReport@Task@U2@@UAEX_N@Z 10007270 f   U2Core:U2Core.dll
 0001:00006276       ?setReportingEnabled@Task@U2@@UAEX_N@Z 10007276 f   U2Core:U2Core.dll
 0001:0000627c       ?setReportingSupported@Task@U2@@UAEX_N@Z 1000727c f   U2Core:U2Core.dll
 0001:00006282       ??0Plugin@U2@@QAE@ABVQString@@0_NW4PluginState@1@@Z 10007282 f   U2Core:U2Core.dll
 0001:00006288       ??1Plugin@U2@@UAE@XZ       10007288 f   U2Core:U2Core.dll
 0001:0000628e       ?getAnnotationsSettingsRegistry@AppContext@U2@@SAPAVAnnotationSettingsRegistry@2@XZ 1000728e f   U2Core:U2Core.dll
 0001:00006294       ?getSecStructPredictAlgRegistry@AppContext@U2@@SAPAVSecStructPredictAlgRegistry@2@XZ 10007294 f   U2Core:U2Core.dll
 0001:0000629a       ??0AnnotationSettings@U2@@QAE@ABVQString@@_NABVQColor@@1@Z 1000729a f   U2Core:U2Core.dll
 0001:000062a0       ?changeSettings@AnnotationSettingsRegistry@U2@@QAEXABV?$QList@PAVAnnotationSettings@U2@@@@_N@Z 100072a0 f   U2Core:U2Core.dll
 0001:000062a6       ?qt_metacast@Plugin@U2@@UAEPAXPBD@Z 100072a6 f   U2Core:U2Core.dll
 0001:000062ac       ?qt_metacall@Plugin@U2@@UAEHW4Call@QMetaObject@@HPAPAX@Z 100072ac f   U2Core:U2Core.dll
 0001:000062b2       ?tr@SecStructPredictTask@U2@@SA?AVQString@@PBD0H@Z 100072b2 f   U2Algorithm:U2Algorithm.dll
 0001:000062b8       ??0SecStructPredictTask@U2@@QAE@ABVQByteArray@@@Z 100072b8 f   U2Algorithm:U2Algorithm.dll
 0001:000062be       ??1SecStructPredictTask@U2@@UAE@XZ 100072be f   U2Algorithm:U2Algorithm.dll
 0001:000062c4       ?prepare@SecStructPredictTask@U2@@UAEXXZ 100072c4 f   U2Algorithm:U2Algorithm.dll
 0001:000062ca       ?registerAlgorithm@SecStructPredictAlgRegistry@U2@@QAE_NPAVSecStructPredictTaskFactory@2@ABVQString@@@Z 100072ca f   U2Algorithm:U2Algorithm.dll
 0001:000062d0       ?qt_metacast@SecStructPredictTask@U2@@UAEPAXPBD@Z 100072d0 f   U2Algorithm:U2Algorithm.dll
 0001:000062d6       ?qt_metacall@SecStructPredictTask@U2@@UAEHW4Call@QMetaObject@@HPAPAX@Z 100072d6 f   U2Algorithm:U2Algorithm.dll
 0001:000062dc       ?saveAlgorithmResultsAsAnnotations@SecStructPredictUtils@U2@@SA?AV?$QList@V?$QSharedDataPointer@VAnnotationData@U2@@@@@@ABVQByteArray@@ABVQString@@@Z 100072dc f   U2View:U2View.dll
 0001:000062e2       ?setRgb@QColor@@QAEXHHHH@Z 100072e2 f   Qt5Gui:Qt5Gui.dll
 0001:000062e8       ??0QMutex@@QAE@W4RecursionMode@0@@Z 100072e8 f   Qt5Core:Qt5Core.dll
 0001:000062ee       ??1QMutex@@QAE@XZ          100072ee f   Qt5Core:Qt5Core.dll
 0001:000062f4       ??0QMutexLocker@@QAE@PAVQBasicMutex@@@Z 100072f4 f   Qt5Core:Qt5Core.dll
 0001:000062fa       ??1QMutexLocker@@QAE@XZ    100072fa f   Qt5Core:Qt5Core.dll
 0001:00006300       ?unlock@QMutexLocker@@QAEXXZ 10007300 f   Qt5Core:Qt5Core.dll
 0001:00006306       ?resize@QByteArray@@QAEXH@Z 10007306 f   Qt5Core:Qt5Core.dll
 0001:0000630c       ?data@QByteArray@@QAEPADXZ 1000730c f   Qt5Core:Qt5Core.dll
 0001:00006312       ?prepend@QByteArray@@QAEAAV1@D@Z 10007312 f   Qt5Core:Qt5Core.dll
 0001:00006318       ??1QString@@QAE@XZ         10007318 f   Qt5Core:Qt5Core.dll
 0001:0000631e       ?fromAscii_helper@QString@@CAPAU?$QTypedArrayData@G@@PBDH@Z 1000731e f   Qt5Core:Qt5Core.dll
 0001:00006324       ?dispose@QListData@@SAXPAUData@1@@Z 10007324 f   Qt5Core:Qt5Core.dll
 0001:0000632a       ?tr@QObject@@SA?AVQString@@PBD0H@Z 1000732a f   Qt5Core:Qt5Core.dll
 0001:00006330       ??0QFile@@QAE@ABVQString@@@Z 10007330 f   Qt5Core:Qt5Core.dll
 0001:00006336       ??1QFile@@UAE@XZ           10007336 f   Qt5Core:Qt5Core.dll
 0001:0000633c       ?open@QFile@@UAE_NV?$QFlags@W4OpenModeFlag@QIODevice@@@@@Z 1000733c f   Qt5Core:Qt5Core.dll
 0001:00006342       ?childEvent@QObject@@MAEXPAVQChildEvent@@@Z 10007342 f   Qt5Core:Qt5Core.dll
 0001:00006348       ?connectNotify@QObject@@MAEXABVQMetaMethod@@@Z 10007348 f   Qt5Core:Qt5Core.dll
 0001:0000634e       ?customEvent@QObject@@MAEXPAVQEvent@@@Z 1000734e f   Qt5Core:Qt5Core.dll
 0001:00006354       ?disconnectNotify@QObject@@MAEXABVQMetaMethod@@@Z 10007354 f   Qt5Core:Qt5Core.dll
 0001:0000635a       ?event@QObject@@UAE_NPAVQEvent@@@Z 1000735a f   Qt5Core:Qt5Core.dll
 0001:00006360       ?eventFilter@QObject@@UAE_NPAV1@PAVQEvent@@@Z 10007360 f   Qt5Core:Qt5Core.dll
 0001:00006366       ?timerEvent@QObject@@MAEXPAVQTimerEvent@@@Z 10007366 f   Qt5Core:Qt5Core.dll
 0001:0000636c       ??0QString@@QAE@ABV0@@Z    1000736c f   Qt5Core:Qt5Core.dll
 0001:00006372       ?tr@QMetaObject@@QBE?AVQString@@PBD0H@Z 10007372 f   Qt5Core:Qt5Core.dll
 0001:00006378       ?detach_grow@QListData@@QAEPAUData@1@PAHH@Z 10007378 f   Qt5Core:Qt5Core.dll
 0001:0000637e       ?append@QListData@@QAEPAPAXXZ 1000737e f   Qt5Core:Qt5Core.dll
 0001:00006384       ??0QChar@@QAE@UQLatin1Char@@@Z 10007384 f   Qt5Core:Qt5Core.dll
 0001:0000638a       ??1QByteArray@@QAE@XZ      1000738a f   Qt5Core:Qt5Core.dll
 0001:00006390       ?constData@QByteArray@@QBEPBDXZ 10007390 f   Qt5Core:Qt5Core.dll
 0001:00006396       ??AQByteArray@@QAE?AVQByteRef@@H@Z 10007396 f   Qt5Core:Qt5Core.dll
 0001:0000639c       ?append@QByteArray@@QAEAAV1@PBD@Z 1000739c f   Qt5Core:Qt5Core.dll
 0001:000063a2       ??8QByteRef@@QBE_ND@Z      100073a2 f   Qt5Core:Qt5Core.dll
 0001:000063a8       ?arg@QString@@QBE?AV1@DHVQChar@@@Z 100073a8 f   Qt5Core:Qt5Core.dll
 0001:000063ae       ?arg@QString@@QBE?AV1@ABV1@HVQChar@@@Z 100073ae f   Qt5Core:Qt5Core.dll
 0001:000063b4       ?toLatin1@QString@@QBE?AVQByteArray@@XZ 100073b4 f   Qt5Core:Qt5Core.dll
 0001:000063ba       ?number@QString@@SA?AV1@HH@Z 100073ba f   Qt5Core:Qt5Core.dll
 0001:000063c0       ??0QTextStream@@QAE@PAVQIODevice@@@Z 100073c0 f   Qt5Core:Qt5Core.dll
 0001:000063c6       ??1QTextStream@@UAE@XZ     100073c6 f   Qt5Core:Qt5Core.dll
 0001:000063cc       ?atEnd@QTextStream@@QBE_NXZ 100073cc f   Qt5Core:Qt5Core.dll
 0001:000063d2       ?readLine@QTextStream@@QAE?AVQString@@_J@Z 100073d2 f   Qt5Core:Qt5Core.dll
 0001:000063d8       ??5QTextStream@@QAEAAV0@AAD@Z 100073d8 f   Qt5Core:Qt5Core.dll
 0001:000063de       ?dynamicMetaObject@QObjectData@@QBEPAUQMetaObject@@XZ 100073de f   Qt5Core:Qt5Core.dll
 0001:000063e4       ?qRegisterResourceData@@YA_NHPBE00@Z 100073e4 f   Qt5Core:Qt5Core.dll
 0001:000063ea       ?qUnregisterResourceData@@YA_NHPBE00@Z 100073ea f   Qt5Core:Qt5Core.dll
 0001:000063f0       ?_Xbad_alloc@std@@YAXXZ    100073f0 f   msvcprt:MSVCP120.dll
 0001:000063f6       ?_Xlength_error@std@@YAXPBD@Z 100073f6 f   msvcprt:MSVCP120.dll
 0001:000063fc       ?_Xout_of_range@std@@YAXPBD@Z 100073fc f   msvcprt:MSVCP120.dll
 0001:00006402       ?_Syserror_map@std@@YAPBDH@Z 10007402 f   msvcprt:MSVCP120.dll
 0001:00006408       ?_Winerror_map@std@@YAPBDH@Z 10007408 f   msvcprt:MSVCP120.dll
 0001:0000640e       __purecall                 1000740e f   MSVCRT:MSVCR120.dll
 0001:00006414       ??2@YAPAXI@Z               10007414 f   MSVCRT:MSVCR120.dll
 0001:0000641a       ??3@YAXPAX@Z               1000741a f   MSVCRT:MSVCR120.dll
 0001:00006420       ___atonexitinit            10007420 f   MSVCRT:atonexit.obj
 0001:0000645c       __onexit                   1000745c f   MSVCRT:atonexit.obj
 0001:00006505       _atexit                    10007505 f   MSVCRT:atonexit.obj
 0001:0000651a       _memmove                   1000751a f   MSVCRT:MSVCR120.dll
 0001:00006520       __hypot                    10007520 f   MSVCRT:MSVCR120.dll
 0001:00006526       @__security_check_cookie@4 10007526 f   MSVCRT:secchk.obj
 0001:00006536       __CxxThrowException@8      10007536 f   MSVCRT:MSVCR120.dll
 0001:0000653c       ___CxxFrameHandler3        1000753c f   MSVCRT:MSVCR120.dll
 0001:00006542       _memcpy                    10007542 f   MSVCRT:MSVCR120.dll
 0001:00006548       ??0type_info@@AAE@ABV0@@Z  10007548 f   MSVCRT:ti_inst.obj
 0001:00006553       ??4type_info@@AAEAAV0@ABV0@@Z 10007553 f   MSVCRT:ti_inst.obj
 0001:00006558       ??_Etype_info@@UAEPAXI@Z   10007558 f i MSVCRT:ti_inst.obj
 0001:000065b0       _fprintf                   100075b0 f   MSVCRT:MSVCR120.dll
 0001:000065b6       _printf                    100075b6 f   MSVCRT:MSVCR120.dll
 0001:000065bc       _strncmp                   100075bc f   MSVCRT:MSVCR120.dll
 0001:000065c2       _strncpy                   100075c2 f   MSVCRT:MSVCR120.dll
 0001:000065c8       _free                      100075c8 f   MSVCRT:MSVCR120.dll
 0001:000065ce       _malloc                    100075ce f   MSVCRT:MSVCR120.dll
 0001:000065d4       __libm_sse2_exp_precise    100075d4 f   MSVCRT:MSVCR120.dll
 0001:000065da       __libm_sse2_log_precise    100075da f   MSVCRT:MSVCR120.dll
 0001:000065e0       ___iob_func                100075e0 f   MSVCRT:MSVCR120.dll
 0001:000065e6       _exit                      100075e6 f   MSVCRT:MSVCR120.dll
 0001:00006638       _NtCurrentTeb              10007638 f i MSVCRT:crtdll.obj
 0001:0000663f       __CRT_INIT@12              1000763f f   MSVCRT:crtdll.obj
 0001:00006836       __DllMainCRTStartup@12     10007836 f   MSVCRT:crtdll.obj
 0001:0000698c       __lock                     1000798c f   MSVCRT:MSVCR120.dll
 0001:00006992       __unlock                   10007992 f   MSVCRT:MSVCR120.dll
 0001:00006998       __calloc_crt               10007998 f   MSVCRT:MSVCR120.dll
 0001:0000699e       ___dllonexit               1000799e f   MSVCRT:MSVCR120.dll
 0001:000069b0       __SEH_prolog4              100079b0 f   MSVCRT:sehprolg4.obj
 0001:000069f5       __SEH_epilog4              100079f5 f   MSVCRT:sehprolg4.obj
 0001:00006a09       __except_handler4          10007a09 f   MSVCRT:chandler4gs.obj
 0001:00006a2c       ___raise_securityfailure   10007a2c f   MSVCRT:gs_report.obj
 0001:00006a69       ___report_gsfailure        10007a69 f   MSVCRT:gs_report.obj
 0001:00006b64       ___report_rangecheckfailure 10007b64 f   MSVCRT:gs_report.obj
 0001:00006b70       ___report_securityfailure  10007b70 f   MSVCRT:gs_report.obj
 0001:00006c40       ___report_securityfailureEx 10007c40 f   MSVCRT:gs_report.obj
 0001:00006d56       ??_M@YGXPAXIHP6EX0@Z@Z     10007d56 f   MSVCRT:ehvecdtr.obj
 0001:00006dde       ?__ArrayUnwind@@YGXPAXIHP6EX0@Z@Z 10007dde f   MSVCRT:ehvecdtr.obj
 0001:00006e3c       ??1type_info@@UAE@XZ       10007e3c f   MSVCRT:MSVCR120.dll
 0001:00006e42       ___CppXcptFilter           10007e42 f   MSVCRT:MSVCR120.dll
 0001:00006e48       __amsg_exit                10007e48 f   MSVCRT:MSVCR120.dll
 0001:00006e50       __FindPESection            10007e50 f   MSVCRT:pesect.obj
 0001:00006ea0       __IsNonwritableInCurrentImage 10007ea0 f   MSVCRT:pesect.obj
 0001:00006f60       __ValidateImageBase        10007f60 f   MSVCRT:pesect.obj
 0001:00006f91       ___security_init_cookie    10007f91 f   MSVCRT:gs_support.obj
 0001:0000702d       _DllMain@12                1000802d f   MSVCRT:dllmain.obj
 0001:00007050       __malloc_crt               10008050 f   MSVCRT:MSVCR120.dll
 0001:00007056       __RTC_Initialize           10008056 f   MSVCRT:initsect.obj
 0001:00007076       __RTC_Terminate            10008076 f   MSVCRT:initsect.obj
 0001:00007096       __initterm                 10008096 f   MSVCRT:MSVCR120.dll
 0001:0000709c       __initterm_e               1000809c f   MSVCRT:MSVCR120.dll
 0001:000070a2       ___clean_type_info_names   100080a2 f   MSVCRT:tncleanup.obj
 0001:000070ae       __except_handler4_common   100080ae f   MSVCRT:MSVCR120.dll
 0001:000070b4       __crt_debugger_hook        100080b4 f   MSVCRT:MSVCR120.dll
 0001:000070ba       ___crtUnhandledException   100080ba f   MSVCRT:MSVCR120.dll
 0001:000070c0       ___crtTerminateProcess     100080c0 f   MSVCRT:MSVCR120.dll
 0001:000070c6       ?terminate@@YAXXZ          100080c6 f   MSVCRT:MSVCR120.dll
 0001:000070cc       ___clean_type_info_names_internal 100080cc f   MSVCRT:MSVCR120.dll
 0001:000070d2       _EncodePointer@4           100080d2 f   kernel32:KERNEL32.dll
 0001:000070d8       _DecodePointer@4           100080d8 f   kernel32:KERNEL32.dll
 0001:000070de       _IsDebuggerPresent@0       100080de f   kernel32:KERNEL32.dll
 0001:000070e4       _IsProcessorFeaturePresent@4 100080e4 f   kernel32:KERNEL32.dll
 0001:000070ea       _QueryPerformanceCounter@4 100080ea f   kernel32:KERNEL32.dll
 0001:000070f0       _GetCurrentProcessId@0     100080f0 f   kernel32:KERNEL32.dll
 0001:000070f6       _GetCurrentThreadId@0      100080f6 f   kernel32:KERNEL32.dll
 0001:000070fc       _GetSystemTimeAsFileTime@4 100080fc f   kernel32:KERNEL32.dll
 0001:00007102       _DisableThreadLibraryCalls@4 10008102 f   kernel32:KERNEL32.dll
 0002:00000000       __imp__DisableThreadLibraryCalls@4 1000a000     kernel32:KERNEL32.dll
 0002:00000004       __imp__GetSystemTimeAsFileTime@4 1000a004     kernel32:KERNEL32.dll
 0002:00000008       __imp__GetCurrentThreadId@0 1000a008     kernel32:KERNEL32.dll
 0002:0000000c       __imp__GetCurrentProcessId@0 1000a00c     kernel32:KERNEL32.dll
 0002:00000010       __imp__QueryPerformanceCounter@4 1000a010     kernel32:KERNEL32.dll
 0002:00000014       __imp__IsProcessorFeaturePresent@4 1000a014     kernel32:KERNEL32.dll
 0002:00000018       __imp__IsDebuggerPresent@0 1000a018     kernel32:KERNEL32.dll
 0002:0000001c       __imp__DecodePointer@4     1000a01c     kernel32:KERNEL32.dll
 0002:00000020       __imp__EncodePointer@4     1000a020     kernel32:KERNEL32.dll
 0002:00000024       \177KERNEL32_NULL_THUNK_DATA 1000a024     kernel32:KERNEL32.dll
 0002:00000028       __imp_?_Xlength_error@std@@YAXPBD@Z 1000a028     msvcprt:MSVCP120.dll
 0002:0000002c       __imp_?_Xout_of_range@std@@YAXPBD@Z 1000a02c     msvcprt:MSVCP120.dll
 0002:00000030       __imp_?_Syserror_map@std@@YAPBDH@Z 1000a030     msvcprt:MSVCP120.dll
 0002:00000034       __imp_?_Winerror_map@std@@YAPBDH@Z 1000a034     msvcprt:MSVCP120.dll
 0002:00000038       __imp_?_Xbad_alloc@std@@YAXXZ 1000a038     msvcprt:MSVCP120.dll
 0002:0000003c       \177MSVCP120_NULL_THUNK_DATA 1000a03c     msvcprt:MSVCP120.dll
 0002:00000040       __imp___initterm_e         1000a040     MSVCRT:MSVCR120.dll
 0002:00000044       __imp___initterm           1000a044     MSVCRT:MSVCR120.dll
 0002:00000048       __imp___malloc_crt         1000a048     MSVCRT:MSVCR120.dll
 0002:0000004c       __imp___amsg_exit          1000a04c     MSVCRT:MSVCR120.dll
 0002:00000050       __imp____CppXcptFilter     1000a050     MSVCRT:MSVCR120.dll
 0002:00000054       __imp_??1type_info@@UAE@XZ 1000a054     MSVCRT:MSVCR120.dll
 0002:00000058       __imp___onexit             1000a058     MSVCRT:MSVCR120.dll
 0002:0000005c       __imp____dllonexit         1000a05c     MSVCRT:MSVCR120.dll
 0002:00000060       __imp___calloc_crt         1000a060     MSVCRT:MSVCR120.dll
 0002:00000064       __imp___except_handler4_common 1000a064     MSVCRT:MSVCR120.dll
 0002:00000068       __imp___lock               1000a068     MSVCRT:MSVCR120.dll
 0002:0000006c       __imp__exit                1000a06c     MSVCRT:MSVCR120.dll
 0002:00000070       __imp____iob_func          1000a070     MSVCRT:MSVCR120.dll
 0002:00000074       __imp___libm_sse2_log_precise 1000a074     MSVCRT:MSVCR120.dll
 0002:00000078       __imp___libm_sse2_exp_precise 1000a078     MSVCRT:MSVCR120.dll
 0002:0000007c       __imp__malloc              1000a07c     MSVCRT:MSVCR120.dll
 0002:00000080       __imp__free                1000a080     MSVCRT:MSVCR120.dll
 0002:00000084       __imp__strncpy             1000a084     MSVCRT:MSVCR120.dll
 0002:00000088       __imp__strncmp             1000a088     MSVCRT:MSVCR120.dll
 0002:0000008c       __imp__printf              1000a08c     MSVCRT:MSVCR120.dll
 0002:00000090       __imp__fprintf             1000a090     MSVCRT:MSVCR120.dll
 0002:00000094       __imp__memcpy              1000a094     MSVCRT:MSVCR120.dll
 0002:00000098       __imp____CxxFrameHandler3  1000a098     MSVCRT:MSVCR120.dll
 0002:0000009c       __imp___CxxThrowException@8 1000a09c     MSVCRT:MSVCR120.dll
 0002:000000a0       __imp___hypot              1000a0a0     MSVCRT:MSVCR120.dll
 0002:000000a4       __imp__memmove             1000a0a4     MSVCRT:MSVCR120.dll
 0002:000000a8       __imp_??3@YAXPAX@Z         1000a0a8     MSVCRT:MSVCR120.dll
 0002:000000ac       __imp_??2@YAPAXI@Z         1000a0ac     MSVCRT:MSVCR120.dll
 0002:000000b0       __imp___purecall           1000a0b0     MSVCRT:MSVCR120.dll
 0002:000000b4       __imp___crt_debugger_hook  1000a0b4     MSVCRT:MSVCR120.dll
 0002:000000b8       __imp____crtUnhandledException 1000a0b8     MSVCRT:MSVCR120.dll
 0002:000000bc       __imp____crtTerminateProcess 1000a0bc     MSVCRT:MSVCR120.dll
 0002:000000c0       __imp_?terminate@@YAXXZ    1000a0c0     MSVCRT:MSVCR120.dll
 0002:000000c4       __imp____clean_type_info_names_internal 1000a0c4     MSVCRT:MSVCR120.dll
 0002:000000c8       __imp___unlock             1000a0c8     MSVCRT:MSVCR120.dll
 0002:000000cc       \177MSVCR120_NULL_THUNK_DATA 1000a0cc     MSVCRT:MSVCR120.dll
 0002:000000d0       __imp_??0QMutex@@QAE@W4RecursionMode@0@@Z 1000a0d0     Qt5Core:Qt5Core.dll
 0002:000000d4       __imp_??1QMutex@@QAE@XZ    1000a0d4     Qt5Core:Qt5Core.dll
 0002:000000d8       __imp_??0QMutexLocker@@QAE@PAVQBasicMutex@@@Z 1000a0d8     Qt5Core:Qt5Core.dll
 0002:000000dc       __imp_??1QMutexLocker@@QAE@XZ 1000a0dc     Qt5Core:Qt5Core.dll
 0002:000000e0       __imp_?unlock@QMutexLocker@@QAEXXZ 1000a0e0     Qt5Core:Qt5Core.dll
 0002:000000e4       __imp_?resize@QByteArray@@QAEXH@Z 1000a0e4     Qt5Core:Qt5Core.dll
 0002:000000e8       __imp_?data@QByteArray@@QAEPADXZ 1000a0e8     Qt5Core:Qt5Core.dll
 0002:000000ec       __imp_?prepend@QByteArray@@QAEAAV1@D@Z 1000a0ec     Qt5Core:Qt5Core.dll
 0002:000000f0       __imp_??1QString@@QAE@XZ   1000a0f0     Qt5Core:Qt5Core.dll
 0002:000000f4       __imp_?fromAscii_helper@QString@@CAPAU?$QTypedArrayData@G@@PBDH@Z 1000a0f4     Qt5Core:Qt5Core.dll
 0002:000000f8       __imp_?dispose@QListData@@SAXPAUData@1@@Z 1000a0f8     Qt5Core:Qt5Core.dll
 0002:000000fc       __imp_?tr@QObject@@SA?AVQString@@PBD0H@Z 1000a0fc     Qt5Core:Qt5Core.dll
 0002:00000100       __imp_??0QFile@@QAE@ABVQString@@@Z 1000a100     Qt5Core:Qt5Core.dll
 0002:00000104       __imp_??1QFile@@UAE@XZ     1000a104     Qt5Core:Qt5Core.dll
 0002:00000108       __imp_?open@QFile@@UAE_NV?$QFlags@W4OpenModeFlag@QIODevice@@@@@Z 1000a108     Qt5Core:Qt5Core.dll
 0002:0000010c       __imp_?childEvent@QObject@@MAEXPAVQChildEvent@@@Z 1000a10c     Qt5Core:Qt5Core.dll
 0002:00000110       __imp_?connectNotify@QObject@@MAEXABVQMetaMethod@@@Z 1000a110     Qt5Core:Qt5Core.dll
 0002:00000114       __imp_?customEvent@QObject@@MAEXPAVQEvent@@@Z 1000a114     Qt5Core:Qt5Core.dll
 0002:00000118       __imp_?disconnectNotify@QObject@@MAEXABVQMetaMethod@@@Z 1000a118     Qt5Core:Qt5Core.dll
 0002:0000011c       __imp_?event@QObject@@UAE_NPAVQEvent@@@Z 1000a11c     Qt5Core:Qt5Core.dll
 0002:00000120       __imp_?eventFilter@QObject@@UAE_NPAV1@PAVQEvent@@@Z 1000a120     Qt5Core:Qt5Core.dll
 0002:00000124       __imp_?timerEvent@QObject@@MAEXPAVQTimerEvent@@@Z 1000a124     Qt5Core:Qt5Core.dll
 0002:00000128       __imp_??0QString@@QAE@ABV0@@Z 1000a128     Qt5Core:Qt5Core.dll
 0002:0000012c       __imp_?tr@QMetaObject@@QBE?AVQString@@PBD0H@Z 1000a12c     Qt5Core:Qt5Core.dll
 0002:00000130       __imp_?detach_grow@QListData@@QAEPAUData@1@PAHH@Z 1000a130     Qt5Core:Qt5Core.dll
 0002:00000134       __imp_?append@QListData@@QAEPAPAXXZ 1000a134     Qt5Core:Qt5Core.dll
 0002:00000138       __imp_?shared_null@QListData@@2UData@1@B 1000a138     Qt5Core:Qt5Core.dll
 0002:0000013c       __imp_??0QChar@@QAE@UQLatin1Char@@@Z 1000a13c     Qt5Core:Qt5Core.dll
 0002:00000140       __imp_??1QByteArray@@QAE@XZ 1000a140     Qt5Core:Qt5Core.dll
 0002:00000144       __imp_?constData@QByteArray@@QBEPBDXZ 1000a144     Qt5Core:Qt5Core.dll
 0002:00000148       __imp_??AQByteArray@@QAE?AVQByteRef@@H@Z 1000a148     Qt5Core:Qt5Core.dll
 0002:0000014c       __imp_?append@QByteArray@@QAEAAV1@PBD@Z 1000a14c     Qt5Core:Qt5Core.dll
 0002:00000150       __imp_??8QByteRef@@QBE_ND@Z 1000a150     Qt5Core:Qt5Core.dll
 0002:00000154       __imp_?arg@QString@@QBE?AV1@DHVQChar@@@Z 1000a154     Qt5Core:Qt5Core.dll
 0002:00000158       __imp_?arg@QString@@QBE?AV1@ABV1@HVQChar@@@Z 1000a158     Qt5Core:Qt5Core.dll
 0002:0000015c       __imp_?toLatin1@QString@@QBE?AVQByteArray@@XZ 1000a15c     Qt5Core:Qt5Core.dll
 0002:00000160       __imp_?number@QString@@SA?AV1@HH@Z 1000a160     Qt5Core:Qt5Core.dll
 0002:00000164       __imp_??0QTextStream@@QAE@PAVQIODevice@@@Z 1000a164     Qt5Core:Qt5Core.dll
 0002:00000168       __imp_??1QTextStream@@UAE@XZ 1000a168     Qt5Core:Qt5Core.dll
 0002:0000016c       __imp_?atEnd@QTextStream@@QBE_NXZ 1000a16c     Qt5Core:Qt5Core.dll
 0002:00000170       __imp_?readLine@QTextStream@@QAE?AVQString@@_J@Z 1000a170     Qt5Core:Qt5Core.dll
 0002:00000174       __imp_??5QTextStream@@QAEAAV0@AAD@Z 1000a174     Qt5Core:Qt5Core.dll
 0002:00000178       __imp_?dynamicMetaObject@QObjectData@@QBEPAUQMetaObject@@XZ 1000a178     Qt5Core:Qt5Core.dll
 0002:0000017c       __imp_?qRegisterResourceData@@YA_NHPBE00@Z 1000a17c     Qt5Core:Qt5Core.dll
 0002:00000180       __imp_?qUnregisterResourceData@@YA_NHPBE00@Z 1000a180     Qt5Core:Qt5Core.dll
 0002:00000184       \177Qt5Core_NULL_THUNK_DATA 1000a184     Qt5Core:Qt5Core.dll
 0002:00000188       __imp_?setRgb@QColor@@QAEXHHHH@Z 1000a188     Qt5Gui:Qt5Gui.dll
 0002:0000018c       \177Qt5Gui_NULL_THUNK_DATA 1000a18c     Qt5Gui:Qt5Gui.dll
 0002:00000190       __imp_??0SecStructPredictTask@U2@@QAE@ABVQByteArray@@@Z 1000a190     U2Algorithm:U2Algorithm.dll
 0002:00000194       __imp_??1SecStructPredictTask@U2@@UAE@XZ 1000a194     U2Algorithm:U2Algorithm.dll
 0002:00000198       __imp_?staticMetaObject@SecStructPredictTask@U2@@2UQMetaObject@@B 1000a198     U2Algorithm:U2Algorithm.dll
 0002:0000019c       __imp_?qt_metacall@SecStructPredictTask@U2@@UAEHW4Call@QMetaObject@@HPAPAX@Z 1000a19c     U2Algorithm:U2Algorithm.dll
 0002:000001a0       __imp_?qt_metacast@SecStructPredictTask@U2@@UAEPAXPBD@Z 1000a1a0     U2Algorithm:U2Algorithm.dll
 0002:000001a4       __imp_??_7SecStructPredictTaskFactory@U2@@6B@ 1000a1a4     U2Algorithm:U2Algorithm.dll
 0002:000001a8       __imp_?registerAlgorithm@SecStructPredictAlgRegistry@U2@@QAE_NPAVSecStructPredictTaskFactory@2@ABVQString@@@Z 1000a1a8     U2Algorithm:U2Algorithm.dll
 0002:000001ac       __imp_?prepare@SecStructPredictTask@U2@@UAEXXZ 1000a1ac     U2Algorithm:U2Algorithm.dll
 0002:000001b0       __imp_?tr@SecStructPredictTask@U2@@SA?AVQString@@PBD0H@Z 1000a1b0     U2Algorithm:U2Algorithm.dll
 0002:000001b4       \177U2Algorithm_NULL_THUNK_DATA 1000a1b4     U2Algorithm:U2Algorithm.dll
 0002:000001b8       __imp_??0GReportableCounter@U2@@QAE@ABVQString@@0N@Z 1000a1b8     U2Core:U2Core.dll
 0002:000001bc       __imp_??0Logger@U2@@QAE@ABVQString@@@Z 1000a1bc     U2Core:U2Core.dll
 0002:000001c0       __imp_?staticMetaObject@Plugin@U2@@2UQMetaObject@@B 1000a1c0     U2Core:U2Core.dll
 0002:000001c4       __imp_?qt_metacall@Plugin@U2@@UAEHW4Call@QMetaObject@@HPAPAX@Z 1000a1c4     U2Core:U2Core.dll
 0002:000001c8       __imp_?qt_metacast@Plugin@U2@@UAEPAXPBD@Z 1000a1c8     U2Core:U2Core.dll
 0002:000001cc       __imp_?SecStructTypeQualifierName@BioStruct3D@U2@@2VQString@@A 1000a1cc     U2Core:U2Core.dll
 0002:000001d0       __imp_?changeSettings@AnnotationSettingsRegistry@U2@@QAEXABV?$QList@PAVAnnotationSettings@U2@@@@_N@Z 1000a1d0     U2Core:U2Core.dll
 0002:000001d4       __imp_??0AnnotationSettings@U2@@QAE@ABVQString@@_NABVQColor@@1@Z 1000a1d4     U2Core:U2Core.dll
 0002:000001d8       __imp_?getSecStructPredictAlgRegistry@AppContext@U2@@SAPAVSecStructPredictAlgRegistry@2@XZ 1000a1d8     U2Core:U2Core.dll
 0002:000001dc       __imp_?getAnnotationsSettingsRegistry@AppContext@U2@@SAPAVAnnotationSettingsRegistry@2@XZ 1000a1dc     U2Core:U2Core.dll
 0002:000001e0       __imp_??1Plugin@U2@@UAE@XZ 1000a1e0     U2Core:U2Core.dll
 0002:000001e4       __imp_??0Plugin@U2@@QAE@ABVQString@@0_NW4PluginState@1@@Z 1000a1e4     U2Core:U2Core.dll
 0002:000001e8       __imp_?setReportingSupported@Task@U2@@UAEX_N@Z 1000a1e8     U2Core:U2Core.dll
 0002:000001ec       __imp_?setReportingEnabled@Task@U2@@UAEX_N@Z 1000a1ec     U2Core:U2Core.dll
 0002:000001f0       __imp_?setNotificationReport@Task@U2@@UAEX_N@Z 1000a1f0     U2Core:U2Core.dll
 0002:000001f4       __imp_?setNoAutoDelete@Task@U2@@UAEX_N@Z 1000a1f4     U2Core:U2Core.dll
 0002:000001f8       __imp_?setCollectChildrensWarningsFlag@Task@U2@@UAEX_N@Z 1000a1f8     U2Core:U2Core.dll
 0002:000001fc       __imp_?report@Task@U2@@UAE?AW4ReportResult@12@XZ 1000a1fc     U2Core:U2Core.dll
 0002:00000200       __imp_?propagateSubtaskError@Task@U2@@UAE_NXZ 1000a200     U2Core:U2Core.dll
 0002:00000204       __imp_?onSubTaskFinished@Task@U2@@MAE?AV?$QList@PAVTask@U2@@@@PAV12@@Z 1000a204     U2Core:U2Core.dll
 0002:00000208       __imp_?isTopLevelTask@Task@U2@@UBE_NXZ 1000a208     U2Core:U2Core.dll
 0002:0000020c       __imp_?isReportingSupported@Task@U2@@UBE_NXZ 1000a20c     U2Core:U2Core.dll
 0002:00000210       __imp_?isReportingEnabled@Task@U2@@UBE_NXZ 1000a210     U2Core:U2Core.dll
 0002:00000214       __imp_?isNotificationReport@Task@U2@@UBE_NXZ 1000a214     U2Core:U2Core.dll
 0002:00000218       __imp_?hasWarning@Task@U2@@UBE_NXZ 1000a218     U2Core:U2Core.dll
 0002:0000021c       __imp_?hasSubtasksWithErrors@Task@U2@@UBE_NXZ 1000a21c     U2Core:U2Core.dll
 0002:00000220       __imp_?getWarnings@Task@U2@@UBE?AVQStringList@@XZ 1000a220     U2Core:U2Core.dll
 0002:00000224       __imp_?getTopLevelParentTask@Task@U2@@UAEPAV12@XZ 1000a224     U2Core:U2Core.dll
 0002:00000228       __imp_?getTaskId@Task@U2@@UBE_JXZ 1000a228     U2Core:U2Core.dll
 0002:0000022c       __imp_?getSubtaskWithErrors@Task@U2@@UBEPAV12@XZ 1000a22c     U2Core:U2Core.dll
 0002:00000230       __imp_?getParentTask@Task@U2@@UBEPAV12@XZ 1000a230     U2Core:U2Core.dll
 0002:00000234       __imp_?getNumParallelSubtasks@Task@U2@@UBEHXZ 1000a234     U2Core:U2Core.dll
 0002:00000238       __imp_?generateReport@Task@U2@@UBE?AVQString@@XZ 1000a238     U2Core:U2Core.dll
 0002:0000023c       __imp_?cleanup@Task@U2@@UAEXXZ 1000a23c     U2Core:U2Core.dll
 0002:00000240       __imp_??1AnnotationData@U2@@QAE@XZ 1000a240     U2Core:U2Core.dll
 0002:00000244       __imp_??1Logger@U2@@UAE@XZ 1000a244     U2Core:U2Core.dll
 0002:00000248       __imp_??1GCounter@U2@@UAE@XZ 1000a248     U2Core:U2Core.dll
 0002:0000024c       \177U2Core_NULL_THUNK_DATA 1000a24c     U2Core:U2Core.dll
 0002:00000250       __imp_?saveAlgorithmResultsAsAnnotations@SecStructPredictUtils@U2@@SA?AV?$QList@V?$QSharedDataPointer@VAnnotationData@U2@@@@@@ABVQByteArray@@ABVQString@@@Z 1000a250     U2View:U2View.dll
 0002:00000254       \177U2View_NULL_THUNK_DATA 1000a254     U2View:U2View.dll
 0002:00000258       ___xc_a                    1000a258     MSVCRT:cinitexe.obj
 0002:00000374       ___xc_z                    1000a374     MSVCRT:cinitexe.obj
 0002:00000378       ___xi_a                    1000a378     MSVCRT:cinitexe.obj
 0002:00000384       ___xi_z                    1000a384     MSVCRT:cinitexe.obj
 0002:000003c8       ??_C@_00CNPNBAHC@?$AA@     1000a3c8     GorIVAlgTask.obj
 0002:000003d0       ??_7error_category@std@@6B@ 1000a3d0     GorIVAlgTask.obj
 0002:000003ec       ??_7_Generic_error_category@std@@6B@ 1000a3ec     GorIVAlgTask.obj
 0002:00000404       ??_C@_07DCLBNMLN@generic?$AA@ 1000a404     GorIVAlgTask.obj
 0002:0000040c       ??_C@_0O@BFJCFAAK@unknown?5error?$AA@ 1000a40c     GorIVAlgTask.obj
 0002:00000420       ??_7_Iostream_error_category@std@@6B@ 1000a420     GorIVAlgTask.obj
 0002:00000438       ??_C@_08LLGCOLLL@iostream?$AA@ 1000a438     GorIVAlgTask.obj
 0002:00000444       ??_C@_0BG@PADBLCHM@iostream?5stream?5error?$AA@ 1000a444     GorIVAlgTask.obj
 0002:00000460       ??_7_System_error_category@std@@6B@ 1000a460     GorIVAlgTask.obj
 0002:00000478       ??_C@_06FHFOAHML@system?$AA@ 1000a478     GorIVAlgTask.obj
 0002:00000484       ??_7?$AbstractId@H@U2@@6B@ 1000a484     GorIVAlgTask.obj
 0002:00000490       ??_7AbstractInt32Id@U2@@6B@ 1000a490     GorIVAlgTask.obj
 0002:0000049c       ??_7ServiceType@U2@@6B@    1000a49c     GorIVAlgTask.obj
 0002:000004a4       ??_C@_0L@JLHNEGIN@Algorithms?$AA@ 1000a4a4     GorIVAlgTask.obj
 0002:000004b0       ??_C@_07PGLPGHFC@Console?$AA@ 1000a4b0     GorIVAlgTask.obj
 0002:000004b8       ??_C@_0O@BOFHOPCF@Core?5Services?$AA@ 1000a4b8     GorIVAlgTask.obj
 0002:000004c8       ??_C@_0N@PPADAKBM@Input?1Output?$AA@ 1000a4c8     GorIVAlgTask.obj
 0002:000004d8       ??_C@_0M@KPPBKPKK@Performance?$AA@ 1000a4d8     GorIVAlgTask.obj
 0002:000004e4       ??_C@_07BFDHHBBI@Scripts?$AA@ 1000a4e4     GorIVAlgTask.obj
 0002:000004ec       ??_C@_05EEGKELMG@Tasks?$AA@ 1000a4ec     GorIVAlgTask.obj
 0002:000004f4       ??_C@_0P@NIIOBHGA@User?5Interface?$AA@ 1000a4f4     GorIVAlgTask.obj
 0002:00000504       ??_C@_0N@JINCGGMN@User?5Actions?$AA@ 1000a504     GorIVAlgTask.obj
 0002:00000518       ??_7GorIVAlgTask@U2@@6B@   1000a518     GorIVAlgTask.obj
 0002:000005a4       ??_C@_05HEGNCAKE@GORIV?$AA@ 1000a5a4     GorIVAlgTask.obj
 0002:000005ac       ??_C@_0N@INHNGEFL@GorIVAlgTask?$AA@ 1000a5ac     GorIVAlgTask.obj
 0002:000005bc       ??_C@_0CB@FOIDGALD@?3gor4?1?1datafiles?1?1New_KS?4267?4seq@ 1000a5bc     GorIVAlgTask.obj
 0002:000005e0       ??_C@_0BH@OICAFECH@seq?5database?5not?5found?$AA@ 1000a5e0     GorIVAlgTask.obj
 0002:000005f8       ??_C@_0CB@HDDFPMJD@?3gor4?1?1datafiles?1?1New_KS?4267?4obs@ 1000a5f8     GorIVAlgTask.obj
 0002:0000061c       ??_C@_0CH@NENJAIAD@observed?5structures?5database?5not@ 1000a61c     GorIVAlgTask.obj
 0002:00000644       ??_C@_0CM@HJGLFIHP@sequence?5is?5too?5long?0?5max?5seq?5si@ 1000a644     GorIVAlgTask.obj
 0002:00000670       ??_C@_0O@DPCHKLGO@gorIV_results?$AA@ 1000a670     GorIVAlgTask.obj
 0002:00000680       ??_C@_0BA@JFNIOLAK@string?5too?5long?$AA@ 1000a680     GorIVAlgTask.obj
 0002:00000690       ??_C@_0BI@CFPLBAOH@invalid?5string?5position?$AA@ 1000a690     GorIVAlgTask.obj
 0002:000006a8       __real@3ff0000000000000    1000a6a8     GorIVAlgTask.obj
 0002:000006b4       ??_7SecStructPredictPlugin@U2@@6B@ 1000a6b4     GorIVPlugin.obj
 0002:000006e4       ??_7Factory@GorIVAlgTask@U2@@6B@ 1000a6e4     GorIVPlugin.obj
 0002:000006ec       ??_C@_0CN@IMOFAHKL@GORIV?5protein?5secondary?5structur@ 1000a6ec     GorIVPlugin.obj
 0002:00000728       ??_C@_0DC@KOPACOIN@There?5are?5?$CFd?5proteins?5in?5Kabsch?9@ 1000a728     gor.obj
 0002:0000075c       ??_C@_0CA@LLBIFPIG@?$CFdth?5protein?5temp?$DN?5?$CFd?5nres?$DN?5?$CFd?6?$AA@ 1000a75c     gor.obj
 0002:0000077c       ??_C@_07NAIDGHCO@?$CFs?6?$CFs?6?6?$AA@ 1000a77c     gor.obj
 0002:00000784       ??_C@_0CD@DIIHDKNC@?6?$CFdth?5data?5base?5protein?6?5?$CFs?5?6?5?$CFs@ 1000a784     gor.obj
 0002:000007a8       ??_C@_0L@OKFEDODA@?$CFd?5errors?6?$AA@ 1000a7a8     gor.obj
 0002:000007b4       ??_C@_09FJGJOEKD@?$CF1?5errors?$AA@ 1000a7b4     gor.obj
 0002:000007c0       ??_C@_01EEMJAFIK@?6?$AA@   1000a7c0     gor.obj
 0002:000007c4       ??_C@_0CM@EMDMGJK@The?5value?5of?5MAXRES?5should?5be?5in@ 1000a7c4     gor.obj
 0002:000007f0       ??_C@_0CM@MDAPGPIL@The?5value?5of?5MAXRES?5should?5be?5in@ 1000a7f0     gor.obj
 0002:0000081c       ??_C@_0BJ@EGDBLLLG@protein?3?5?$CFd?5residue?3?5?$CFd?6?$AA@ 1000a81c     gor.obj
 0002:00000838       ??_C@_0EA@LKOCLJGE@Invalid?5amino?5acid?5type?5or?5secon@ 1000a838     gor.obj
 0002:00000878       ??_C@_0FI@EOKCPGMP@protein?3?5?$CF1?5residue?3?5?$CF2?6Invalid?5@ 1000a878     gor.obj
 0002:000008d0       ??_C@_0BP@PONIEGCC@Error?5invalid?5value?5of?5np?$DN?5?$CFd?6?$AA@ 1000a8d0     gor.obj
 0002:000008f0       ??_C@_0BO@CLEEBEJH@Error?5invalid?5value?5of?5np?$DN?5?$CF1?$AA@ 1000a8f0     gor.obj
 0002:00000910       ??_C@_06ECNNDLMB@?6?6?$DO?$CFs?6?$AA@ 1000a910     gor.obj
 0002:00000918       ??_C@_02HAOIJKIC@?$CFc?$AA@ 1000a918     gor.obj
 0002:0000091c       ??_C@_08DOCONEG@Sequence?$AA@ 1000a91c     gor.obj
 0002:00000928       ??_C@_07FBMPDAOB@?5?5?5?5?$CFs?6?$AA@ 1000a928     gor.obj
 0002:00000930       ??_C@_0BH@PBKKCCJH@Predicted?5Sec?4?5Struct?4?$AA@ 1000a930     gor.obj
 0002:00000948       ??_C@_02PHMGELLB@?6?6?$AA@ 1000a948     gor.obj
 0002:0000094c       ??_C@_08GFEGNIII@?6?6?$CFs?6?$CFd?6?$AA@ 1000a94c     gor.obj
 0002:00000958       ??_C@_0BJ@JPDJLPHI@SEQ?5PRD?5?5?5H?5?5?5?5?5E?5?5?5?5?5C?6?$AA@ 1000a958     gor.obj
 0002:00000974       ??_C@_0BN@MFMGHJNK@?5?$CFc?5?5?5?$CFc?5?5?$CF5?43f?5?$CF5?43f?5?$CF5?43f?6?$AA@ 1000a974     gor.obj
 0002:00000998       __real@3eb0c6f7a0b5ed8d    1000a998     gor.obj
 0002:000009a0       __real@3f400000            1000a9a0     gor.obj
 0002:000009a4       __real@3f800000            1000a9a4     gor.obj
 0002:000009a8       __real@3fbe1e1e20000000    1000a9a8     gor.obj
 0002:000009b0       __real@3fec3c3c3c000000    1000a9b0     gor.obj
 0002:000009b8       __real@41200000            1000a9b8     gor.obj
 0002:000009c0       __xmm@00000000000000020000000400000000 1000a9c0     gor.obj
 0002:000009d0       ??_C@_0BD@DDGIPLEJ@run?9time?5error?4?4?4?6?$AA@ 1000a9d0     nrutil.obj
 0002:000009e4       ??_C@_03OFAPEBGM@?$CFs?6?$AA@ 1000a9e4     nrutil.obj
 0002:000009e8       ??_C@_0BN@ELEEGBCK@?4?4?4now?5exiting?5to?5system?4?4?4?6?$AA@ 1000a9e8     nrutil.obj
 0002:00000a08       ??_C@_0DP@MCADMMKA@Warning?3?5the?5upper?5boundary?5has?5@ 1000aa08     nrutil.obj
 0002:00000a48       ??_C@_0DP@EJPCMDCB@Warning?3?5the?5lower?5boundary?5has?5@ 1000aa48     nrutil.obj
 0002:00000a88       ??_C@_0BP@NJKBEJKL@allocation?5failure?5in?5vector?$CI?$CJ?$AA@ 1000aa88     nrutil.obj
 0002:00000aa8       ??_C@_0CA@HGHGGPEO@allocation?5failure?5in?5ivector?$CI?$CJ?$AA@ 1000aaa8     nrutil.obj
 0002:00000ac8       ??_C@_0CA@GBFEPPIH@allocation?5failure?5in?5cvector?$CI?$CJ?$AA@ 1000aac8     nrutil.obj
 0002:00000ae8       ??_C@_0CA@JAFPKEAK@allocation?5failure?5in?5lvector?$CI?$CJ?$AA@ 1000aae8     nrutil.obj
 0002:00000b08       ??_C@_0CA@EGPKHOGP@allocation?5failure?5in?5svector?$CI?$CJ?$AA@ 1000ab08     nrutil.obj
 0002:00000b28       ??_C@_0CA@IDIIOEPO@allocation?5failure?5in?5dvector?$CI?$CJ?$AA@ 1000ab28     nrutil.obj
 0002:00000b48       ??_C@_0CB@CNNMNEGI@allocation?5failure?51?5in?5matrix?$CI?$CJ@ 1000ab48     nrutil.obj
 0002:00000b6c       ??_C@_0CB@FBLNPBLD@allocation?5failure?52?5in?5matrix?$CI?$CJ@ 1000ab6c     nrutil.obj
 0002:00000b90       ??_C@_0CC@LEPGFBAB@allocation?5failure?51?5in?5dmatrix?$CI@ 1000ab90     nrutil.obj
 0002:00000bb4       ??_C@_0CC@KFILDLHI@allocation?5failure?52?5in?5dmatrix?$CI@ 1000abb4     nrutil.obj
 0002:00000bd8       ??_C@_0CC@EBAINKLB@allocation?5failure?51?5in?5imatrix?$CI@ 1000abd8     nrutil.obj
 0002:00000bfc       ??_C@_0CC@FAHFLAMI@allocation?5failure?52?5in?5imatrix?$CI@ 1000abfc     nrutil.obj
 0002:00000c20       ??_C@_0CC@FGCKEKHI@allocation?5failure?51?5in?5cmatrix?$CI@ 1000ac20     nrutil.obj
 0002:00000c44       ??_C@_0CC@EHFHCAAB@allocation?5failure?52?5in?5cmatrix?$CI@ 1000ac44     nrutil.obj
 0002:00000c68       ??_C@_0CC@NDJMKNLF@allocation?5failure?5in?5submatrix?$CI@ 1000ac68     nrutil.obj
 0002:00000c8c       ??_C@_0CH@GOIADKKN@allocation?5failure?5in?5convert_ma@ 1000ac8c     nrutil.obj
 0002:00000cb4       ??_C@_0CD@OPIDHJLJ@allocation?5failure?51?5in?5f3tensor@ 1000acb4     nrutil.obj
 0002:00000cd8       ??_C@_0CD@MGELMNEL@allocation?5failure?52?5in?5f3tensor@ 1000acd8     nrutil.obj
 0002:00000cfc       ??_C@_0CD@GICDFMNK@allocation?5failure?53?5in?5f3tensor@ 1000acfc     nrutil.obj
 0002:00000d20       ??_C@_0M@HKGIIPEA@val?$FL0?$FN?$DN?5?$CFf?6?$AA@ 1000ad20     nrutil.obj
 0002:0001ab6e       ?value@?$integral_constant@_N$0A@@std@@2_NB 10024b6e     MSVCRT:ti_inst.obj
 0002:0001ab6f       ?value@?$integral_constant@_N$00@std@@2_NB 10024b6f     MSVCRT:ti_inst.obj
 0002:0001ab74       ??_7type_info@@6B@         10024b74     MSVCRT:ti_inst.obj
 0002:0001ab78       __pRawDllMain              10024b78     MSVCRT:crtdll.obj
 0002:0001ab78       __pDefaultRawDllMain       10024b78     MSVCRT:crtdll.obj
 0002:0001ab84       ?ProcessDetach@NativeDll@<CrtImplementationDetails>@@0IB 10024b84     MSVCRT:initsect.obj
 0002:0001ab88       ?ProcessAttach@NativeDll@<CrtImplementationDetails>@@0IB 10024b88     MSVCRT:initsect.obj
 0002:0001ab8c       ?ThreadAttach@NativeDll@<CrtImplementationDetails>@@0IB 10024b8c     MSVCRT:initsect.obj
 0002:0001ab90       ?ThreadDetach@NativeDll@<CrtImplementationDetails>@@0IB 10024b90     MSVCRT:initsect.obj
 0002:0001ab94       ?ProcessVerifier@NativeDll@<CrtImplementationDetails>@@0IB 10024b94     MSVCRT:initsect.obj
 0002:0001ab98       __load_config_used         10024b98     MSVCRT:loadcfg.obj
 0002:0001ac4c       ??_R4error_category@std@@6B@ 10024c4c     GorIVAlgTask.obj
 0002:0001ac60       ??_R3error_category@std@@8 10024c60     GorIVAlgTask.obj
 0002:0001ac70       ??_R2error_category@std@@8 10024c70     GorIVAlgTask.obj
 0002:0001ac78       ??_R1A@?0A@EA@error_category@std@@8 10024c78     GorIVAlgTask.obj
 0002:0001ac94       ??_R4_Generic_error_category@std@@6B@ 10024c94     GorIVAlgTask.obj
 0002:0001aca8       ??_R3_Generic_error_category@std@@8 10024ca8     GorIVAlgTask.obj
 0002:0001acb8       ??_R2_Generic_error_category@std@@8 10024cb8     GorIVAlgTask.obj
 0002:0001acc4       ??_R1A@?0A@EA@_Generic_error_category@std@@8 10024cc4     GorIVAlgTask.obj
 0002:0001ace0       ??_R4_Iostream_error_category@std@@6B@ 10024ce0     GorIVAlgTask.obj
 0002:0001acf4       ??_R3_Iostream_error_category@std@@8 10024cf4     GorIVAlgTask.obj
 0002:0001ad04       ??_R2_Iostream_error_category@std@@8 10024d04     GorIVAlgTask.obj
 0002:0001ad14       ??_R1A@?0A@EA@_Iostream_error_category@std@@8 10024d14     GorIVAlgTask.obj
 0002:0001ad30       ??_R4_System_error_category@std@@6B@ 10024d30     GorIVAlgTask.obj
 0002:0001ad44       ??_R3_System_error_category@std@@8 10024d44     GorIVAlgTask.obj
 0002:0001ad54       ??_R2_System_error_category@std@@8 10024d54     GorIVAlgTask.obj
 0002:0001ad64       ??_R1A@?0A@EA@_System_error_category@std@@8 10024d64     GorIVAlgTask.obj
 0002:0001ad80       ??_R4AbstractInt32Id@U2@@6B@ 10024d80     GorIVAlgTask.obj
 0002:0001ad94       ??_R3AbstractInt32Id@U2@@8 10024d94     GorIVAlgTask.obj
 0002:0001ada4       ??_R2AbstractInt32Id@U2@@8 10024da4     GorIVAlgTask.obj
 0002:0001adb0       ??_R1A@?0A@EA@AbstractInt32Id@U2@@8 10024db0     GorIVAlgTask.obj
 0002:0001adcc       ??_R1A@?0A@EA@?$AbstractId@H@U2@@8 10024dcc     GorIVAlgTask.obj
 0002:0001ade8       ??_R3?$AbstractId@H@U2@@8  10024de8     GorIVAlgTask.obj
 0002:0001adf8       ??_R2?$AbstractId@H@U2@@8  10024df8     GorIVAlgTask.obj
 0002:0001ae00       ??_R4?$AbstractId@H@U2@@6B@ 10024e00     GorIVAlgTask.obj
 0002:0001ae14       ??_R4ServiceType@U2@@6B@   10024e14     GorIVAlgTask.obj
 0002:0001ae28       ??_R3ServiceType@U2@@8     10024e28     GorIVAlgTask.obj
 0002:0001ae38       ??_R2ServiceType@U2@@8     10024e38     GorIVAlgTask.obj
 0002:0001ae48       ??_R1A@?0A@EA@ServiceType@U2@@8 10024e48     GorIVAlgTask.obj
 0002:0001ae64       ??_R4GorIVAlgTask@U2@@6B@  10024e64     GorIVAlgTask.obj
 0002:0001ae78       ??_R3GorIVAlgTask@U2@@8    10024e78     GorIVAlgTask.obj
 0002:0001ae88       ??_R2GorIVAlgTask@U2@@8    10024e88     GorIVAlgTask.obj
 0002:0001ae9c       ??_R1A@?0A@EA@GorIVAlgTask@U2@@8 10024e9c     GorIVAlgTask.obj
 0002:0001aeb8       ??_R1A@?0A@EA@SecStructPredictTask@U2@@8 10024eb8     GorIVAlgTask.obj
 0002:0001aed4       ??_R3SecStructPredictTask@U2@@8 10024ed4     GorIVAlgTask.obj
 0002:0001aee4       ??_R2SecStructPredictTask@U2@@8 10024ee4     GorIVAlgTask.obj
 0002:0001aef4       ??_R1A@?0A@EA@Task@U2@@8   10024ef4     GorIVAlgTask.obj
 0002:0001af10       ??_R3Task@U2@@8            10024f10     GorIVAlgTask.obj
 0002:0001af20       ??_R2Task@U2@@8            10024f20     GorIVAlgTask.obj
 0002:0001af2c       ??_R1A@?0A@EA@QObject@@8   10024f2c     GorIVAlgTask.obj
 0002:0001af48       ??_R3QObject@@8            10024f48     GorIVAlgTask.obj
 0002:0001af58       ??_R2QObject@@8            10024f58     GorIVAlgTask.obj
 0002:0001af60       ??_R4SecStructPredictPlugin@U2@@6B@ 10024f60     GorIVPlugin.obj
 0002:0001af74       ??_R3SecStructPredictPlugin@U2@@8 10024f74     GorIVPlugin.obj
 0002:0001af84       ??_R2SecStructPredictPlugin@U2@@8 10024f84     GorIVPlugin.obj
 0002:0001af94       ??_R1A@?0A@EA@SecStructPredictPlugin@U2@@8 10024f94     GorIVPlugin.obj
 0002:0001afb0       ??_R1A@?0A@EA@Plugin@U2@@8 10024fb0     GorIVPlugin.obj
 0002:0001afcc       ??_R3Plugin@U2@@8          10024fcc     GorIVPlugin.obj
 0002:0001afdc       ??_R2Plugin@U2@@8          10024fdc     GorIVPlugin.obj
 0002:0001afe8       ??_R4Factory@GorIVAlgTask@U2@@6B@ 10024fe8     GorIVPlugin.obj
 0002:0001affc       ??_R3Factory@GorIVAlgTask@U2@@8 10024ffc     GorIVPlugin.obj
 0002:0001b00c       ??_R2Factory@GorIVAlgTask@U2@@8 1002500c     GorIVPlugin.obj
 0002:0001b018       ??_R1A@?0A@EA@Factory@GorIVAlgTask@U2@@8 10025018     GorIVPlugin.obj
 0002:0001b034       ??_R1A@?0A@EA@SecStructPredictTaskFactory@U2@@8 10025034     GorIVPlugin.obj
 0002:0001b050       ??_R3SecStructPredictTaskFactory@U2@@8 10025050     GorIVPlugin.obj
 0002:0001b060       ??_R2SecStructPredictTaskFactory@U2@@8 10025060     GorIVPlugin.obj
 0002:0001b068       ??_R4type_info@@6B@        10025068     MSVCRT:ti_inst.obj
 0002:0001b07c       ??_R3type_info@@8          1002507c     MSVCRT:ti_inst.obj
 0002:0001b08c       ??_R2type_info@@8          1002508c     MSVCRT:ti_inst.obj
 0002:0001b094       ??_R1A@?0A@EA@type_info@@8 10025094     MSVCRT:ti_inst.obj
 0002:0001b0b0       ___safe_se_handler_table   100250b0     <linker-defined>
 0002:0001b17c       ___rtc_iaa                 1002517c     MSVCRT:initsect.obj
 0002:0001b180       ___rtc_izz                 10025180     MSVCRT:initsect.obj
 0002:0001b184       ___rtc_taa                 10025184     MSVCRT:initsect.obj
 0002:0001b188       ___rtc_tzz                 10025188     MSVCRT:initsect.obj
 0002:0001bed0       __IMPORT_DESCRIPTOR_U2Core 10025ed0     U2Core:U2Core.dll
 0002:0001bee4       __IMPORT_DESCRIPTOR_U2Algorithm 10025ee4     U2Algorithm:U2Algorithm.dll
 0002:0001bef8       __IMPORT_DESCRIPTOR_U2View 10025ef8     U2View:U2View.dll
 0002:0001bf0c       __IMPORT_DESCRIPTOR_Qt5Gui 10025f0c     Qt5Gui:Qt5Gui.dll
 0002:0001bf20       __IMPORT_DESCRIPTOR_Qt5Core 10025f20     Qt5Core:Qt5Core.dll
 0002:0001bf34       __IMPORT_DESCRIPTOR_MSVCP120 10025f34     msvcprt:MSVCP120.dll
 0002:0001bf48       __IMPORT_DESCRIPTOR_MSVCR120 10025f48     MSVCRT:MSVCR120.dll
 0002:0001bf5c       __IMPORT_DESCRIPTOR_KERNEL32 10025f5c     kernel32:KERNEL32.dll
 0002:0001bf70       __NULL_IMPORT_DESCRIPTOR   10025f70     U2Core:U2Core.dll
 0003:00000000       ?_Generic_object@?$_Error_objects@H@std@@2V_Generic_error_category@2@A 10028000     GorIVAlgTask.obj
 0003:00000004       ?_Iostream_object@?$_Error_objects@H@std@@2V_Iostream_error_category@2@A 10028004     GorIVAlgTask.obj
 0003:00000008       ?_System_object@?$_Error_objects@H@std@@2V_System_error_category@2@A 10028008     GorIVAlgTask.obj
 0003:000000dc       ?staticMetaObject@GorIVAlgTask@U2@@2UQMetaObject@@B 100280dc     moc_GorIVAlgTask.obj
 0003:000000f4       ?staticMetaObject@SecStructPredictPlugin@U2@@2UQMetaObject@@B 100280f4     moc_GorIVPlugin.obj
 0003:0000010c       ___security_cookie         1002810c     MSVCRT:gs_cookie.obj
 0003:00000110       ___security_cookie_complement 10028110     MSVCRT:gs_cookie.obj
 0003:00000120       ___native_dllmain_reason   10028120     MSVCRT:natstart.obj
 0003:00000124       ??_R0?AVerror_category@std@@@8 10028124     GorIVAlgTask.obj
 0003:00000148       ??_R0?AV_Generic_error_category@std@@@8 10028148     GorIVAlgTask.obj
 0003:00000174       ??_R0?AV_Iostream_error_category@std@@@8 10028174     GorIVAlgTask.obj
 0003:000001a0       ??_R0?AV_System_error_category@std@@@8 100281a0     GorIVAlgTask.obj
 0003:000001cc       ??_R0?AVAbstractInt32Id@U2@@@8 100281cc     GorIVAlgTask.obj
 0003:000001f0       ??_R0?AV?$AbstractId@H@U2@@@8 100281f0     GorIVAlgTask.obj
 0003:00000210       ??_R0?AVServiceType@U2@@@8 10028210     GorIVAlgTask.obj
 0003:00000230       ??_R0?AVGorIVAlgTask@U2@@@8 10028230     GorIVAlgTask.obj
 0003:00000250       ??_R0?AVSecStructPredictTask@U2@@@8 10028250     GorIVAlgTask.obj
 0003:00000278       ??_R0?AVTask@U2@@@8        10028278     GorIVAlgTask.obj
 0003:00000290       ??_R0?AVQObject@@@8        10028290     GorIVAlgTask.obj
 0003:000002a8       ??_R0?AVSecStructPredictPlugin@U2@@@8 100282a8     GorIVPlugin.obj
 0003:000002d0       ??_R0?AVPlugin@U2@@@8      100282d0     GorIVPlugin.obj
 0003:000002e8       ??_R0?AVFactory@GorIVAlgTask@U2@@@8 100282e8     GorIVPlugin.obj
 0003:00000310       ??_R0?AVSecStructPredictTaskFactory@U2@@@8 10028310     GorIVPlugin.obj
 0003:00000340       ??_R0?AVtype_info@@@8      10028340     MSVCRT:ti_inst.obj
 0003:0000037c       ?taskName@GorIVAlgTask@U2@@2VQString@@B 1002837c     GorIVAlgTask.obj
 0003:00000388       ?runLock@GorIVAlgTask@U2@@0VQMutex@@A 10028388     GorIVAlgTask.obj
 0003:000003ac       ?id@?$num_put@DV?$back_insert_iterator@V?$basic_string@DU?$char_traits@D@std@@V?$allocator@D@2@@std@@@std@@@std@@2V0locale@2@A 100283ac     GorIVAlgTask.obj
 0003:000003b0       ?id@?$num_put@_WV?$back_insert_iterator@V?$basic_string@_WU?$char_traits@_W@std@@V?$allocator@_W@2@@std@@@std@@@std@@2V0locale@2@A 100283b0     GorIVAlgTask.obj
 0003:00000430       ?infopair@@3PAY2IJ@BH@BH@NA 10028430     gor.obj
 0003:001a8e88       ?infodir@@3PAY1BC@BH@NA    101d0e88     gor.obj
 0003:001ab558       ?nS@@3PAMA                 101d3558     gor.obj
 0003:001ab568       ?pS@@3PAMA                 101d3568     gor.obj
 0003:002c818c       ?dummy@?A0xa2c253da@@3Uinitializer@1@A 102f018c     qrc_gor4.obj
 0003:002c84b8       ?__type_info_root_node@@3U__type_info_node@@A 102f04b8     MSVCRT:tncleanup.obj
 0003:002c84c0       ___native_startup_lock     102f04c0     <common>
 0003:002c84c4       ___native_startup_state    102f04c4     <common>
 0003:002c84c8       ___dyn_tls_init_callback   102f04c8     <common>
 0003:002c84cc       ___onexitend               102f04cc     <common>
 0003:002c84d0       ___onexitbegin             102f04d0     <common>

 entry point at        0001:00006836

 Static symbols

 0000:ffd0b000       .debug$S                   10000000     MSVCRT:MSVCR120.dll
 0000:ffd0b000       .debug$S                   10000000     MSVCRT:MSVCR120.dll
 0000:ffd0b000       .debug$S                   10000000     MSVCRT:MSVCR120.dll
 0000:ffd0b000       .debug$S                   10000000     MSVCRT:MSVCR120.dll
 0000:ffd0b000       .debug$S                   10000000     MSVCRT:MSVCR120.dll
 0000:ffd0b000       .debug$S                   10000000     MSVCRT:MSVCR120.dll
 0000:ffd0b000       .debug$S                   10000000     MSVCRT:MSVCR120.dll
 0000:ffd0b000       .debug$S                   10000000     U2Core:U2Core.dll
 0000:ffd0b000       .debug$S                   10000000     U2Core:U2Core.dll
 0000:ffd0b000       .debug$S                   10000000     U2Core:U2Core.dll
 0000:ffd0b000       .debug$S                   10000000     U2Core:U2Core.dll
 0000:ffd0b000       .debug$S                   10000000     U2Core:U2Core.dll
 0000:ffd0b000       .debug$S                   10000000     U2Core:U2Core.dll
 0000:ffd0b000       .debug$S                   10000000     U2Core:U2Core.dll
 0000:ffd0b000       .debug$S                   10000000     U2Core:U2Core.dll
 0000:ffd0b000       .debug$S                   10000000     U2Core:U2Core.dll
 0000:ffd0b000       .debug$S                   10000000     U2Core:U2Core.dll
 0000:ffd0b000       .debug$S                   10000000     U2Core:U2Core.dll
 0000:ffd0b000       .debug$S                   10000000     U2Core:U2Core.dll
 0000:ffd0b000       .debug$S                   10000000     U2Core:U2Core.dll
 0000:ffd0b000       .debug$S                   10000000     U2Core:U2Core.dll
 0000:ffd0b000       .debug$S                   10000000     U2Core:U2Core.dll
 0001:fffff000       __ehhandler$?_Copy@?$basic_string@DU?$char_traits@D@std@@V?$allocator@D@2@@std@@QAEXII@Z 10000000 f   moc_GorIVPlugin.obj
 0002:ffff6000       __catchsym$?_Copy@?$basic_string@DU?$char_traits@D@std@@V?$allocator@D@2@@std@@QAEXII@Z$5 10000000     gor.obj
 0000:ffd0b000       .debug$S                   10000000     msvcprt:MSVCP120.dll
 0000:ffd0b000       .debug$S                   10000000     msvcprt:MSVCP120.dll
 0000:ffd0b000       .debug$S                   10000000     msvcprt:MSVCP120.dll
 0000:ffd0b000       .debug$S                   10000000     kernel32:KERNEL32.dll
 0000:ffd0b000       .debug$S                   10000000     kernel32:KERNEL32.dll
 0002:ffff6000       __catchsym$?_Copy@?$basic_string@DU?$char_traits@D@std@@V?$allocator@D@2@@std@@QAEXII@Z$5 10000000     moc_GorIVPlugin.obj
 0000:ffd0b000       .debug$S                   10000000     MSVCRT:MSVCR120.dll
 0000:ffd0b000       .debug$S                   10000000     MSVCRT:MSVCR120.dll
 0000:ffd0b000       .debug$S                   10000000     MSVCRT:MSVCR120.dll
 0000:ffd0b000       .debug$S                   10000000     MSVCRT:MSVCR120.dll
 0000:ffd0b000       .debug$S                   10000000     U2Core:U2Core.dll
 0002:ffff6000       ?_Generic_object$initializer$@?$_Error_objects@H@std@@2P6AXXZA 10000000     moc_GorIVPlugin.obj
 0002:ffff6000       ?_Iostream_object$initializer$@?$_Error_objects@H@std@@2P6AXXZA 10000000     moc_GorIVPlugin.obj
 0002:ffff6000       ?_System_object$initializer$@?$_Error_objects@H@std@@2P6AXXZA 10000000     moc_GorIVPlugin.obj
 0000:ffd0b000       .debug$S                   10000000     U2Core:U2Core.dll
 0000:ffd0b000       .debug$S                   10000000     U2Core:U2Core.dll
 0000:ffd0b000       .debug$S                   10000000     kernel32:KERNEL32.dll
 0000:ffd0b000       .debug$S                   10000000     kernel32:KERNEL32.dll
 0000:ffd0b000       .debug$S                   10000000     kernel32:KERNEL32.dll
 0000:ffd0b000       .debug$S                   10000000     kernel32:KERNEL32.dll
 0000:ffd0b000       .debug$S                   10000000     kernel32:KERNEL32.dll
 0000:ffd0b000       .debug$S                   10000000     kernel32:KERNEL32.dll
 0000:ffd0b000       .debug$S                   10000000     kernel32:KERNEL32.dll
 0000:ffd0b000       .debug$S                   10000000     Qt5Core:Qt5Core.dll
 0000:ffd0b000       .debug$S                   10000000     Qt5Core:Qt5Core.dll
 0000:ffd0b000       .debug$S                   10000000     Qt5Core:Qt5Core.dll
 0000:ffd0b000       .debug$S                   10000000     Qt5Core:Qt5Core.dll
 0000:ffd0b000       .debug$S                   10000000     Qt5Core:Qt5Core.dll
 0000:ffd0b000       .debug$S                   10000000     Qt5Core:Qt5Core.dll
 0000:ffd0b000       .debug$S                   10000000     Qt5Core:Qt5Core.dll
 0000:ffd0b000       .debug$S                   10000000     Qt5Core:Qt5Core.dll
 0000:ffd0b000       .debug$S                   10000000     Qt5Core:Qt5Core.dll
 0000:ffd0b000       .debug$S                   10000000     Qt5Core:Qt5Core.dll
 0000:ffd0b000       .debug$S                   10000000     Qt5Core:Qt5Core.dll
 0000:ffd0b000       .debug$S                   10000000     Qt5Core:Qt5Core.dll
 0000:ffd0b000       .debug$S                   10000000     Qt5Core:Qt5Core.dll
 0000:ffd0b000       .debug$S                   10000000     Qt5Core:Qt5Core.dll
 0000:ffd0b000       .debug$S                   10000000     Qt5Core:Qt5Core.dll
 0000:ffd0b000       .debug$S                   10000000     Qt5Core:Qt5Core.dll
 0000:ffd0b000       .debug$S                   10000000     Qt5Core:Qt5Core.dll
 0000:ffd0b000       .debug$S                   10000000     Qt5Core:Qt5Core.dll
 0001:fffff000       __ehhandler$?_Copy@?$basic_string@DU?$char_traits@D@std@@V?$allocator@D@2@@std@@QAEXII@Z 10000000 f   moc_GorIVAlgTask.obj
 0000:ffd0b000       .debug$S                   10000000     Qt5Core:Qt5Core.dll
 0000:ffd0b000       .debug$S                   10000000     Qt5Core:Qt5Core.dll
 0000:ffd0b000       .debug$S                   10000000     Qt5Core:Qt5Core.dll
 0000:ffd0b000       .debug$S                   10000000     Qt5Core:Qt5Core.dll
 0002:ffff6000       ?_System_object$initializer$@?$_Error_objects@H@std@@2P6AXXZA 10000000     GorIVPlugin.obj
 0002:ffff6000       ?_Iostream_object$initializer$@?$_Error_objects@H@std@@2P6AXXZA 10000000     GorIVPlugin.obj
 0002:ffff6000       ?_Generic_object$initializer$@?$_Error_objects@H@std@@2P6AXXZA 10000000     GorIVPlugin.obj
 0000:ffd0b000       .debug$S                   10000000     U2Core:U2Core.dll
 0000:ffd0b000       .debug$S                   10000000     U2Core:U2Core.dll
 0000:ffd0b000       .debug$S                   10000000     U2Core:U2Core.dll
 0000:ffd0b000       .debug$S                   10000000     U2Core:U2Core.dll
 0000:ffd0b000       .debug$S                   10000000     U2Core:U2Core.dll
 0000:ffd0b000       .debug$S                   10000000     U2Core:U2Core.dll
 0000:ffd0b000       .debug$S                   10000000     U2Core:U2Core.dll
 0000:ffd0b000       .debug$S                   10000000     U2Core:U2Core.dll
 0000:ffd0b000       .debug$S                   10000000     U2Core:U2Core.dll
 0000:ffd0b000       .debug$S                   10000000     U2Core:U2Core.dll
 0000:ffd0b000       .debug$S                   10000000     U2Core:U2Core.dll
 0000:ffd0b000       .debug$S                   10000000     U2Core:U2Core.dll
 0000:ffd0b000       .debug$S                   10000000     U2Core:U2Core.dll
 0000:ffd0b000       .debug$S                   10000000     Qt5Core:Qt5Core.dll
 0000:ffd0b000       .debug$S                   10000000     Qt5Core:Qt5Core.dll
 0000:ffd0b000       .debug$S                   10000000     Qt5Core:Qt5Core.dll
 0000:ffd0b000       .debug$S                   10000000     Qt5Core:Qt5Core.dll
 0002:ffff6000       __catchsym$?_Copy@?$basic_string@DU?$char_traits@D@std@@V?$allocator@D@2@@std@@QAEXII@Z$5 10000000     moc_GorIVAlgTask.obj
 0000:ffd0b000       .debug$S                   10000000     MSVCRT:MSVCR120.dll
 0000:ffd0b000       .debug$S                   10000000     MSVCRT:MSVCR120.dll
 0000:ffd0b000       .debug$S                   10000000     MSVCRT:MSVCR120.dll
 0000:ffd0b000       .debug$S                   10000000     MSVCRT:MSVCR120.dll
 0000:ffd0b000       .debug$S                   10000000     MSVCRT:MSVCR120.dll
 0000:ffd0b000       .debug$S                   10000000     MSVCRT:MSVCR120.dll
 0000:ffd0b000       .debug$S                   10000000     MSVCRT:MSVCR120.dll
 0000:ffd0b000       .debug$S                   10000000     MSVCRT:MSVCR120.dll
 0000:ffd0b000       .debug$S                   10000000     MSVCRT:MSVCR120.dll
 0000:ffd0b000       .debug$S                   10000000     MSVCRT:MSVCR120.dll
 0000:ffd0b000       .debug$S                   10000000     MSVCRT:MSVCR120.dll
 0000:ffd0b000       .debug$S                   10000000     MSVCRT:MSVCR120.dll
 0000:ffd0b000       .debug$S                   10000000     MSVCRT:MSVCR120.dll
 0000:ffd0b000       .debug$S                   10000000     MSVCRT:MSVCR120.dll
 0000:ffd0b000       .debug$S                   10000000     MSVCRT:MSVCR120.dll
 0000:ffd0b000       .debug$S                   10000000     MSVCRT:MSVCR120.dll
 0000:ffd0b000       .debug$S                   10000000     MSVCRT:MSVCR120.dll
 0000:ffd0b000       .debug$S                   10000000     MSVCRT:MSVCR120.dll
 0000:ffd0b000       .debug$S                   10000000     MSVCRT:MSVCR120.dll
 0000:ffd0b000       .debug$S                   10000000     MSVCRT:MSVCR120.dll
 0000:ffd0b000       .debug$S                   10000000     MSVCRT:MSVCR120.dll
 0000:ffd0b000       .debug$S                   10000000     MSVCRT:MSVCR120.dll
 0000:ffd0b000       .debug$S                   10000000     MSVCRT:MSVCR120.dll
 0000:ffd0b000       .debug$S                   10000000     MSVCRT:MSVCR120.dll
 0000:ffd0b000       .debug$S                   10000000     U2Core:U2Core.dll
 0000:ffd0b000       .debug$S                   10000000     U2Core:U2Core.dll
 0000:ffd0b000       .debug$S                   10000000     U2Core:U2Core.dll
 0000:ffd0b000       .debug$S                   10000000     U2Core:U2Core.dll
 0000:ffd0b000       .debug$S                   10000000     U2Core:U2Core.dll
 0000:ffd0b000       .debug$S                   10000000     U2Core:U2Core.dll
 0000:ffd0b000       .debug$S                   10000000     U2Algorithm:U2Algorithm.dll
 0000:ffd0b000       .debug$S                   10000000     U2Algorithm:U2Algorithm.dll
 0000:ffd0b000       .debug$S                   10000000     U2Algorithm:U2Algorithm.dll
 0000:ffd0b000       .debug$S                   10000000     U2Algorithm:U2Algorithm.dll
 0000:ffd0b000       .debug$S                   10000000     U2Algorithm:U2Algorithm.dll
 0000:ffd0b000       .debug$S                   10000000     U2Algorithm:U2Algorithm.dll
 0000:ffd0b000       .debug$S                   10000000     U2Algorithm:U2Algorithm.dll
 0000:ffd0b000       .debug$S                   10000000     U2Algorithm:U2Algorithm.dll
 0000:ffd0b000       .debug$S                   10000000     U2Algorithm:U2Algorithm.dll
 0000:ffd0b000       .debug$S                   10000000     U2View:U2View.dll
 0000:ffd0b000       .debug$S                   10000000     Qt5Gui:Qt5Gui.dll
 0002:ffff6000       ?_Generic_object$initializer$@?$_Error_objects@H@std@@2P6AXXZA 10000000     moc_GorIVAlgTask.obj
 0002:ffff6000       ?_Iostream_object$initializer$@?$_Error_objects@H@std@@2P6AXXZA 10000000     moc_GorIVAlgTask.obj
 0002:ffff6000       ?_System_object$initializer$@?$_Error_objects@H@std@@2P6AXXZA 10000000     moc_GorIVAlgTask.obj
 0000:ffd0b000       .debug$S                   10000000     msvcprt:MSVCP120.dll
 0000:ffd0b000       .debug$S                   10000000     msvcprt:MSVCP120.dll
 0000:ffd0b000       .debug$S                   10000000     Qt5Core:Qt5Core.dll
 0000:ffd0b000       .debug$S                   10000000     Qt5Core:Qt5Core.dll
 0000:ffd0b000       .debug$S                   10000000     Qt5Core:Qt5Core.dll
 0000:ffd0b000       .debug$S                   10000000     Qt5Core:Qt5Core.dll
 0000:ffd0b000       .debug$S                   10000000     Qt5Core:Qt5Core.dll
 0000:ffd0b000       .debug$S                   10000000     Qt5Core:Qt5Core.dll
 0000:ffd0b000       .debug$S                   10000000     Qt5Core:Qt5Core.dll
 0000:ffd0b000       .debug$S                   10000000     Qt5Core:Qt5Core.dll
 0000:ffd0b000       .debug$S                   10000000     Qt5Core:Qt5Core.dll
 0000:ffd0b000       .debug$S                   10000000     Qt5Core:Qt5Core.dll
 0000:ffd0b000       .debug$S                   10000000     Qt5Core:Qt5Core.dll
 0000:ffd0b000       .debug$S                   10000000     Qt5Core:Qt5Core.dll
 0000:ffd0b000       .debug$S                   10000000     Qt5Core:Qt5Core.dll
 0000:ffd0b000       .debug$S                   10000000     Qt5Core:Qt5Core.dll
 0000:ffd0b000       .debug$S                   10000000     Qt5Core:Qt5Core.dll
 0000:ffd0b000       .debug$S                   10000000     Qt5Core:Qt5Core.dll
 0000:ffd0b000       .debug$S                   10000000     Qt5Core:Qt5Core.dll
 0000:ffd0b000       .debug$S                   10000000     Qt5Core:Qt5Core.dll
 0002:ffff6000       __catchsym$?_Copy@?$basic_string@DU?$char_traits@D@std@@V?$allocator@D@2@@std@@QAEXII@Z$5 10000000     GorIVPlugin.obj
 0000:ffd0b000       .debug$S                   10000000     Qt5Core:Qt5Core.dll
 0002:ffff6000       ?_Generic_object$initializer$@?$_Error_objects@H@std@@2P6AXXZA 10000000     gor.obj
 0002:ffff6000       ?_Iostream_object$initializer$@?$_Error_objects@H@std@@2P6AXXZA 10000000     gor.obj
 0002:ffff6000       ?_System_object$initializer$@?$_Error_objects@H@std@@2P6AXXZA 10000000     gor.obj
 0001:fffff000       __ehhandler$?_Copy@?$basic_string@DU?$char_traits@D@std@@V?$allocator@D@2@@std@@QAEXII@Z 10000000 f   gor.obj
 0001:fffff000       __ehhandler$?_Copy@?$basic_string@DU?$char_traits@D@std@@V?$allocator@D@2@@std@@QAEXII@Z 10000000 f   GorIVPlugin.obj
 0002:ffff6010       __catchsym$?_Copy@?$basic_string@DU?$char_traits@D@std@@V?$allocator@D@2@@std@@QAEXII@Z$4 10000010     gor.obj
 0002:ffff6010       __catchsym$?_Copy@?$basic_string@DU?$char_traits@D@std@@V?$allocator@D@2@@std@@QAEXII@Z$4 10000010     moc_GorIVAlgTask.obj
 0002:ffff6010       __catchsym$?_Copy@?$basic_string@DU?$char_traits@D@std@@V?$allocator@D@2@@std@@QAEXII@Z$4 10000010     GorIVPlugin.obj
 0002:ffff6010       __catchsym$?_Copy@?$basic_string@DU?$char_traits@D@std@@V?$allocator@D@2@@std@@QAEXII@Z$4 10000010     moc_GorIVPlugin.obj
 0002:ffff6020       __unwindtable$?_Copy@?$basic_string@DU?$char_traits@D@std@@V?$allocator@D@2@@std@@QAEXII@Z 10000020     gor.obj
 0002:ffff6020       __unwindtable$?_Copy@?$basic_string@DU?$char_traits@D@std@@V?$allocator@D@2@@std@@QAEXII@Z 10000020     GorIVPlugin.obj
 0002:ffff6020       __unwindtable$?_Copy@?$basic_string@DU?$char_traits@D@std@@V?$allocator@D@2@@std@@QAEXII@Z 10000020     moc_GorIVPlugin.obj
 0002:ffff6020       __unwindtable$?_Copy@?$basic_string@DU?$char_traits@D@std@@V?$allocator@D@2@@std@@QAEXII@Z 10000020     moc_GorIVAlgTask.obj
 0002:ffff6040       __ehfuncinfo$?_Copy@?$basic_string@DU?$char_traits@D@std@@V?$allocator@D@2@@std@@QAEXII@Z 10000040     GorIVPlugin.obj
 0002:ffff6040       __ehfuncinfo$?_Copy@?$basic_string@DU?$char_traits@D@std@@V?$allocator@D@2@@std@@QAEXII@Z 10000040     moc_GorIVPlugin.obj
 0002:ffff6040       __ehfuncinfo$?_Copy@?$basic_string@DU?$char_traits@D@std@@V?$allocator@D@2@@std@@QAEXII@Z 10000040     gor.obj
 0002:ffff6040       __ehfuncinfo$?_Copy@?$basic_string@DU?$char_traits@D@std@@V?$allocator@D@2@@std@@QAEXII@Z 10000040     moc_GorIVAlgTask.obj
 0002:ffff6064       __tryblocktable$?_Copy@?$basic_string@DU?$char_traits@D@std@@V?$allocator@D@2@@std@@QAEXII@Z 10000064     moc_GorIVPlugin.obj
 0002:ffff6064       __tryblocktable$?_Copy@?$basic_string@DU?$char_traits@D@std@@V?$allocator@D@2@@std@@QAEXII@Z 10000064     gor.obj
 0002:ffff6064       __tryblocktable$?_Copy@?$basic_string@DU?$char_traits@D@std@@V?$allocator@D@2@@std@@QAEXII@Z 10000064     GorIVPlugin.obj
 0002:ffff6064       __tryblocktable$?_Copy@?$basic_string@DU?$char_traits@D@std@@V?$allocator@D@2@@std@@QAEXII@Z 10000064     moc_GorIVAlgTask.obj
 0001:fffff096       __catch$?_Copy@?$basic_string@DU?$char_traits@D@std@@V?$allocator@D@2@@std@@QAEXII@Z$0 10000096 f   gor.obj
 0001:fffff096       __catch$?_Copy@?$basic_string@DU?$char_traits@D@std@@V?$allocator@D@2@@std@@QAEXII@Z$0 10000096 f   moc_GorIVPlugin.obj
 0001:fffff096       __catch$?_Copy@?$basic_string@DU?$char_traits@D@std@@V?$allocator@D@2@@std@@QAEXII@Z$0 10000096 f   GorIVPlugin.obj
 0001:fffff096       __catch$?_Copy@?$basic_string@DU?$char_traits@D@std@@V?$allocator@D@2@@std@@QAEXII@Z$0 10000096 f   moc_GorIVAlgTask.obj
 0001:fffff0d3       __catch$?_Copy@?$basic_string@DU?$char_traits@D@std@@V?$allocator@D@2@@std@@QAEXII@Z$1 100000d3 f   moc_GorIVPlugin.obj
 0001:fffff0d3       __catch$?_Copy@?$basic_string@DU?$char_traits@D@std@@V?$allocator@D@2@@std@@QAEXII@Z$1 100000d3 f   GorIVPlugin.obj
 0001:fffff0d3       __catch$?_Copy@?$basic_string@DU?$char_traits@D@std@@V?$allocator@D@2@@std@@QAEXII@Z$1 100000d3 f   moc_GorIVAlgTask.obj
 0001:fffff0d3       __catch$?_Copy@?$basic_string@DU?$char_traits@D@std@@V?$allocator@D@2@@std@@QAEXII@Z$1 100000d3 f   gor.obj
 0001:00000000       ??__E?_Generic_object@?$_Error_objects@H@std@@2V_Generic_error_category@2@A@@YAXXZ 10001000 f   GorIVAlgTask.obj
 0001:00000010       ??__E?_Iostream_object@?$_Error_objects@H@std@@2V_Iostream_error_category@2@A@@YAXXZ 10001010 f   GorIVAlgTask.obj
 0001:00000020       ??__E?_System_object@?$_Error_objects@H@std@@2V_System_error_category@2@A@@YAXXZ 10001020 f   GorIVAlgTask.obj
 0001:00000030       ??__E?runLock@GorIVAlgTask@U2@@0VQMutex@@A@@YAXXZ 10001030 f   GorIVAlgTask.obj
 0001:00000050       ??__E?taskName@GorIVAlgTask@U2@@2VQString@@B@@YAXXZ 10001050 f   GorIVAlgTask.obj
 0001:00000080       ??__EService_DNAExport@U2@@YAXXZ 10001080 f   GorIVAlgTask.obj
 0001:00000090       ??__EService_DNAGraphPack@U2@@YAXXZ 10001090 f   GorIVAlgTask.obj
 0001:000000a0       ??__EService_ExternalToolSupport@U2@@YAXXZ 100010a0 f   GorIVAlgTask.obj
 0001:000000b0       ??__EService_GUITesting@U2@@YAXXZ 100010b0 f   GorIVAlgTask.obj
 0001:000000c0       ??__EService_MaxCoreServiceId@U2@@YAXXZ 100010c0 f   GorIVAlgTask.obj
 0001:000000d0       ??__EService_MinCoreServiceId@U2@@YAXXZ 100010d0 f   GorIVAlgTask.obj
 0001:000000e0       ??__EService_PluginViewer@U2@@YAXXZ 100010e0 f   GorIVAlgTask.obj
 0001:000000f0       ??__EService_Project@U2@@YAXXZ 100010f0 f   GorIVAlgTask.obj
 0001:00000100       ??__EService_ProjectView@U2@@YAXXZ 10001100 f   GorIVAlgTask.obj
 0001:00000110       ??__EService_QueryDesigner@U2@@YAXXZ 10001110 f   GorIVAlgTask.obj
 0001:00000120       ??__EService_ScriptRegistry@U2@@YAXXZ 10001120 f   GorIVAlgTask.obj
 0001:00000130       ??__EService_TestRunner@U2@@YAXXZ 10001130 f   GorIVAlgTask.obj
 0001:00000140       ??__EService_WorkflowDesigner@U2@@YAXXZ 10001140 f   GorIVAlgTask.obj
 0001:00000150       ??__EalgoLog@U2@@YAXXZ     10001150 f   GorIVAlgTask.obj
 0001:000001d0       ??__EcmdLog@U2@@YAXXZ      100011d0 f   GorIVAlgTask.obj
 0001:00000250       ??__EcoreLog@U2@@YAXXZ     10001250 f   GorIVAlgTask.obj
 0001:000002d0       ??__EioLog@U2@@YAXXZ       100012d0 f   GorIVAlgTask.obj
 0001:00000350       ??__EperfLog@U2@@YAXXZ     10001350 f   GorIVAlgTask.obj
 0001:000003d0       ??__EscriptLog@U2@@YAXXZ   100013d0 f   GorIVAlgTask.obj
 0001:00000450       ??__EtaskLog@U2@@YAXXZ     10001450 f   GorIVAlgTask.obj
 0001:000004d0       ??__EuiLog@U2@@YAXXZ       100014d0 f   GorIVAlgTask.obj
 0001:00000550       ??__EuserActLog@U2@@YAXXZ  10001550 f   GorIVAlgTask.obj
 0001:000005d0       ??__E?_Generic_object@?$_Error_objects@H@std@@2V_Generic_error_category@2@A@@YAXXZ 100015d0 f   GorIVPlugin.obj
 0001:000005e0       ??__E?_Iostream_object@?$_Error_objects@H@std@@2V_Iostream_error_category@2@A@@YAXXZ 100015e0 f   GorIVPlugin.obj
 0001:000005f0       ??__E?_System_object@?$_Error_objects@H@std@@2V_System_error_category@2@A@@YAXXZ 100015f0 f   GorIVPlugin.obj
 0001:00000600       ??__EService_DNAExport@U2@@YAXXZ 10001600 f   GorIVPlugin.obj
 0001:00000610       ??__EService_DNAGraphPack@U2@@YAXXZ 10001610 f   GorIVPlugin.obj
 0001:00000620       ??__EService_ExternalToolSupport@U2@@YAXXZ 10001620 f   GorIVPlugin.obj
 0001:00000630       ??__EService_GUITesting@U2@@YAXXZ 10001630 f   GorIVPlugin.obj
 0001:00000640       ??__EService_MaxCoreServiceId@U2@@YAXXZ 10001640 f   GorIVPlugin.obj
 0001:00000650       ??__EService_MinCoreServiceId@U2@@YAXXZ 10001650 f   GorIVPlugin.obj
 0001:00000660       ??__EService_PluginViewer@U2@@YAXXZ 10001660 f   GorIVPlugin.obj
 0001:00000670       ??__EService_Project@U2@@YAXXZ 10001670 f   GorIVPlugin.obj
 0001:00000680       ??__EService_ProjectView@U2@@YAXXZ 10001680 f   GorIVPlugin.obj
 0001:00000690       ??__EService_QueryDesigner@U2@@YAXXZ 10001690 f   GorIVPlugin.obj
 0001:000006a0       ??__EService_ScriptRegistry@U2@@YAXXZ 100016a0 f   GorIVPlugin.obj
 0001:000006b0       ??__EService_TestRunner@U2@@YAXXZ 100016b0 f   GorIVPlugin.obj
 0001:000006c0       ??__EService_WorkflowDesigner@U2@@YAXXZ 100016c0 f   GorIVPlugin.obj
 0001:000006d0       ??__EalgoLog@U2@@YAXXZ     100016d0 f   GorIVPlugin.obj
 0001:00000750       ??__EcmdLog@U2@@YAXXZ      10001750 f   GorIVPlugin.obj
 0001:000007d0       ??__EcoreLog@U2@@YAXXZ     100017d0 f   GorIVPlugin.obj
 0001:00000850       ??__EioLog@U2@@YAXXZ       10001850 f   GorIVPlugin.obj
 0001:000008d0       ??__EperfLog@U2@@YAXXZ     100018d0 f   GorIVPlugin.obj
 0001:00000950       ??__EscriptLog@U2@@YAXXZ   10001950 f   GorIVPlugin.obj
 0001:000009d0       ??__EtaskLog@U2@@YAXXZ     100019d0 f   GorIVPlugin.obj
 0001:00000a50       ??__EuiLog@U2@@YAXXZ       10001a50 f   GorIVPlugin.obj
 0001:00000ad0       ??__EuserActLog@U2@@YAXXZ  10001ad0 f   GorIVPlugin.obj
 0001:00000b50       ??__E?_Generic_object@?$_Error_objects@H@std@@2V_Generic_error_category@2@A@@YAXXZ 10001b50 f   gor.obj
 0001:00000b60       ??__E?_Iostream_object@?$_Error_objects@H@std@@2V_Iostream_error_category@2@A@@YAXXZ 10001b60 f   gor.obj
 0001:00000b70       ??__E?_System_object@?$_Error_objects@H@std@@2V_System_error_category@2@A@@YAXXZ 10001b70 f   gor.obj
 0001:00000b80       ??__EalgoLog@U2@@YAXXZ     10001b80 f   gor.obj
 0001:00000c00       ??__EcmdLog@U2@@YAXXZ      10001c00 f   gor.obj
 0001:00000c80       ??__EcoreLog@U2@@YAXXZ     10001c80 f   gor.obj
 0001:00000d00       ??__EioLog@U2@@YAXXZ       10001d00 f   gor.obj
 0001:00000d80       ??__EperfLog@U2@@YAXXZ     10001d80 f   gor.obj
 0001:00000e00       ??__EscriptLog@U2@@YAXXZ   10001e00 f   gor.obj
 0001:00000e80       ??__EtaskLog@U2@@YAXXZ     10001e80 f   gor.obj
 0001:00000f00       ??__EuiLog@U2@@YAXXZ       10001f00 f   gor.obj
 0001:00000f80       ??__EuserActLog@U2@@YAXXZ  10001f80 f   gor.obj
 0001:00001000       ??__E?_Generic_object@?$_Error_objects@H@std@@2V_Generic_error_category@2@A@@YAXXZ 10002000 f   moc_GorIVAlgTask.obj
 0001:00001010       ??__E?_Iostream_object@?$_Error_objects@H@std@@2V_Iostream_error_category@2@A@@YAXXZ 10002010 f   moc_GorIVAlgTask.obj
 0001:00001020       ??__E?_System_object@?$_Error_objects@H@std@@2V_System_error_category@2@A@@YAXXZ 10002020 f   moc_GorIVAlgTask.obj
 0001:00001030       ??__E?staticMetaObject@GorIVAlgTask@U2@@2UQMetaObject@@B@@YAXXZ 10002030 f   moc_GorIVAlgTask.obj
 0001:00001040       ??__EalgoLog@U2@@YAXXZ     10002040 f   moc_GorIVAlgTask.obj
 0001:000010c0       ??__EcmdLog@U2@@YAXXZ      100020c0 f   moc_GorIVAlgTask.obj
 0001:00001140       ??__EcoreLog@U2@@YAXXZ     10002140 f   moc_GorIVAlgTask.obj
 0001:000011c0       ??__EioLog@U2@@YAXXZ       100021c0 f   moc_GorIVAlgTask.obj
 0001:00001240       ??__EperfLog@U2@@YAXXZ     10002240 f   moc_GorIVAlgTask.obj
 0001:000012c0       ??__EscriptLog@U2@@YAXXZ   100022c0 f   moc_GorIVAlgTask.obj
 0001:00001340       ??__EtaskLog@U2@@YAXXZ     10002340 f   moc_GorIVAlgTask.obj
 0001:000013c0       ??__EuiLog@U2@@YAXXZ       100023c0 f   moc_GorIVAlgTask.obj
 0001:00001440       ??__EuserActLog@U2@@YAXXZ  10002440 f   moc_GorIVAlgTask.obj
 0001:000014c0       ??__E?_Generic_object@?$_Error_objects@H@std@@2V_Generic_error_category@2@A@@YAXXZ 100024c0 f   moc_GorIVPlugin.obj
 0001:000014d0       ??__E?_Iostream_object@?$_Error_objects@H@std@@2V_Iostream_error_category@2@A@@YAXXZ 100024d0 f   moc_GorIVPlugin.obj
 0001:000014e0       ??__E?_System_object@?$_Error_objects@H@std@@2V_System_error_category@2@A@@YAXXZ 100024e0 f   moc_GorIVPlugin.obj
 0001:000014f0       ??__E?staticMetaObject@SecStructPredictPlugin@U2@@2UQMetaObject@@B@@YAXXZ 100024f0 f   moc_GorIVPlugin.obj
 0001:00001500       ??__Edummy@?A0xa2c253da@@YAXXZ 10002500 f   qrc_gor4.obj
 0001:00001d66       __catch$?_Copy@?$basic_string@DU?$char_traits@D@std@@V?$allocator@D@2@@std@@QAEXII@Z$0 10002d66 f i GorIVAlgTask.obj
 0001:00001da3       __catch$?_Copy@?$basic_string@DU?$char_traits@D@std@@V?$allocator@D@2@@std@@QAEXII@Z$1 10002da3 f i GorIVAlgTask.obj
 0001:00002df5       __catch$?append@?$QList@PAVAnnotationSettings@U2@@@@QAEXABQAVAnnotationSettings@U2@@@Z$4 10003df5 f i GorIVPlugin.obj
 0001:00002e7d       __catch$?append@?$QList@VQString@@@@QAEXABVQString@@@Z$0 10003e7d f i GorIVPlugin.obj
 0001:00002ece       __catch$?append@?$QList@VQString@@@@QAEXABVQString@@@Z$4 10003ece f i GorIVPlugin.obj
 0001:000030b1       __catch$?detach_helper_grow@?$QList@PAVAnnotationSettings@U2@@@@AAEPAUNode@1@HH@Z$0 100040b1 f i GorIVPlugin.obj
 0001:000030b1       __catch$?detach_helper_grow@?$QList@PAVAnnotationSettings@U2@@@@AAEPAUNode@1@HH@Z$2 100040b1 f i GorIVPlugin.obj
 0001:000031ee       __catch$?detach_helper_grow@?$QList@VQString@@@@AAEPAUNode@1@HH@Z$2 100041ee f i GorIVPlugin.obj
 0001:00003229       __catch$?detach_helper_grow@?$QList@VQString@@@@AAEPAUNode@1@HH@Z$0 10004229 f i GorIVPlugin.obj
 0001:00003372       __catch$?node_copy@?$QList@VQString@@@@AAEXPAUNode@1@00@Z$2 10004372 f i GorIVPlugin.obj
 0001:00003698       $LN100                     10004698     gor.obj
 0001:000036ac       $LN94                      100046ac     gor.obj
 0001:000036c4       $LN101                     100046c4     gor.obj
 0001:000036d8       $LN95                      100046d8     gor.obj
 0001:000036f0       $LN102                     100046f0     gor.obj
 0001:00003704       $LN96                      10004704     gor.obj
 0001:00003f34       $LN203                     10004f34     gor.obj
 0001:00003f48       $LN198                     10004f48     gor.obj
 0001:0000442c       $LN144                     1000542c     gor.obj
 0001:00004440       $LN136                     10005440     gor.obj
 0001:00004458       $LN145                     10005458     gor.obj
 0001:0000446c       $LN137                     1000546c     gor.obj
 0001:00004484       $LN146                     10005484     gor.obj
 0001:00004498       $LN138                     10005498     gor.obj
 0001:000044b0       $LN147                     100054b0     gor.obj
 0001:000044c4       $LN139                     100054c4     gor.obj
 0001:0000453c       $LN14                      1000553c     gor.obj
 0001:00004550       $LN12                      10005550     gor.obj
 0001:00005394       $LN30                      10006394     gor.obj
 0001:000053f0       $LN28                      100063f0     gor.obj
 0001:000065ec       _pre_c_init                100075ec f   MSVCRT:crtdll.obj
 0001:00006859       ___DllMainCRTStartup       10007859 f   MSVCRT:crtdll.obj
 0001:000069b0       $$000000                   100079b0     MSVCRT:sehprolg4.obj
 0001:00006dc5       ?ArrayUnwindFilter@@YAHPAU_EXCEPTION_POINTERS@@@Z 10007dc5 f   MSVCRT:ehvecdtr.obj
 0001:00007110       __unwindfunclet$??0GorIVAlgTask@U2@@QAE@ABVQByteArray@@@Z$0 10008110 f   GorIVAlgTask.obj
 0001:00007119       __unwindfunclet$??0GorIVAlgTask@U2@@QAE@ABVQByteArray@@@Z$1 10008119 f   GorIVAlgTask.obj
 0001:00007127       __unwindfunclet$??0GorIVAlgTask@U2@@QAE@ABVQByteArray@@@Z$2 10008127 f   GorIVAlgTask.obj
 0001:00007130       __unwindfunclet$??0GorIVAlgTask@U2@@QAE@ABVQByteArray@@@Z$3 10008130 f   GorIVAlgTask.obj
 0001:00007139       __ehhandler$??0GorIVAlgTask@U2@@QAE@ABVQByteArray@@@Z 10008139 f   GorIVAlgTask.obj
 0001:00007160       __unwindfunclet$??__EalgoLog@U2@@YAXXZ$0 10008160 f   GorIVAlgTask.obj
 0001:00007169       __ehhandler$??__EalgoLog@U2@@YAXXZ 10008169 f   GorIVAlgTask.obj
 0001:00007190       __unwindfunclet$??__EcmdLog@U2@@YAXXZ$0 10008190 f   GorIVAlgTask.obj
 0001:00007199       __ehhandler$??__EcmdLog@U2@@YAXXZ 10008199 f   GorIVAlgTask.obj
 0001:000071c0       __unwindfunclet$??__EcoreLog@U2@@YAXXZ$0 100081c0 f   GorIVAlgTask.obj
 0001:000071c9       __ehhandler$??__EcoreLog@U2@@YAXXZ 100081c9 f   GorIVAlgTask.obj
 0001:000071f0       __unwindfunclet$??__EioLog@U2@@YAXXZ$0 100081f0 f   GorIVAlgTask.obj
 0001:000071f9       __ehhandler$??__EioLog@U2@@YAXXZ 100081f9 f   GorIVAlgTask.obj
 0001:00007220       __unwindfunclet$??__EperfLog@U2@@YAXXZ$0 10008220 f   GorIVAlgTask.obj
 0001:00007229       __ehhandler$??__EperfLog@U2@@YAXXZ 10008229 f   GorIVAlgTask.obj
 0001:00007250       __unwindfunclet$??__EscriptLog@U2@@YAXXZ$0 10008250 f   GorIVAlgTask.obj
 0001:00007259       __ehhandler$??__EscriptLog@U2@@YAXXZ 10008259 f   GorIVAlgTask.obj
 0001:00007280       __unwindfunclet$??__EtaskLog@U2@@YAXXZ$0 10008280 f   GorIVAlgTask.obj
 0001:00007289       __ehhandler$??__EtaskLog@U2@@YAXXZ 10008289 f   GorIVAlgTask.obj
 0001:000072b0       __unwindfunclet$??__EuiLog@U2@@YAXXZ$0 100082b0 f   GorIVAlgTask.obj
 0001:000072b9       __ehhandler$??__EuiLog@U2@@YAXXZ 100082b9 f   GorIVAlgTask.obj
 0001:000072e0       __unwindfunclet$??__EuserActLog@U2@@YAXXZ$0 100082e0 f   GorIVAlgTask.obj
 0001:000072e9       __ehhandler$??__EuserActLog@U2@@YAXXZ 100082e9 f   GorIVAlgTask.obj
 0001:00007310       __ehhandler$?_Copy@?$basic_string@DU?$char_traits@D@std@@V?$allocator@D@2@@std@@QAEXII@Z 10008310 f   GorIVAlgTask.obj
 0001:00007330       __unwindfunclet$?run@GorIVAlgTask@U2@@UAEXXZ$0 10008330 f   GorIVAlgTask.obj
 0001:00007339       __unwindfunclet$?run@GorIVAlgTask@U2@@UAEXXZ$1 10008339 f   GorIVAlgTask.obj
 0001:00007342       __unwindfunclet$?run@GorIVAlgTask@U2@@UAEXXZ$2 10008342 f   GorIVAlgTask.obj
 0001:0000734b       __unwindfunclet$?run@GorIVAlgTask@U2@@UAEXXZ$3 1000834b f   GorIVAlgTask.obj
 0001:00007354       __unwindfunclet$?run@GorIVAlgTask@U2@@UAEXXZ$4 10008354 f   GorIVAlgTask.obj
 0001:0000735d       __unwindfunclet$?run@GorIVAlgTask@U2@@UAEXXZ$5 1000835d f   GorIVAlgTask.obj
 0001:00007366       __unwindfunclet$?run@GorIVAlgTask@U2@@UAEXXZ$6 10008366 f   GorIVAlgTask.obj
 0001:0000736f       __unwindfunclet$?run@GorIVAlgTask@U2@@UAEXXZ$7 1000836f f   GorIVAlgTask.obj
 0001:00007378       __unwindfunclet$?run@GorIVAlgTask@U2@@UAEXXZ$8 10008378 f   GorIVAlgTask.obj
 0001:00007381       __ehhandler$?run@GorIVAlgTask@U2@@UAEXXZ 10008381 f   GorIVAlgTask.obj
 0001:000073a0       __unwindfunclet$??0SecStructPredictPlugin@U2@@QAE@XZ$0 100083a0 f   GorIVPlugin.obj
 0001:000073a9       __unwindfunclet$??0SecStructPredictPlugin@U2@@QAE@XZ$1 100083a9 f   GorIVPlugin.obj
 0001:000073b2       __unwindfunclet$??0SecStructPredictPlugin@U2@@QAE@XZ$2 100083b2 f   GorIVPlugin.obj
 0001:000073bb       __unwindfunclet$??0SecStructPredictPlugin@U2@@QAE@XZ$4 100083bb f   GorIVPlugin.obj
 0001:000073c6       __unwindfunclet$??0SecStructPredictPlugin@U2@@QAE@XZ$5 100083c6 f   GorIVPlugin.obj
 0001:000073e0       __unwindfunclet$??0SecStructPredictPlugin@U2@@QAE@XZ$6 100083e0 f   GorIVPlugin.obj
 0001:000073e8       __ehhandler$??0SecStructPredictPlugin@U2@@QAE@XZ 100083e8 f   GorIVPlugin.obj
 0001:00007410       __unwindfunclet$??__EalgoLog@U2@@YAXXZ$0 10008410 f   GorIVPlugin.obj
 0001:00007419       __ehhandler$??__EalgoLog@U2@@YAXXZ 10008419 f   GorIVPlugin.obj
 0001:00007440       __unwindfunclet$??__EcmdLog@U2@@YAXXZ$0 10008440 f   GorIVPlugin.obj
 0001:00007449       __ehhandler$??__EcmdLog@U2@@YAXXZ 10008449 f   GorIVPlugin.obj
 0001:00007470       __unwindfunclet$??__EcoreLog@U2@@YAXXZ$0 10008470 f   GorIVPlugin.obj
 0001:00007479       __ehhandler$??__EcoreLog@U2@@YAXXZ 10008479 f   GorIVPlugin.obj
 0001:000074a0       __unwindfunclet$??__EioLog@U2@@YAXXZ$0 100084a0 f   GorIVPlugin.obj
 0001:000074a9       __ehhandler$??__EioLog@U2@@YAXXZ 100084a9 f   GorIVPlugin.obj
 0001:000074d0       __unwindfunclet$??__EperfLog@U2@@YAXXZ$0 100084d0 f   GorIVPlugin.obj
 0001:000074d9       __ehhandler$??__EperfLog@U2@@YAXXZ 100084d9 f   GorIVPlugin.obj
 0001:00007500       __unwindfunclet$??__EscriptLog@U2@@YAXXZ$0 10008500 f   GorIVPlugin.obj
 0001:00007509       __ehhandler$??__EscriptLog@U2@@YAXXZ 10008509 f   GorIVPlugin.obj
 0001:00007530       __unwindfunclet$??__EtaskLog@U2@@YAXXZ$0 10008530 f   GorIVPlugin.obj
 0001:00007539       __ehhandler$??__EtaskLog@U2@@YAXXZ 10008539 f   GorIVPlugin.obj
 0001:00007560       __unwindfunclet$??__EuiLog@U2@@YAXXZ$0 10008560 f   GorIVPlugin.obj
 0001:00007569       __ehhandler$??__EuiLog@U2@@YAXXZ 10008569 f   GorIVPlugin.obj
 0001:00007590       __unwindfunclet$??__EuserActLog@U2@@YAXXZ$0 10008590 f   GorIVPlugin.obj
 0001:00007599       __ehhandler$??__EuserActLog@U2@@YAXXZ 10008599 f   GorIVPlugin.obj
 0001:000075c0       __ehhandler$?append@?$QList@PAVAnnotationSettings@U2@@@@QAEXABQAVAnnotationSettings@U2@@@Z 100085c0 f   GorIVPlugin.obj
 0001:000075e0       __unwindfunclet$?append@?$QList@VQString@@@@QAEXABVQString@@@Z$7 100085e0 f   GorIVPlugin.obj
 0001:000075f1       __unwindfunclet$?append@?$QList@VQString@@@@QAEXABVQString@@@Z$11 100085f1 f   GorIVPlugin.obj
 0001:00007602       __ehhandler$?append@?$QList@VQString@@@@QAEXABVQString@@@Z 10008602 f   GorIVPlugin.obj
 0001:00007620       __unwindfunclet$?createTaskInstance@Factory@GorIVAlgTask@U2@@UAEPAVSecStructPredictTask@3@ABVQByteArray@@@Z$0 10008620 f   GorIVPlugin.obj
 0001:0000762b       __ehhandler$?createTaskInstance@Factory@GorIVAlgTask@U2@@UAEPAVSecStructPredictTask@3@ABVQByteArray@@@Z 1000862b f   GorIVPlugin.obj
 0001:00007650       __ehhandler$?detach_helper_grow@?$QList@PAVAnnotationSettings@U2@@@@AAEPAUNode@1@HH@Z 10008650 f   GorIVPlugin.obj
 0001:00007670       __ehhandler$?detach_helper_grow@?$QList@VQString@@@@AAEPAUNode@1@HH@Z 10008670 f   GorIVPlugin.obj
 0001:00007690       __unwindfunclet$?node_construct@?$QList@VQString@@@@AAEXPAUNode@1@ABVQString@@@Z$1 10008690 f   GorIVPlugin.obj
 0001:000076a1       __ehhandler$?node_construct@?$QList@VQString@@@@AAEXPAUNode@1@ABVQString@@@Z 100086a1 f   GorIVPlugin.obj
 0001:000076c0       __unwindfunclet$?node_copy@?$QList@VQString@@@@AAEXPAUNode@1@00@Z$5 100086c0 f   GorIVPlugin.obj
 0001:000076d1       __ehhandler$?node_copy@?$QList@VQString@@@@AAEXPAUNode@1@00@Z 100086d1 f   GorIVPlugin.obj
 0001:000076f0       __unwindfunclet$??__EalgoLog@U2@@YAXXZ$0 100086f0 f   gor.obj
 0001:000076f9       __ehhandler$??__EalgoLog@U2@@YAXXZ 100086f9 f   gor.obj
 0001:00007720       __unwindfunclet$??__EcmdLog@U2@@YAXXZ$0 10008720 f   gor.obj
 0001:00007729       __ehhandler$??__EcmdLog@U2@@YAXXZ 10008729 f   gor.obj
 0001:00007750       __unwindfunclet$??__EcoreLog@U2@@YAXXZ$0 10008750 f   gor.obj
 0001:00007759       __ehhandler$??__EcoreLog@U2@@YAXXZ 10008759 f   gor.obj
 0001:00007780       __unwindfunclet$??__EioLog@U2@@YAXXZ$0 10008780 f   gor.obj
 0001:00007789       __ehhandler$??__EioLog@U2@@YAXXZ 10008789 f   gor.obj
 0001:000077b0       __unwindfunclet$??__EperfLog@U2@@YAXXZ$0 100087b0 f   gor.obj
 0001:000077b9       __ehhandler$??__EperfLog@U2@@YAXXZ 100087b9 f   gor.obj
 0001:000077e0       __unwindfunclet$??__EscriptLog@U2@@YAXXZ$0 100087e0 f   gor.obj
 0001:000077e9       __ehhandler$??__EscriptLog@U2@@YAXXZ 100087e9 f   gor.obj
 0001:00007810       __unwindfunclet$??__EtaskLog@U2@@YAXXZ$0 10008810 f   gor.obj
 0001:00007819       __ehhandler$??__EtaskLog@U2@@YAXXZ 10008819 f   gor.obj
 0001:00007840       __unwindfunclet$??__EuiLog@U2@@YAXXZ$0 10008840 f   gor.obj
 0001:00007849       __ehhandler$??__EuiLog@U2@@YAXXZ 10008849 f   gor.obj
 0001:00007870       __unwindfunclet$??__EuserActLog@U2@@YAXXZ$0 10008870 f   gor.obj
 0001:00007879       __ehhandler$??__EuserActLog@U2@@YAXXZ 10008879 f   gor.obj
 0001:000078a0       __unwindfunclet$?Indices@@YAXHPAH0AAVU2OpStatus@U2@@@Z$0 100088a0 f   gor.obj
 0001:000078a9       __unwindfunclet$?Indices@@YAXHPAH0AAVU2OpStatus@U2@@@Z$1 100088a9 f   gor.obj
 0001:000078b2       __unwindfunclet$?Indices@@YAXHPAH0AAVU2OpStatus@U2@@@Z$2 100088b2 f   gor.obj
 0001:000078bb       __ehhandler$?Indices@@YAXHPAH0AAVU2OpStatus@U2@@@Z 100088bb f   gor.obj
 0001:000078e0       __unwindfunclet$?readFile@@YAXAAVQFile@@HPAPAD1PAHAAVU2OpStatus@U2@@@Z$0 100088e0 f   gor.obj
 0001:000078e9       __unwindfunclet$?readFile@@YAXAAVQFile@@HPAPAD1PAHAAVU2OpStatus@U2@@@Z$1 100088e9 f   gor.obj
 0001:000078f2       __unwindfunclet$?readFile@@YAXAAVQFile@@HPAPAD1PAHAAVU2OpStatus@U2@@@Z$2 100088f2 f   gor.obj
 0001:000078fb       __unwindfunclet$?readFile@@YAXAAVQFile@@HPAPAD1PAHAAVU2OpStatus@U2@@@Z$6 100088fb f   gor.obj
 0001:00007904       __unwindfunclet$?readFile@@YAXAAVQFile@@HPAPAD1PAHAAVU2OpStatus@U2@@@Z$7 10008904 f   gor.obj
 0001:0000790d       __unwindfunclet$?readFile@@YAXAAVQFile@@HPAPAD1PAHAAVU2OpStatus@U2@@@Z$8 1000890d f   gor.obj
 0001:00007916       __unwindfunclet$?readFile@@YAXAAVQFile@@HPAPAD1PAHAAVU2OpStatus@U2@@@Z$9 10008916 f   gor.obj
 0001:0000791f       __unwindfunclet$?readFile@@YAXAAVQFile@@HPAPAD1PAHAAVU2OpStatus@U2@@@Z$10 1000891f f   gor.obj
 0001:00007928       __unwindfunclet$?readFile@@YAXAAVQFile@@HPAPAD1PAHAAVU2OpStatus@U2@@@Z$11 10008928 f   gor.obj
 0001:00007931       __unwindfunclet$?readFile@@YAXAAVQFile@@HPAPAD1PAHAAVU2OpStatus@U2@@@Z$3 10008931 f   gor.obj
 0001:0000793a       __unwindfunclet$?readFile@@YAXAAVQFile@@HPAPAD1PAHAAVU2OpStatus@U2@@@Z$4 1000893a f   gor.obj
 0001:00007943       __unwindfunclet$?readFile@@YAXAAVQFile@@HPAPAD1PAHAAVU2OpStatus@U2@@@Z$5 10008943 f   gor.obj
 0001:0000794c       __ehhandler$?readFile@@YAXAAVQFile@@HPAPAD1PAHAAVU2OpStatus@U2@@@Z 1000894c f   gor.obj
 0001:00007970       __unwindfunclet$?runGORIV@@YAHAAVQFile@@0PADH1AAVU2OpStatus@U2@@@Z$0 10008970 f   gor.obj
 0001:00007979       __unwindfunclet$?runGORIV@@YAHAAVQFile@@0PADH1AAVU2OpStatus@U2@@@Z$1 10008979 f   gor.obj
 0001:00007982       __unwindfunclet$?runGORIV@@YAHAAVQFile@@0PADH1AAVU2OpStatus@U2@@@Z$2 10008982 f   gor.obj
 0001:0000798b       __unwindfunclet$?runGORIV@@YAHAAVQFile@@0PADH1AAVU2OpStatus@U2@@@Z$3 1000898b f   gor.obj
 0001:00007994       __unwindfunclet$?runGORIV@@YAHAAVQFile@@0PADH1AAVU2OpStatus@U2@@@Z$4 10008994 f   gor.obj
 0001:0000799d       __unwindfunclet$?runGORIV@@YAHAAVQFile@@0PADH1AAVU2OpStatus@U2@@@Z$5 1000899d f   gor.obj
 0001:000079a6       __ehhandler$?runGORIV@@YAHAAVQFile@@0PADH1AAVU2OpStatus@U2@@@Z 100089a6 f   gor.obj
 0001:000079d0       __unwindfunclet$??__EalgoLog@U2@@YAXXZ$0 100089d0 f   moc_GorIVAlgTask.obj
 0001:000079d9       __ehhandler$??__EalgoLog@U2@@YAXXZ 100089d9 f   moc_GorIVAlgTask.obj
 0001:00007a00       __unwindfunclet$??__EcmdLog@U2@@YAXXZ$0 10008a00 f   moc_GorIVAlgTask.obj
 0001:00007a09       __ehhandler$??__EcmdLog@U2@@YAXXZ 10008a09 f   moc_GorIVAlgTask.obj
 0001:00007a30       __unwindfunclet$??__EcoreLog@U2@@YAXXZ$0 10008a30 f   moc_GorIVAlgTask.obj
 0001:00007a39       __ehhandler$??__EcoreLog@U2@@YAXXZ 10008a39 f   moc_GorIVAlgTask.obj
 0001:00007a60       __unwindfunclet$??__EioLog@U2@@YAXXZ$0 10008a60 f   moc_GorIVAlgTask.obj
 0001:00007a69       __ehhandler$??__EioLog@U2@@YAXXZ 10008a69 f   moc_GorIVAlgTask.obj
 0001:00007a90       __unwindfunclet$??__EperfLog@U2@@YAXXZ$0 10008a90 f   moc_GorIVAlgTask.obj
 0001:00007a99       __ehhandler$??__EperfLog@U2@@YAXXZ 10008a99 f   moc_GorIVAlgTask.obj
 0001:00007ac0       __unwindfunclet$??__EscriptLog@U2@@YAXXZ$0 10008ac0 f   moc_GorIVAlgTask.obj
 0001:00007ac9       __ehhandler$??__EscriptLog@U2@@YAXXZ 10008ac9 f   moc_GorIVAlgTask.obj
 0001:00007af0       __unwindfunclet$??__EtaskLog@U2@@YAXXZ$0 10008af0 f   moc_GorIVAlgTask.obj
 0001:00007af9       __ehhandler$??__EtaskLog@U2@@YAXXZ 10008af9 f   moc_GorIVAlgTask.obj
 0001:00007b20       __unwindfunclet$??__EuiLog@U2@@YAXXZ$0 10008b20 f   moc_GorIVAlgTask.obj
 0001:00007b29       __ehhandler$??__EuiLog@U2@@YAXXZ 10008b29 f   moc_GorIVAlgTask.obj
 0001:00007b50       __unwindfunclet$??__EuserActLog@U2@@YAXXZ$0 10008b50 f   moc_GorIVAlgTask.obj
 0001:00007b59       __ehhandler$??__EuserActLog@U2@@YAXXZ 10008b59 f   moc_GorIVAlgTask.obj
 0001:00007b80       ??__F?_Generic_object@?$_Error_objects@H@std@@2V_Generic_error_category@2@A@@YAXXZ 10008b80 f   GorIVAlgTask.obj
 0001:00007b90       ??__F?_Iostream_object@?$_Error_objects@H@std@@2V_Iostream_error_category@2@A@@YAXXZ 10008b90 f   GorIVAlgTask.obj
 0001:00007ba0       ??__F?_System_object@?$_Error_objects@H@std@@2V_System_error_category@2@A@@YAXXZ 10008ba0 f   GorIVAlgTask.obj
 0001:00007bb0       ??__F?runLock@GorIVAlgTask@U2@@0VQMutex@@A@@YAXXZ 10008bb0 f   GorIVAlgTask.obj
 0001:00007bc0       ??__F?taskName@GorIVAlgTask@U2@@2VQString@@B@@YAXXZ 10008bc0 f   GorIVAlgTask.obj
 0001:00007bd0       ??__FService_DNAExport@U2@@YAXXZ 10008bd0 f   GorIVAlgTask.obj
 0001:00007be0       ??__FService_DNAGraphPack@U2@@YAXXZ 10008be0 f   GorIVAlgTask.obj
 0001:00007bf0       ??__FService_ExternalToolSupport@U2@@YAXXZ 10008bf0 f   GorIVAlgTask.obj
 0001:00007c00       ??__FService_GUITesting@U2@@YAXXZ 10008c00 f   GorIVAlgTask.obj
 0001:00007c10       ??__FService_MaxCoreServiceId@U2@@YAXXZ 10008c10 f   GorIVAlgTask.obj
 0001:00007c20       ??__FService_MinCoreServiceId@U2@@YAXXZ 10008c20 f   GorIVAlgTask.obj
 0001:00007c30       ??__FService_PluginViewer@U2@@YAXXZ 10008c30 f   GorIVAlgTask.obj
 0001:00007c40       ??__FService_Project@U2@@YAXXZ 10008c40 f   GorIVAlgTask.obj
 0001:00007c50       ??__FService_ProjectView@U2@@YAXXZ 10008c50 f   GorIVAlgTask.obj
 0001:00007c60       ??__FService_QueryDesigner@U2@@YAXXZ 10008c60 f   GorIVAlgTask.obj
 0001:00007c70       ??__FService_ScriptRegistry@U2@@YAXXZ 10008c70 f   GorIVAlgTask.obj
 0001:00007c80       ??__FService_TestRunner@U2@@YAXXZ 10008c80 f   GorIVAlgTask.obj
 0001:00007c90       ??__FService_WorkflowDesigner@U2@@YAXXZ 10008c90 f   GorIVAlgTask.obj
 0001:00007ca0       ??__FalgoLog@U2@@YAXXZ     10008ca0 f   GorIVAlgTask.obj
 0001:00007cb0       ??__FcmdLog@U2@@YAXXZ      10008cb0 f   GorIVAlgTask.obj
 0001:00007cc0       ??__FcoreLog@U2@@YAXXZ     10008cc0 f   GorIVAlgTask.obj
 0001:00007cd0       ??__Fcvar@?1???0GorIVAlgTask@U2@@QAE@ABVQByteArray@@@Z@YAXXZ 10008cd0 f   GorIVAlgTask.obj
 0001:00007ce0       ??__FioLog@U2@@YAXXZ       10008ce0 f   GorIVAlgTask.obj
 0001:00007cf0       ??__FperfLog@U2@@YAXXZ     10008cf0 f   GorIVAlgTask.obj
 0001:00007d00       ??__FscriptLog@U2@@YAXXZ   10008d00 f   GorIVAlgTask.obj
 0001:00007d10       ??__FtaskLog@U2@@YAXXZ     10008d10 f   GorIVAlgTask.obj
 0001:00007d20       ??__FuiLog@U2@@YAXXZ       10008d20 f   GorIVAlgTask.obj
 0001:00007d30       ??__FuserActLog@U2@@YAXXZ  10008d30 f   GorIVAlgTask.obj
 0001:00007d40       ??__F?_Generic_object@?$_Error_objects@H@std@@2V_Generic_error_category@2@A@@YAXXZ 10008d40 f   GorIVPlugin.obj
 0001:00007d50       ??__F?_Iostream_object@?$_Error_objects@H@std@@2V_Iostream_error_category@2@A@@YAXXZ 10008d50 f   GorIVPlugin.obj
 0001:00007d60       ??__F?_System_object@?$_Error_objects@H@std@@2V_System_error_category@2@A@@YAXXZ 10008d60 f   GorIVPlugin.obj
 0001:00007d70       ??__FService_DNAExport@U2@@YAXXZ 10008d70 f   GorIVPlugin.obj
 0001:00007d80       ??__FService_DNAGraphPack@U2@@YAXXZ 10008d80 f   GorIVPlugin.obj
 0001:00007d90       ??__FService_ExternalToolSupport@U2@@YAXXZ 10008d90 f   GorIVPlugin.obj
 0001:00007da0       ??__FService_GUITesting@U2@@YAXXZ 10008da0 f   GorIVPlugin.obj
 0001:00007db0       ??__FService_MaxCoreServiceId@U2@@YAXXZ 10008db0 f   GorIVPlugin.obj
 0001:00007dc0       ??__FService_MinCoreServiceId@U2@@YAXXZ 10008dc0 f   GorIVPlugin.obj
 0001:00007dd0       ??__FService_PluginViewer@U2@@YAXXZ 10008dd0 f   GorIVPlugin.obj
 0001:00007de0       ??__FService_Project@U2@@YAXXZ 10008de0 f   GorIVPlugin.obj
 0001:00007df0       ??__FService_ProjectView@U2@@YAXXZ 10008df0 f   GorIVPlugin.obj
 0001:00007e00       ??__FService_QueryDesigner@U2@@YAXXZ 10008e00 f   GorIVPlugin.obj
 0001:00007e10       ??__FService_ScriptRegistry@U2@@YAXXZ 10008e10 f   GorIVPlugin.obj
 0001:00007e20       ??__FService_TestRunner@U2@@YAXXZ 10008e20 f   GorIVPlugin.obj
 0001:00007e30       ??__FService_WorkflowDesigner@U2@@YAXXZ 10008e30 f   GorIVPlugin.obj
 0001:00007e40       ??__FalgoLog@U2@@YAXXZ     10008e40 f   GorIVPlugin.obj
 0001:00007e50       ??__FcmdLog@U2@@YAXXZ      10008e50 f   GorIVPlugin.obj
 0001:00007e60       ??__FcoreLog@U2@@YAXXZ     10008e60 f   GorIVPlugin.obj
 0001:00007e70       ??__FioLog@U2@@YAXXZ       10008e70 f   GorIVPlugin.obj
 0001:00007e80       ??__FperfLog@U2@@YAXXZ     10008e80 f   GorIVPlugin.obj
 0001:00007e90       ??__FscriptLog@U2@@YAXXZ   10008e90 f   GorIVPlugin.obj
 0001:00007ea0       ??__FtaskLog@U2@@YAXXZ     10008ea0 f   GorIVPlugin.obj
 0001:00007eb0       ??__FuiLog@U2@@YAXXZ       10008eb0 f   GorIVPlugin.obj
 0001:00007ec0       ??__FuserActLog@U2@@YAXXZ  10008ec0 f   GorIVPlugin.obj
 0001:00007ed0       ??__F?_Generic_object@?$_Error_objects@H@std@@2V_Generic_error_category@2@A@@YAXXZ 10008ed0 f   gor.obj
 0001:00007ee0       ??__F?_Iostream_object@?$_Error_objects@H@std@@2V_Iostream_error_category@2@A@@YAXXZ 10008ee0 f   gor.obj
 0001:00007ef0       ??__F?_System_object@?$_Error_objects@H@std@@2V_System_error_category@2@A@@YAXXZ 10008ef0 f   gor.obj
 0001:00007f00       ??__FalgoLog@U2@@YAXXZ     10008f00 f   gor.obj
 0001:00007f10       ??__FcmdLog@U2@@YAXXZ      10008f10 f   gor.obj
 0001:00007f20       ??__FcoreLog@U2@@YAXXZ     10008f20 f   gor.obj
 0001:00007f30       ??__FioLog@U2@@YAXXZ       10008f30 f   gor.obj
 0001:00007f40       ??__FperfLog@U2@@YAXXZ     10008f40 f   gor.obj
 0001:00007f50       ??__FscriptLog@U2@@YAXXZ   10008f50 f   gor.obj
 0001:00007f60       ??__FtaskLog@U2@@YAXXZ     10008f60 f   gor.obj
 0001:00007f70       ??__FuiLog@U2@@YAXXZ       10008f70 f   gor.obj
 0001:00007f80       ??__FuserActLog@U2@@YAXXZ  10008f80 f   gor.obj
 0001:00007f90       ??__F?_Generic_object@?$_Error_objects@H@std@@2V_Generic_error_category@2@A@@YAXXZ 10008f90 f   moc_GorIVAlgTask.obj
 0001:00007fa0       ??__F?_Iostream_object@?$_Error_objects@H@std@@2V_Iostream_error_category@2@A@@YAXXZ 10008fa0 f   moc_GorIVAlgTask.obj
 0001:00007fb0       ??__F?_System_object@?$_Error_objects@H@std@@2V_System_error_category@2@A@@YAXXZ 10008fb0 f   moc_GorIVAlgTask.obj
 0001:00007fc0       ??__FalgoLog@U2@@YAXXZ     10008fc0 f   moc_GorIVAlgTask.obj
 0001:00007fd0       ??__FcmdLog@U2@@YAXXZ      10008fd0 f   moc_GorIVAlgTask.obj
 0001:00007fe0       ??__FcoreLog@U2@@YAXXZ     10008fe0 f   moc_GorIVAlgTask.obj
 0001:00007ff0       ??__FioLog@U2@@YAXXZ       10008ff0 f   moc_GorIVAlgTask.obj
 0001:00008000       ??__FperfLog@U2@@YAXXZ     10009000 f   moc_GorIVAlgTask.obj
 0001:00008010       ??__FscriptLog@U2@@YAXXZ   10009010 f   moc_GorIVAlgTask.obj
 0001:00008020       ??__FtaskLog@U2@@YAXXZ     10009020 f   moc_GorIVAlgTask.obj
 0001:00008030       ??__FuiLog@U2@@YAXXZ       10009030 f   moc_GorIVAlgTask.obj
 0001:00008040       ??__FuserActLog@U2@@YAXXZ  10009040 f   moc_GorIVAlgTask.obj
 0001:00008050       ??__F?_Generic_object@?$_Error_objects@H@std@@2V_Generic_error_category@2@A@@YAXXZ 10009050 f   moc_GorIVPlugin.obj
 0001:00008060       ??__F?_Iostream_object@?$_Error_objects@H@std@@2V_Iostream_error_category@2@A@@YAXXZ 10009060 f   moc_GorIVPlugin.obj
 0001:00008070       ??__F?_System_object@?$_Error_objects@H@std@@2V_System_error_category@2@A@@YAXXZ 10009070 f   moc_GorIVPlugin.obj
 0001:00008080       ??__Fdummy@?A0xa2c253da@@YAXXZ 10009080 f   qrc_gor4.obj
 0002:0000025c       _algoLog$initializer$      1000a25c     GorIVAlgTask.obj
 0002:00000260       _cmdLog$initializer$       1000a260     GorIVAlgTask.obj
 0002:00000264       _coreLog$initializer$      1000a264     GorIVAlgTask.obj
 0002:00000268       _ioLog$initializer$        1000a268     GorIVAlgTask.obj
 0002:0000026c       _perfLog$initializer$      1000a26c     GorIVAlgTask.obj
 0002:00000270       _scriptLog$initializer$    1000a270     GorIVAlgTask.obj
 0002:00000274       _taskLog$initializer$      1000a274     GorIVAlgTask.obj
 0002:00000278       _uiLog$initializer$        1000a278     GorIVAlgTask.obj
 0002:0000027c       _userActLog$initializer$   1000a27c     GorIVAlgTask.obj
 0002:00000280       _Service_PluginViewer$initializer$ 1000a280     GorIVAlgTask.obj
 0002:00000284       _Service_Project$initializer$ 1000a284     GorIVAlgTask.obj
 0002:00000288       _Service_ProjectView$initializer$ 1000a288     GorIVAlgTask.obj
 0002:0000028c       _Service_DNAGraphPack$initializer$ 1000a28c     GorIVAlgTask.obj
 0002:00000290       _Service_DNAExport$initializer$ 1000a290     GorIVAlgTask.obj
 0002:00000294       _Service_TestRunner$initializer$ 1000a294     GorIVAlgTask.obj
 0002:00000298       _Service_ScriptRegistry$initializer$ 1000a298     GorIVAlgTask.obj
 0002:0000029c       _Service_ExternalToolSupport$initializer$ 1000a29c     GorIVAlgTask.obj
 0002:000002a0       _Service_GUITesting$initializer$ 1000a2a0     GorIVAlgTask.obj
 0002:000002a4       _Service_WorkflowDesigner$initializer$ 1000a2a4     GorIVAlgTask.obj
 0002:000002a8       _Service_QueryDesigner$initializer$ 1000a2a8     GorIVAlgTask.obj
 0002:000002ac       _Service_MinCoreServiceId$initializer$ 1000a2ac     GorIVAlgTask.obj
 0002:000002b0       _Service_MaxCoreServiceId$initializer$ 1000a2b0     GorIVAlgTask.obj
 0002:000002b4       ?taskName$initializer$@GorIVAlgTask@U2@@2P6AXXZA 1000a2b4     GorIVAlgTask.obj
 0002:000002b8       ?runLock$initializer$@GorIVAlgTask@U2@@0P6AXXZA 1000a2b8     GorIVAlgTask.obj
 0002:000002bc       ?_Generic_object$initializer$@?$_Error_objects@H@std@@2P6AXXZA 1000a2bc     GorIVAlgTask.obj
 0002:000002c0       ?_Iostream_object$initializer$@?$_Error_objects@H@std@@2P6AXXZA 1000a2c0     GorIVAlgTask.obj
 0002:000002c4       ?_System_object$initializer$@?$_Error_objects@H@std@@2P6AXXZA 1000a2c4     GorIVAlgTask.obj
 0002:000002c8       _algoLog$initializer$      1000a2c8     GorIVPlugin.obj
 0002:000002cc       _cmdLog$initializer$       1000a2cc     GorIVPlugin.obj
 0002:000002d0       _coreLog$initializer$      1000a2d0     GorIVPlugin.obj
 0002:000002d4       _ioLog$initializer$        1000a2d4     GorIVPlugin.obj
 0002:000002d8       _perfLog$initializer$      1000a2d8     GorIVPlugin.obj
 0002:000002dc       _scriptLog$initializer$    1000a2dc     GorIVPlugin.obj
 0002:000002e0       _taskLog$initializer$      1000a2e0     GorIVPlugin.obj
 0002:000002e4       _uiLog$initializer$        1000a2e4     GorIVPlugin.obj
 0002:000002e8       _userActLog$initializer$   1000a2e8     GorIVPlugin.obj
 0002:000002ec       _Service_PluginViewer$initializer$ 1000a2ec     GorIVPlugin.obj
 0002:000002f0       _Service_Project$initializer$ 1000a2f0     GorIVPlugin.obj
 0002:000002f4       _Service_ProjectView$initializer$ 1000a2f4     GorIVPlugin.obj
 0002:000002f8       _Service_DNAGraphPack$initializer$ 1000a2f8     GorIVPlugin.obj
 0002:000002fc       _Service_DNAExport$initializer$ 1000a2fc     GorIVPlugin.obj
 0002:00000300       _Service_TestRunner$initializer$ 1000a300     GorIVPlugin.obj
 0002:00000304       _Service_ScriptRegistry$initializer$ 1000a304     GorIVPlugin.obj
 0002:00000308       _Service_ExternalToolSupport$initializer$ 1000a308     GorIVPlugin.obj
 0002:0000030c       _Service_GUITesting$initializer$ 1000a30c     GorIVPlugin.obj
 0002:00000310       _Service_WorkflowDesigner$initializer$ 1000a310     GorIVPlugin.obj
 0002:00000314       _Service_QueryDesigner$initializer$ 1000a314     GorIVPlugin.obj
 0002:00000318       _Service_MinCoreServiceId$initializer$ 1000a318     GorIVPlugin.obj
 0002:0000031c       _Service_MaxCoreServiceId$initializer$ 1000a31c     GorIVPlugin.obj
 0002:00000320       _algoLog$initializer$      1000a320     gor.obj
 0002:00000324       _cmdLog$initializer$       1000a324     gor.obj
 0002:00000328       _coreLog$initializer$      1000a328     gor.obj
 0002:0000032c       _ioLog$initializer$        1000a32c     gor.obj
 0002:00000330       _perfLog$initializer$      1000a330     gor.obj
 0002:00000334       _scriptLog$initializer$    1000a334     gor.obj
 0002:00000338       _taskLog$initializer$      1000a338     gor.obj
 0002:0000033c       _uiLog$initializer$        1000a33c     gor.obj
 0002:00000340       _userActLog$initializer$   1000a340     gor.obj
 0002:00000344       _algoLog$initializer$      1000a344     moc_GorIVAlgTask.obj
 0002:00000348       _cmdLog$initializer$       1000a348     moc_GorIVAlgTask.obj
 0002:0000034c       _coreLog$initializer$      1000a34c     moc_GorIVAlgTask.obj
 0002:00000350       _ioLog$initializer$        1000a350     moc_GorIVAlgTask.obj
 0002:00000354       _perfLog$initializer$      1000a354     moc_GorIVAlgTask.obj
 0002:00000358       _scriptLog$initializer$    1000a358     moc_GorIVAlgTask.obj
 0002:0000035c       _taskLog$initializer$      1000a35c     moc_GorIVAlgTask.obj
 0002:00000360       _uiLog$initializer$        1000a360     moc_GorIVAlgTask.obj
 0002:00000364       _userActLog$initializer$   1000a364     moc_GorIVAlgTask.obj
 0002:00000368       ?staticMetaObject$initializer$@GorIVAlgTask@U2@@2P6AXXZA 1000a368     moc_GorIVAlgTask.obj
 0002:0000036c       ?staticMetaObject$initializer$@SecStructPredictPlugin@U2@@2P6AXXZA 1000a36c     moc_GorIVPlugin.obj
 0002:00000370       _dummy$initializer$        1000a370     qrc_gor4.obj
 0002:0000037c       _pcinit                    1000a37c     MSVCRT:crtdll.obj
 0002:00000380       _pinit                     1000a380     MSVCRT:atonexit.obj
 0002:0000071c       _ExpInv                    1000a71c     gor.obj
 0002:00000720       _conf                      1000a720     gor.obj
 0002:00000d2c       _qt_meta_stringdata_U2__GorIVAlgTask 1000ad2c     moc_GorIVAlgTask.obj
 0002:00000d50       _qt_meta_data_U2__GorIVAlgTask 1000ad50     moc_GorIVAlgTask.obj
 0002:00000d8c       _qt_meta_stringdata_U2__SecStructPredictPlugin 1000ad8c     moc_GorIVPlugin.obj
 0002:00000db8       _qt_meta_data_U2__SecStructPredictPlugin 1000adb8     moc_GorIVPlugin.obj
 0002:00000df8       _qt_resource_data          1000adf8     qrc_gor4.obj
 0002:0001aab8       _qt_resource_name          10024ab8     qrc_gor4.obj
 0002:0001ab28       _qt_resource_struct        10024b28     qrc_gor4.obj
 0002:0001ab7c       _GS_ExceptionPointers      10024b7c     MSVCRT:gs_report.obj
 0002:0001b190       __catchsym$?_Copy@?$basic_string@DU?$char_traits@D@std@@V?$allocator@D@2@@std@@QAEXII@Z$5 10025190     GorIVAlgTask.obj
 0002:0001b1a0       __catchsym$?_Copy@?$basic_string@DU?$char_traits@D@std@@V?$allocator@D@2@@std@@QAEXII@Z$4 100251a0     GorIVAlgTask.obj
 0002:0001b1b0       __unwindtable$?_Copy@?$basic_string@DU?$char_traits@D@std@@V?$allocator@D@2@@std@@QAEXII@Z 100251b0     GorIVAlgTask.obj
 0002:0001b1d0       __ehfuncinfo$?_Copy@?$basic_string@DU?$char_traits@D@std@@V?$allocator@D@2@@std@@QAEXII@Z 100251d0     GorIVAlgTask.obj
 0002:0001b1f4       __tryblocktable$?_Copy@?$basic_string@DU?$char_traits@D@std@@V?$allocator@D@2@@std@@QAEXII@Z 100251f4     GorIVAlgTask.obj
 0002:0001b21c       __unwindtable$??__EalgoLog@U2@@YAXXZ 1002521c     GorIVAlgTask.obj
 0002:0001b224       __ehfuncinfo$??__EalgoLog@U2@@YAXXZ 10025224     GorIVAlgTask.obj
 0002:0001b248       __unwindtable$??__EcmdLog@U2@@YAXXZ 10025248     GorIVAlgTask.obj
 0002:0001b250       __ehfuncinfo$??__EcmdLog@U2@@YAXXZ 10025250     GorIVAlgTask.obj
 0002:0001b274       __unwindtable$??__EcoreLog@U2@@YAXXZ 10025274     GorIVAlgTask.obj
 0002:0001b27c       __ehfuncinfo$??__EcoreLog@U2@@YAXXZ 1002527c     GorIVAlgTask.obj
 0002:0001b2a0       __unwindtable$??__EioLog@U2@@YAXXZ 100252a0     GorIVAlgTask.obj
 0002:0001b2a8       __ehfuncinfo$??__EioLog@U2@@YAXXZ 100252a8     GorIVAlgTask.obj
 0002:0001b2cc       __unwindtable$??__EperfLog@U2@@YAXXZ 100252cc     GorIVAlgTask.obj
 0002:0001b2d4       __ehfuncinfo$??__EperfLog@U2@@YAXXZ 100252d4     GorIVAlgTask.obj
 0002:0001b2f8       __unwindtable$??__EscriptLog@U2@@YAXXZ 100252f8     GorIVAlgTask.obj
 0002:0001b300       __ehfuncinfo$??__EscriptLog@U2@@YAXXZ 10025300     GorIVAlgTask.obj
 0002:0001b324       __unwindtable$??__EtaskLog@U2@@YAXXZ 10025324     GorIVAlgTask.obj
 0002:0001b32c       __ehfuncinfo$??__EtaskLog@U2@@YAXXZ 1002532c     GorIVAlgTask.obj
 0002:0001b350       __unwindtable$??__EuiLog@U2@@YAXXZ 10025350     GorIVAlgTask.obj
 0002:0001b358       __ehfuncinfo$??__EuiLog@U2@@YAXXZ 10025358     GorIVAlgTask.obj
 0002:0001b37c       __unwindtable$??__EuserActLog@U2@@YAXXZ 1002537c     GorIVAlgTask.obj
 0002:0001b384       __ehfuncinfo$??__EuserActLog@U2@@YAXXZ 10025384     GorIVAlgTask.obj
 0002:0001b3a8       __unwindtable$??0GorIVAlgTask@U2@@QAE@ABVQByteArray@@@Z 100253a8     GorIVAlgTask.obj
 0002:0001b3c8       __ehfuncinfo$??0GorIVAlgTask@U2@@QAE@ABVQByteArray@@@Z 100253c8     GorIVAlgTask.obj
 0002:0001b3ec       __ehfuncinfo$?run@GorIVAlgTask@U2@@UAEXXZ 100253ec     GorIVAlgTask.obj
 0002:0001b410       __unwindtable$?run@GorIVAlgTask@U2@@UAEXXZ 10025410     GorIVAlgTask.obj
 0002:0001b468       __catchsym$?append@?$QList@VQString@@@@QAEXABVQString@@@Z$13 10025468     GorIVPlugin.obj
 0002:0001b478       __catchsym$?append@?$QList@VQString@@@@QAEXABVQString@@@Z$12 10025478     GorIVPlugin.obj
 0002:0001b488       __ehfuncinfo$?append@?$QList@VQString@@@@QAEXABVQString@@@Z 10025488     GorIVPlugin.obj
 0002:0001b4ac       __tryblocktable$?append@?$QList@VQString@@@@QAEXABVQString@@@Z 100254ac     GorIVPlugin.obj
 0002:0001b4d4       __unwindtable$?append@?$QList@VQString@@@@QAEXABVQString@@@Z 100254d4     GorIVPlugin.obj
 0002:0001b534       __catchsym$?detach_helper_grow@?$QList@VQString@@@@AAEPAUNode@1@HH@Z$5 10025534     GorIVPlugin.obj
 0002:0001b544       __catchsym$?detach_helper_grow@?$QList@VQString@@@@AAEPAUNode@1@HH@Z$4 10025544     GorIVPlugin.obj
 0002:0001b554       __unwindtable$?detach_helper_grow@?$QList@VQString@@@@AAEPAUNode@1@HH@Z 10025554     GorIVPlugin.obj
 0002:0001b574       __ehfuncinfo$?detach_helper_grow@?$QList@VQString@@@@AAEPAUNode@1@HH@Z 10025574     GorIVPlugin.obj
 0002:0001b598       __tryblocktable$?detach_helper_grow@?$QList@VQString@@@@AAEPAUNode@1@HH@Z 10025598     GorIVPlugin.obj
 0002:0001b5c0       __unwindtable$?node_construct@?$QList@VQString@@@@AAEXPAUNode@1@ABVQString@@@Z 100255c0     GorIVPlugin.obj
 0002:0001b5d0       __ehfuncinfo$?node_construct@?$QList@VQString@@@@AAEXPAUNode@1@ABVQString@@@Z 100255d0     GorIVPlugin.obj
 0002:0001b5f4       __catchsym$?node_copy@?$QList@VQString@@@@AAEXPAUNode@1@00@Z$6 100255f4     GorIVPlugin.obj
 0002:0001b604       __tryblocktable$?node_copy@?$QList@VQString@@@@AAEXPAUNode@1@00@Z 10025604     GorIVPlugin.obj
 0002:0001b618       __ehfuncinfo$?node_copy@?$QList@VQString@@@@AAEXPAUNode@1@00@Z 10025618     GorIVPlugin.obj
 0002:0001b63c       __unwindtable$?node_copy@?$QList@VQString@@@@AAEXPAUNode@1@00@Z 1002563c     GorIVPlugin.obj
 0002:0001b66c       __unwindtable$??__EalgoLog@U2@@YAXXZ 1002566c     GorIVPlugin.obj
 0002:0001b674       __ehfuncinfo$??__EalgoLog@U2@@YAXXZ 10025674     GorIVPlugin.obj
 0002:0001b698       __unwindtable$??__EcmdLog@U2@@YAXXZ 10025698     GorIVPlugin.obj
 0002:0001b6a0       __ehfuncinfo$??__EcmdLog@U2@@YAXXZ 100256a0     GorIVPlugin.obj
 0002:0001b6c4       __unwindtable$??__EcoreLog@U2@@YAXXZ 100256c4     GorIVPlugin.obj
 0002:0001b6cc       __ehfuncinfo$??__EcoreLog@U2@@YAXXZ 100256cc     GorIVPlugin.obj
 0002:0001b6f0       __unwindtable$??__EioLog@U2@@YAXXZ 100256f0     GorIVPlugin.obj
 0002:0001b6f8       __ehfuncinfo$??__EioLog@U2@@YAXXZ 100256f8     GorIVPlugin.obj
 0002:0001b71c       __unwindtable$??__EperfLog@U2@@YAXXZ 1002571c     GorIVPlugin.obj
 0002:0001b724       __ehfuncinfo$??__EperfLog@U2@@YAXXZ 10025724     GorIVPlugin.obj
 0002:0001b748       __unwindtable$??__EscriptLog@U2@@YAXXZ 10025748     GorIVPlugin.obj
 0002:0001b750       __ehfuncinfo$??__EscriptLog@U2@@YAXXZ 10025750     GorIVPlugin.obj
 0002:0001b774       __unwindtable$??__EtaskLog@U2@@YAXXZ 10025774     GorIVPlugin.obj
 0002:0001b77c       __ehfuncinfo$??__EtaskLog@U2@@YAXXZ 1002577c     GorIVPlugin.obj
 0002:0001b7a0       __unwindtable$??__EuiLog@U2@@YAXXZ 100257a0     GorIVPlugin.obj
 0002:0001b7a8       __ehfuncinfo$??__EuiLog@U2@@YAXXZ 100257a8     GorIVPlugin.obj
 0002:0001b7cc       __unwindtable$??__EuserActLog@U2@@YAXXZ 100257cc     GorIVPlugin.obj
 0002:0001b7d4       __ehfuncinfo$??__EuserActLog@U2@@YAXXZ 100257d4     GorIVPlugin.obj
 0002:0001b7f8       __ehfuncinfo$??0SecStructPredictPlugin@U2@@QAE@XZ 100257f8     GorIVPlugin.obj
 0002:0001b81c       __unwindtable$??0SecStructPredictPlugin@U2@@QAE@XZ 1002581c     GorIVPlugin.obj
 0002:0001b864       __unwindtable$?createTaskInstance@Factory@GorIVAlgTask@U2@@UAEPAVSecStructPredictTask@3@ABVQByteArray@@@Z 10025864     GorIVPlugin.obj
 0002:0001b86c       __ehfuncinfo$?createTaskInstance@Factory@GorIVAlgTask@U2@@UAEPAVSecStructPredictTask@3@ABVQByteArray@@@Z 1002586c     GorIVPlugin.obj
 0002:0001b890       __catchsym$?append@?$QList@PAVAnnotationSettings@U2@@@@QAEXABQAVAnnotationSettings@U2@@@Z$6 10025890     GorIVPlugin.obj
 0002:0001b8a0       __tryblocktable$?append@?$QList@PAVAnnotationSettings@U2@@@@QAEXABQAVAnnotationSettings@U2@@@Z 100258a0     GorIVPlugin.obj
 0002:0001b8b4       __ehfuncinfo$?append@?$QList@PAVAnnotationSettings@U2@@@@QAEXABQAVAnnotationSettings@U2@@@Z 100258b4     GorIVPlugin.obj
 0002:0001b8d8       __unwindtable$?append@?$QList@PAVAnnotationSettings@U2@@@@QAEXABQAVAnnotationSettings@U2@@@Z 100258d8     GorIVPlugin.obj
 0002:0001b908       __catchsym$?detach_helper_grow@?$QList@PAVAnnotationSettings@U2@@@@AAEPAUNode@1@HH@Z$5 10025908     GorIVPlugin.obj
 0002:0001b918       __catchsym$?detach_helper_grow@?$QList@PAVAnnotationSettings@U2@@@@AAEPAUNode@1@HH@Z$4 10025918     GorIVPlugin.obj
 0002:0001b928       __unwindtable$?detach_helper_grow@?$QList@PAVAnnotationSettings@U2@@@@AAEPAUNode@1@HH@Z 10025928     GorIVPlugin.obj
 0002:0001b948       __ehfuncinfo$?detach_helper_grow@?$QList@PAVAnnotationSettings@U2@@@@AAEPAUNode@1@HH@Z 10025948     GorIVPlugin.obj
 0002:0001b96c       __tryblocktable$?detach_helper_grow@?$QList@PAVAnnotationSettings@U2@@@@AAEPAUNode@1@HH@Z 1002596c     GorIVPlugin.obj
 0002:0001b994       __unwindtable$??__EalgoLog@U2@@YAXXZ 10025994     gor.obj
 0002:0001b99c       __ehfuncinfo$??__EalgoLog@U2@@YAXXZ 1002599c     gor.obj
 0002:0001b9c0       __unwindtable$??__EcmdLog@U2@@YAXXZ 100259c0     gor.obj
 0002:0001b9c8       __ehfuncinfo$??__EcmdLog@U2@@YAXXZ 100259c8     gor.obj
 0002:0001b9ec       __unwindtable$??__EcoreLog@U2@@YAXXZ 100259ec     gor.obj
 0002:0001b9f4       __ehfuncinfo$??__EcoreLog@U2@@YAXXZ 100259f4     gor.obj
 0002:0001ba18       __unwindtable$??__EioLog@U2@@YAXXZ 10025a18     gor.obj
 0002:0001ba20       __ehfuncinfo$??__EioLog@U2@@YAXXZ 10025a20     gor.obj
 0002:0001ba44       __unwindtable$??__EperfLog@U2@@YAXXZ 10025a44     gor.obj
 0002:0001ba4c       __ehfuncinfo$??__EperfLog@U2@@YAXXZ 10025a4c     gor.obj
 0002:0001ba70       __unwindtable$??__EscriptLog@U2@@YAXXZ 10025a70     gor.obj
 0002:0001ba78       __ehfuncinfo$??__EscriptLog@U2@@YAXXZ 10025a78     gor.obj
 0002:0001ba9c       __unwindtable$??__EtaskLog@U2@@YAXXZ 10025a9c     gor.obj
 0002:0001baa4       __ehfuncinfo$??__EtaskLog@U2@@YAXXZ 10025aa4     gor.obj
 0002:0001bac8       __unwindtable$??__EuiLog@U2@@YAXXZ 10025ac8     gor.obj
 0002:0001bad0       __ehfuncinfo$??__EuiLog@U2@@YAXXZ 10025ad0     gor.obj
 0002:0001baf4       __unwindtable$??__EuserActLog@U2@@YAXXZ 10025af4     gor.obj
 0002:0001bafc       __ehfuncinfo$??__EuserActLog@U2@@YAXXZ 10025afc     gor.obj
 0002:0001bb20       __ehfuncinfo$?runGORIV@@YAHAAVQFile@@0PADH1AAVU2OpStatus@U2@@@Z 10025b20     gor.obj
 0002:0001bb44       __unwindtable$?runGORIV@@YAHAAVQFile@@0PADH1AAVU2OpStatus@U2@@@Z 10025b44     gor.obj
 0002:0001bb7c       __ehfuncinfo$?readFile@@YAXAAVQFile@@HPAPAD1PAHAAVU2OpStatus@U2@@@Z 10025b7c     gor.obj
 0002:0001bba0       __unwindtable$?readFile@@YAXAAVQFile@@HPAPAD1PAHAAVU2OpStatus@U2@@@Z 10025ba0     gor.obj
 0002:0001bc08       __unwindtable$?Indices@@YAXHPAH0AAVU2OpStatus@U2@@@Z 10025c08     gor.obj
 0002:0001bc20       __ehfuncinfo$?Indices@@YAXHPAH0AAVU2OpStatus@U2@@@Z 10025c20     gor.obj
 0002:0001bc44       __unwindtable$??__EalgoLog@U2@@YAXXZ 10025c44     moc_GorIVAlgTask.obj
 0002:0001bc4c       __ehfuncinfo$??__EalgoLog@U2@@YAXXZ 10025c4c     moc_GorIVAlgTask.obj
 0002:0001bc70       __unwindtable$??__EcmdLog@U2@@YAXXZ 10025c70     moc_GorIVAlgTask.obj
 0002:0001bc78       __ehfuncinfo$??__EcmdLog@U2@@YAXXZ 10025c78     moc_GorIVAlgTask.obj
 0002:0001bc9c       __unwindtable$??__EcoreLog@U2@@YAXXZ 10025c9c     moc_GorIVAlgTask.obj
 0002:0001bca4       __ehfuncinfo$??__EcoreLog@U2@@YAXXZ 10025ca4     moc_GorIVAlgTask.obj
 0002:0001bcc8       __unwindtable$??__EioLog@U2@@YAXXZ 10025cc8     moc_GorIVAlgTask.obj
 0002:0001bcd0       __ehfuncinfo$??__EioLog@U2@@YAXXZ 10025cd0     moc_GorIVAlgTask.obj
 0002:0001bcf4       __unwindtable$??__EperfLog@U2@@YAXXZ 10025cf4     moc_GorIVAlgTask.obj
 0002:0001bcfc       __ehfuncinfo$??__EperfLog@U2@@YAXXZ 10025cfc     moc_GorIVAlgTask.obj
 0002:0001bd20       __unwindtable$??__EscriptLog@U2@@YAXXZ 10025d20     moc_GorIVAlgTask.obj
 0002:0001bd28       __ehfuncinfo$??__EscriptLog@U2@@YAXXZ 10025d28     moc_GorIVAlgTask.obj
 0002:0001bd4c       __unwindtable$??__EtaskLog@U2@@YAXXZ 10025d4c     moc_GorIVAlgTask.obj
 0002:0001bd54       __ehfuncinfo$??__EtaskLog@U2@@YAXXZ 10025d54     moc_GorIVAlgTask.obj
 0002:0001bd78       __unwindtable$??__EuiLog@U2@@YAXXZ 10025d78     moc_GorIVAlgTask.obj
 0002:0001bd80       __ehfuncinfo$??__EuiLog@U2@@YAXXZ 10025d80     moc_GorIVAlgTask.obj
 0002:0001bda4       __unwindtable$??__EuserActLog@U2@@YAXXZ 10025da4     moc_GorIVAlgTask.obj
 0002:0001bdac       __ehfuncinfo$??__EuserActLog@U2@@YAXXZ 10025dac     moc_GorIVAlgTask.obj
 0002:0001bdd0       __sehtable$__onexit        10025dd0     MSVCRT:atonexit.obj
 0002:0001bdf0       __sehtable$___DllMainCRTStartup 10025df0     MSVCRT:crtdll.obj
 0002:0001be18       __sehtable$??_M@YGXPAXIHP6EX0@Z@Z 10025e18     MSVCRT:ehvecdtr.obj
 0002:0001be38       __sehtable$?__ArrayUnwind@@YGXPAXIHP6EX0@Z@Z 10025e38     MSVCRT:ehvecdtr.obj
 0002:0001be58       __sehtable$__IsNonwritableInCurrentImage 10025e58     MSVCRT:pesect.obj
 0002:0001be80       .edata                     10025e80     gor4.exp
 0002:0001bea8       rgpv                       10025ea8     gor4.exp
 0002:0001beac       rgszName                   10025eac     gor4.exp
 0002:0001beb0       rgwOrd                     10025eb0     gor4.exp
 0002:0001beb2       szName                     10025eb2     gor4.exp
 0002:0001bebb       $N00001                    10025ebb     gor4.exp
 0002:0001c894       .idata$6                   10026894     U2Core:U2Core.dll
 0002:0001caac       .idata$6                   10026aac     U2Algorithm:U2Algorithm.dll
 0002:0001cb54       .idata$6                   10026b54     U2View:U2View.dll
 0002:0001cb7e       .idata$6                   10026b7e     Qt5Gui:Qt5Gui.dll
 0002:0001d224       .idata$6                   10027224     Qt5Core:Qt5Core.dll
 0002:0001d2ca       .idata$6                   100272ca     msvcprt:MSVCP120.dll
 0002:0001d3d2       .idata$6                   100273d2     MSVCRT:MSVCR120.dll
 0002:0001d5de       .idata$6                   100275de     kernel32:KERNEL32.dll
 0003:0000000c       _Service_PluginViewer      1002800c     GorIVAlgTask.obj
 0003:00000014       _Service_Project           10028014     GorIVAlgTask.obj
 0003:0000001c       _Service_ProjectView       1002801c     GorIVAlgTask.obj
 0003:00000024       _Service_DNAGraphPack      10028024     GorIVAlgTask.obj
 0003:0000002c       _Service_DNAExport         1002802c     GorIVAlgTask.obj
 0003:00000034       _Service_TestRunner        10028034     GorIVAlgTask.obj
 0003:0000003c       _Service_ScriptRegistry    1002803c     GorIVAlgTask.obj
 0003:00000044       _Service_ExternalToolSupport 10028044     GorIVAlgTask.obj
 0003:0000004c       _Service_GUITesting        1002804c     GorIVAlgTask.obj
 0003:00000054       _Service_WorkflowDesigner  10028054     GorIVAlgTask.obj
 0003:0000005c       _Service_QueryDesigner     1002805c     GorIVAlgTask.obj
 0003:00000064       _Service_MinCoreServiceId  10028064     GorIVAlgTask.obj
 0003:0000006c       _Service_MaxCoreServiceId  1002806c     GorIVAlgTask.obj
 0003:00000074       _Service_PluginViewer      10028074     GorIVPlugin.obj
 0003:0000007c       _Service_Project           1002807c     GorIVPlugin.obj
 0003:00000084       _Service_ProjectView       10028084     GorIVPlugin.obj
 0003:0000008c       _Service_DNAGraphPack      1002808c     GorIVPlugin.obj
 0003:00000094       _Service_DNAExport         10028094     GorIVPlugin.obj
 0003:0000009c       _Service_TestRunner        1002809c     GorIVPlugin.obj
 0003:000000a4       _Service_ScriptRegistry    100280a4     GorIVPlugin.obj
 0003:000000ac       _Service_ExternalToolSupport 100280ac     GorIVPlugin.obj
 0003:000000b4       _Service_GUITesting        100280b4     GorIVPlugin.obj
 0003:000000bc       _Service_WorkflowDesigner  100280bc     GorIVPlugin.obj
 0003:000000c4       _Service_QueryDesigner     100280c4     GorIVPlugin.obj
 0003:000000cc       _Service_MinCoreServiceId  100280cc     GorIVPlugin.obj
 0003:000000d4       _Service_MaxCoreServiceId  100280d4     GorIVPlugin.obj
 0003:00000358       __Tuple_alloc              10028358     GorIVAlgTask.obj
 0003:00000359       _ignore                    10028359     GorIVAlgTask.obj
 0003:0000035a       _allocator_arg             1002835a     GorIVAlgTask.obj
 0003:0000035b       _piecewise_construct       1002835b     GorIVAlgTask.obj
 0003:0000035c       _taskLog                   1002835c     GorIVAlgTask.obj
 0003:00000364       _algoLog                   10028364     GorIVAlgTask.obj
 0003:0000036c       _userActLog                1002836c     GorIVAlgTask.obj
 0003:00000374       _ioLog                     10028374     GorIVAlgTask.obj
 0003:00000380       _coreLog                   10028380     GorIVAlgTask.obj
 0003:0000038c       _uiLog                     1002838c     GorIVAlgTask.obj
 0003:00000394       _scriptLog                 10028394     GorIVAlgTask.obj
 0003:0000039c       _perfLog                   1002839c     GorIVAlgTask.obj
 0003:000003a4       _cmdLog                    100283a4     GorIVAlgTask.obj
 0003:000003b8       ?cvar@?1???0GorIVAlgTask@U2@@QAE@ABVQByteArray@@@Z@4VGReportableCounter@2@A 100283b8     GorIVAlgTask.obj
 0003:000003e0       ?$S1@?1???0GorIVAlgTask@U2@@QAE@ABVQByteArray@@@Z@4IA 100283e0     GorIVAlgTask.obj
 0003:000003e4       __Tuple_alloc              100283e4     GorIVPlugin.obj
 0003:000003e5       _ignore                    100283e5     GorIVPlugin.obj
 0003:000003e6       _allocator_arg             100283e6     GorIVPlugin.obj
 0003:000003e7       _piecewise_construct       100283e7     GorIVPlugin.obj
 0003:000003e8       _taskLog                   100283e8     GorIVPlugin.obj
 0003:000003f0       _algoLog                   100283f0     GorIVPlugin.obj
 0003:000003f8       _userActLog                100283f8     GorIVPlugin.obj
 0003:00000400       _ioLog                     10028400     GorIVPlugin.obj
 0003:00000408       _coreLog                   10028408     GorIVPlugin.obj
 0003:00000410       _uiLog                     10028410     GorIVPlugin.obj
 0003:00000418       _scriptLog                 10028418     GorIVPlugin.obj
 0003:00000420       _perfLog                   10028420     GorIVPlugin.obj
 0003:00000428       _cmdLog                    10028428     GorIVPlugin.obj
 0003:001ab578       __Tuple_alloc              101d3578     gor.obj
 0003:001ab579       _ignore                    101d3579     gor.obj
 0003:001ab57a       _allocator_arg             101d357a     gor.obj
 0003:001ab57b       _piecewise_construct       101d357b     gor.obj
 0003:001ab57c       _taskLog                   101d357c     gor.obj
 0003:001ab584       _algoLog                   101d3584     gor.obj
 0003:001ab58c       _userActLog                101d358c     gor.obj
 0003:001ab594       _ioLog                     101d3594     gor.obj
 0003:001ab59c       _coreLog                   101d359c     gor.obj
 0003:001ab5a4       _uiLog                     101d35a4     gor.obj
 0003:001ab5ac       _scriptLog                 101d35ac     gor.obj
 0003:001ab5b4       _perfLog                   101d35b4     gor.obj
 0003:001ab5bc       _cmdLog                    101d35bc     gor.obj
 0003:001ab5c8       ?Singlet@?1??Parameters@@YAXHPAHPAPAD1AAVU2OpStatus@U2@@@Z@4PAY1BC@BH@MA 101d35c8     gor.obj
 0003:001acfa8       ?Doublet@?1??Parameters@@YAXHPAHPAPAD1AAVU2OpStatus@U2@@@Z@4PAY2IJ@BH@BH@MA 101d4fa8     gor.obj
 0003:002c8138       _allocator_arg             102f0138     nrutil.obj
 0003:002c8139       _piecewise_construct       102f0139     nrutil.obj
 0003:002c813c       __Tuple_alloc              102f013c     moc_GorIVAlgTask.obj
 0003:002c813d       _ignore                    102f013d     moc_GorIVAlgTask.obj
 0003:002c813e       _allocator_arg             102f013e     moc_GorIVAlgTask.obj
 0003:002c813f       _piecewise_construct       102f013f     moc_GorIVAlgTask.obj
 0003:002c8140       _taskLog                   102f0140     moc_GorIVAlgTask.obj
 0003:002c8148       _algoLog                   102f0148     moc_GorIVAlgTask.obj
 0003:002c8150       _userActLog                102f0150     moc_GorIVAlgTask.obj
 0003:002c8158       _ioLog                     102f0158     moc_GorIVAlgTask.obj
 0003:002c8160       _coreLog                   102f0160     moc_GorIVAlgTask.obj
 0003:002c8168       _uiLog                     102f0168     moc_GorIVAlgTask.obj
 0003:002c8170       _scriptLog                 102f0170     moc_GorIVAlgTask.obj
 0003:002c8178       _perfLog                   102f0178     moc_GorIVAlgTask.obj
 0003:002c8180       _cmdLog                    102f0180     moc_GorIVAlgTask.obj
 0003:002c8188       __Tuple_alloc              102f0188     moc_GorIVPlugin.obj
 0003:002c8189       _ignore                    102f0189     moc_GorIVPlugin.obj
 0003:002c818a       _allocator_arg             102f018a     moc_GorIVPlugin.obj
 0003:002c818b       _piecewise_construct       102f018b     moc_GorIVPlugin.obj
 0003:002c8190       ___proc_attached           102f0190     MSVCRT:crtdll.obj
 0003:002c8198       _GS_ExceptionRecord        102f0198     MSVCRT:gs_report.obj
 0003:002c81e8       _GS_ContextRecord          102f01e8     MSVCRT:gs_report.obj
 0003:002c84b4       _DebuggerWasPresent        102f04b4     MSVCRT:gs_report.obj
 0004:00000060       $R000000                   102f1060     * linker generated manifest res *

 Exports

  ordinal    name

        1    _ugene_plugin_init
               exported name: ugene_plugin_init
